:020000040800F2
:10000000000001108DC3030835860308C1D700081E
:1000100091C4030891C4030891C4030800000000C0
:100020000000000000000000000000007D8C0308BC
:10003000798C030800000000758C0308CDED0008E2
:1000400091C4030891C4030891C4030891C4030830
:1000500091C4030891C40308F99A0008259C00087C
:10006000E99B0008AD9B0008719B0008B9BA000825
:10007000A9BA000899BA000889BA000879BA000834
:1000800065BA000851BA000891C4030891C4030876
:1000900091C4030891C4030891C40308359B000868
:1000A00091C4030891C4030891C4030891C40308D0
:1000B00009DF0008F9DE000891C40308D5C2000872
:1000C000DDC20008C9C20008D1C2000891C40308FB
:1000D00091C403081D90000891C40308818F000893
:1000E000BD9A000891C40308998C0308B9DE000882
:1000F000C9DE000891C40308D9DE00083DBA000833
:1001000091C4030891C40308E9DE000891C4030800
:10011000F5EE000891C4030885AC010869AC01083C
:1001200029BA000815BA000801BA0008EDB900089C
:10013000D9B9000891C4030891C4030891C4030805
:1001400091C4030891C4030891C4030839860308C5
:10015000C5B90008B1B900089DB9000859EE0008FA
:10016000BDC20008C5C2000891C4030891C40308B9
:1001700091C4030891C4030891C4030891C40308FF
:0801800091C4030891C40308B7
:1001880002020300DC1F0020D81F0020000000002E
:100198000000000016000800E81F0020F01F0020E3
:1001A8000000000024060008030001008C2600203F
:1001B8009426002000000000000000000101040057
:1001C800D8260020643A002000000000000000004B
:1001D80008020900A2390020683A00200000000047
:1001E8002982000806020C00183A0020743A002000
:1001F80000000000B18D0008070202004C3A002000
:10020800803A0020000000002C06000802000C00C4
:10021800243A0020843A002000000000000000007A
:10022800F70106009C390020903A002000000000E9
:100238002E0600080A020A0068270020983A0020C3
:1002480000000000340600080312330003420020B7
:10025800D0410020000000004006000825005A0098
:100268001C41002076410020000000000000000032
:10027800F6110C001041002004410020000000008D
:10028800740600082F00110038420020F0400020BA
:10029800000000008006000828000C006C480020C0
:1002A8008C48002000000000920600082900500039
:1002B80000480020984800200000000000000000CE
:1002C80014000200FC470020E8480020000000005D
:1002D8009E0600082C001000784D0020684D002074
:1002E800000000000D4C02082B002400AC4D00203B
:1002F800884D002000000000DD4B0208230010009C
:10030800FC4C0020D04D002000000000D94202081B
:100318001D000100F44D0020884E00200000000060
:10032800A006000819000500E04D00208C4E0020B2
:1003380000000000A2060008000104007C4E002016
:10034800944E002000000000A806000827000400C2
:10035800144E0020984E002000000000AC06000853
:100368001F000E00E04F00201C500020000000007D
:10037800B006000805020100C84F00202C500020DC
:1003880000000000BE060008030106005A4F0020C6
:100398003050002000000000C006000800020500E0
:1003A80038500020A053002000000000000000008A
:1003B8001E00040078510020A8530020000000000F
:1003C800C606000822000C00F8500020AC5300209C
:1003D80000000000CA06000801200800E05B0020B9
:1003E800E85B002000000000D60600081A0008009C
:1003F800C45B0020F05B002000000000DE0600085F
:10040800F8110100905A0020F85B0020000000005D
:10041800E60600082A0060005C5C0020FC5B002007
:100428000000000039BA0208150070004855002085
:10043800BC5C0020000000000000000004008000F8
:1004480050780020047A002000000000000000001E
:10045800F9010400506D0020847A0020000000009B
:10046800118200080D003C005C8D0020988D002052
:100478000000000085D9010811000C00F08100205F
:10048800D48D00200000000039D90108FA010200CB
:100498002C7B0020E08D002000000000E5C3000850
:1004A800FD012400F87A0020E48D002000000000FF
:1004B800A1810008FE010800E47A0020088E0020CF
:1004C80000000000D9C300081B00F400188E0020AB
:1004D800B8900020000000008D9F020826000E0042
:1004E800BC910020AC91002000000000010103082D
:1004F80009020100389200209092002000000000BC
:10050800E806000812100C00F191002094920020D7
:1005180000000000EA0600080C00240004920020F5
:10052800A0920020000000002DA20108050006008E
:100538000A94002014A1002000000000F80600081A
:100548000E20EA00EE9200201CA10020000000000E
:10055800A5BA0208130004002494002008A2002071
:10056800000000000007000802010300D9920020E3
:100578000CA200200000000055A2010818102C0051
:1005880070A800209CA80020000000003158020834
:10059800FB01010034A80020C8A8002000000000CA
:1005A800D1C30008FC01090000A70020CCA8002046
:1005B800000000009DC300080A101200D4A6002005
:1005C800D8A8002000000000040700080600160054
:1005D800A4A30020ECA8002000000000C5BA02086F
:1005E8003400100010A2002004A900200000000020
:1005F80061BA02080B20100044AD00207CAD002039
:10060800000000001607000810000300F8AD0020E5
:0C06180000AE00200000000026070008D3
:10062400C409000019012828013C00000100000051
:1006340000004A01B400D6010000000000000000E0
:1006440000000000000000000000000000000000A6
:100654000000000000000000000000000000000096
:100664000000000000000000000000000000010085
:100674000000000000000000000000000000000076
:100684000000000000000000000000000000000066
:100694000001000000000000000003000000000052
:1006A4002801000090010000200300000000000069
:1006B400000001000000000500000000040101002A
:1006C400000000000100C800141E010064002C0199
:1006D4002800E8036400040A00017E05EA05B40565
:1006E400320004002E00000000010005504F444970
:1006F40000000000200003000100000008040000C6
:1007040000300100005A0000000090012C01C800D4
:1007140064002B21231E64000200000001000A0172
:050724002900000105A1
:100729005001000007000000020000000000803FA7
:100739000000803F0000803F000000000000000032
:100749000102030406070809010100000421040845
:10075900AC4904080000000000000000142104084E
:100769001C210408000000000120000020210408C9
:100779002821040800000000014000002C21040881
:100789008439040800000000012000003821040811
:100799004421040800000000040000004821040866
:1007A9005421040800000000040000005821040836
:1007B9001C4F0408000000000100000002010000B5
:1007C900685E0C00FF0000000000803F48F303084A
:1007D9000508040000000000A81D0408441D0408C1
:1007E90034F303080000000074F3030805080A0045
:1007F90000000000A81D0408441D0408F41D040895
:1008090000000000D184030889840308D983030800
:1008190000000000C98003084D820308CD82030847
:10082900B58103080000000000000000BD80030836
:10083900A18003089D800308998003088D8003081F
:10084900898003089580030891800308B180030813
:10085900A58003088D810308A18103087981030814
:100869006581030851810308FFFFFFFF00010101B2
:1008790001010000594802080000000000000000C2
:10088900010000000000803F303030302D30312D24
:1008990030315430303A30303A30300000FFFF0008
:1008A90000000000AA5503009FAA5505010000AAEF
:1008B900550701000001AA550B010000AA550902BC
:1008C9000000000001000000C01200000000803F8D
:1008D9000000803F006002401060024000000000FC
:1008E900000B0000000020000000000000000000D4
:1008F900006002402860024000000000060C000071
:10090900000020000000000000000000006002401C
:100919004060024000000000100D000000002000AF
:100929000000000000000000006002405860024022
:1009390000000000160E000000002000000000006A
:1009490000000000006002407060024000000000EA
:10095900200F00000000200000000000000000003F
:10096900006002408860024000000000261000007C
:1009790000002000000000000000000000600240AC
:10098900A0600240000000003011000000002000BB
:10099900000000000000000000600240B860024052
:1009A90000000000362F00000000200000000000B9
:1009B90000000000006402401064024000000000D2
:1009C90000380000000040000000000000000000A6
:1009D900006402402864024000000000063900005B
:1009E9000000400000000000000000000064024018
:1009F9004064024000000000103A0000000040007E
:100A09000000000000000000006402405864024039
:100A190000000000163B000000004000000000003C
:100A29000000000000640240706402400000000001
:100A3900203C000000004000000000000000000011
:100A4900006402408864024000000000264400005F
:100A590000004000000000000000000000640240A7
:100A6900A064024000000000304500000000400082
:100A7900000000000000000000640240B864024069
:100A890000000000364600000000400000000000A1
:100A9900000000000000000100000000000000004C
:100AA9000000000000000101FFFF000044400408AD
:100AB900000000000000000069A20108A0860100F2
:100AC9000400000000000000000000000000000019
:100AD900000000000000000000000000000000000D
:100AE900F4450408983F040800000000415C01082F
:100AF9007D0000000600000000000000000000006A
:100B090000000000000000000000000000000000DC
:100B190000000000804F04080000000000000000F1
:100B2900497A0308E8030000030000000000000000
:100B390000000000000000000000000000000000AC
:100B49000000000000000000884F040800000000B9
:100B590000000000CDBB02081027000003000000C0
:100B6900000000000000000000000000000000007C
:100B7900000000000000000000000000A05404086C
:100B890000000000654A0208313D0108204E0000BE
:100B99000500000000000000000000000000000047
:100BA900000000000000000000000000000000003C
:100BB900B8410408000000000000000005750308A2
:100BC90010270000010000000000000000000000E4
:100BD900000000000000000000000000000000000C
:100BE90000000000944F040800000000000000000D
:100BF90069C30008E80300000500000000000000C8
:100C090000000000000000000000000000000000DB
:100C19000000000000000000A04F040800000000D0
:100C2900000000008DA40108204E00000300000010
:100C390000000000000000000000000000000000AB
:100C4900000000000000000000000000B04F040890
:100C5900000000000000000095A20108204E0000DD
:100C69000300000000000000000000000000000078
:100C7900000000000000000000000000000000006B
:100C8900C04F04080000000000000000957203082E
:100C9900400D0300030000000000000000000000F8
:100CA900000000000000000000000000000000003B
:100CB90000000000F84004080000000000000000E7
:100CC900C9F201081027000001000000000000001F
:100CD900000000000000000000000000000000000B
:100CE9000000000000000000B43F040800000000FC
:100CF9000000000011B002081027000003000000E6
:100D090000000000000000000000000000000000DA
:100D1900000000000000000000000000D04F04089F
:100D29000000000000000000BD3B0108A086010092
:100D390001000000000000000000000000000000A9
:100D4900000000000000000000000000000000009A
:100D5900A43F04080000000000000000DD3A01087B
:100D690050C3000001000000000000000000000066
:100D7900000000000000000000000000000000006A
:100D890000000000D84F0408000000000000000027
:100D990045360108A86100000100000000000000BC
:100DA900000000000000000000000000000000003A
:100DB9000000000000000000E44F040800000000EB
:100DC900000000005DB80208A086010001000000D3
:100DD900000000000000000000000000000000000A
:100DE900000000000000000000000000C0410408ED
:100DF900000000000000000091EF0008A00F0000B3
:100E090001000000000000000000000000000000D8
:100E190000000000000000000000000000000000C9
:100E2900F04F040800000000000000000905030855
:100E39001027000001000000000000000000000071
:100E49000000000000000000000000000000000099
:100E5900000000002041040800000000000000001C
:100E690069D80108A00F000001000000000000007F
:100E79000000000000000000000000000000000069
:100E890000000000000000002442040800000000E7
:100E990000000000618D0208102700000100000019
:100EA9000000000000000000000000000000000039
:100EB9000000000000000000000000008C3F040852
:100EC9000000000000000000816703081A410000CB
:100ED9000100000000000000000000000000000008
:100EE90000000000000000000000000000000000F9
:100EF900FC4F0408000000000000000051B703087F
:100F0900400D030000000000000000000000000088
:100F190000000000000000000000000000000000C8
:100F29000000000004500408000000000000000058
:100F39000DB70308400D0300000000000000000089
:100F49000000000000000000000000000000000098
:100F590000000000000000000C5004080000000020
:100F69000000000095A60108A0860100030000000A
:100F79000000000000000000000000000000000068
:100F89000000000000000000000000000101010055
:100F9900445304080E000000A52A030800000000BD
:100FA90000000000F00900200853040800000000B8
:100FB900000000000000000000000000AC49040827
:100FC90000000000000000007C0A0020040000006E
:100FD900945204080C00000075300308900E00209C
:100FE90000000000B85104080C0000004530030857
:100FF900840E0020000000002853040808000000A7
:1010090000000000780E00200400000018530408B6
:101019000C0000005D2F03086C0E0020000000008A
:10102900A45104080300000059660308540E002067
:10103900000000002053040803000000596603085B
:101049003C0E002000000000A85104080100000027
:101059000000000000000000000000000000000087
:101069000D0000000000000000000000000000006A
:101079000853040800000000000000000000000000
:1010890000000000AC490408000000000000000056
:101099007C0A002004000000385204080300000004
:1010A900012F0308240E002008000000185304082B
:1010B9000C0000005D2F03086C0E002000000000EA
:1010C900A45104080300000059660308540E0020C7
:1010D90000000000205304080300000059660308BB
:1010E9003C0E002000000000A85104080100000087
:1010F90000000000000000000000000000000000E7
:101109000D000000000000000000000000000000C9
:101119003053040800000000000000000000000037
:1011290000000000AC4904080000000000000000B5
:101139007C0A00200400000040520408030000005B
:10114900596603089C0E002000000000A8510408FD
:101159000100000000000000000000000000000085
:10116900000000000D000000000000000000000069
:101179000000000020700020702D72002D202D2D00
:10118900202D2D2D2D202D2D2D2D000000000000AE
:101199000000000000000000000000002D202D2D9F
:1011A900202D2D2D2D202D2D2D00000000000000BB
:1011B900000000000000000000000000D2920020A2
:1011C90088130C1701000000D492002088130C1713
:1011D900000000007C51040800000000000000002D
:1011E90000000000000000008C5104080800000005
:1011F90000000000A80A002004000000985104081B
:1012090008000000000000009C0A00200000000007
:10121900A451040804000000412F03080000000045
:1012290000000000A85104080100000000000000AF
:101239000000000000000000000000000D00000098
:10124900000000000000000000000000D092002013
:1012590088130C1701000000CE92002088130C1788
:1012690000000000E85104080E000000FD2A0308F0
:101279000000000000000000B40A002022940020B1
:1012890001000000681D0408CD9200200100000043
:10129900741D0408C44F0020020000007C1D0408CE
:1012A90016790020000000000000000014790020D9
:1012B900000000000000000012790020000000007A
:1012C900000000001079002000000000000000006C
:1012D9000E79002000000000000000000C790020B9
:1012E9000000000000000000A8010020000000002C
:1012F90000000000CC92002002000000881D0408B4
:10130900F051040800000000000000000000000087
:10131900000000008C5104080800000000000000D3
:10132900380B002004000000985104080800000050
:10133900000000002C0B002000000000A45104084C
:1013490004000000DD2A030800000000000000007E
:10135900A85104080100000000000000000000007E
:1013690000000000000000000D0000000000000067
:101379000000000000000000005204080000000006
:1013890000000000000000000000000010520408E6
:101399000C000000E52F0308740B00200400000076
:1013A9001C5204080C000000212B0308680B0020C4
:1013B90004000000285204080C000000A52F0308AF
:1013C9005C0B0020000000003452040803000000F8
:1013D900212F0308440B0020080000004052040894
:1013E90003000000596603089C0E0020000000005D
:1013F900A8510408010000000000000000000000DE
:1014090000000000000000000D00000000000000C6
:10141900000000000000000048520408000000001D
:101429000000000000000000000000005052040805
:1014390004000000A53003080000000000000000BF
:10144900A85104080100000000000000000000008D
:1014590000000000000000000D0000000000000076
:1014690000000000000000009C5204080000000079
:10147900000000000000000000000000B84204085D
:101489000C00000000000000D40B00200400000044
:10149900AC5204080800000000000000C80B00203E
:1014A90004000000B8520408080000000000000011
:1014B900BC0B002004000000C05204080800000012
:1014C90000000000B00B002004000000C85204080E
:1014D9000800000000000000A40B00200400000028
:1014E900D05204080800000000000000980B0020FA
:1014F90004000000D85204080800000000000000A1
:101509008C0B002004000000E052040808000000D1
:1015190000000000800B002004000000A85104080E
:1015290001000000000000000000000000000000B1
:10153900000000000D000000000000000000000095
:1015490000000000E85204080E000000ED2A03081C
:101559000000000000000000E00B0020F052040829
:101569000E00000000000000000000000000000064
:10157900580C0020F85204080E000000000000007A
:101589000000000000000000F80C00202194002059
:1015990004000000941D0408C8920020E0150C17EF
:1015A90000000000CB92002008000000441D040840
:1015B900CA92002005000000A81D04080053040871
:1015C9000E00000000000000000000000000000004
:1015D900480D002001000000000000000102030482
:1015E9000102030406070809D85804080E00000080
:1015F900000000000000000000000000B41C0020F2
:10160900FFFFFFFFFA0000000100000001000000D9
:10161900485204080000000000000000000000001B
:10162900000000006E53040804000000932E030814
:101639000000000000000000A8510408010000009B
:101649000000000000000000000000000000000091
:101659000D00000000000000000000000000000074
:10166900BA7900200100C40900000000B8790020FF
:101679000100C40900000000B67900200100C40976
:1016890000000000B47900200100C4090000000036
:10169900B07900200100C40900000000B2790020DF
:1016A9000100C40900000000AE7900200100C4094E
:1016B90000000000AC7900200100C409000000000E
:1016C900985304080E00000000000000000000000C
:1016D90000000000F00E0020984F00209CFF2C0114
:1016E900000000006E0800200A000000F41D040834
:1016F900C4920020E0150C17000000006D080020BE
:1017090008000000441D04086C08002005000000C2
:10171900A81D0408C6920020020000000C1E04083F
:10172900109400200100FF7F0100000008940020B0
:1017390002000000181E0408E292002003000000C5
:10174900281E0408E192002003000000281E040856
:10175900E09300200000F40101000000DE93002066
:101769000000F40101000000DC9300200000F401F6
:1017790001000000DA9300200000F40101000000DC
:10178900D893002000FF0100F4930020E803D0075C
:101799000A000000F2930020006401000A00000022
:1017A900F3930020006401000A000000EC9300207C
:1017B900006401000A000000F193002000640100A8
:1017C9000A000000F0930020006401000A000000F4
:1017D900EF930020006401000A000000EB93002051
:1017E90000FF01000A000000EA93002000FF010049
:1017F9000A000000EA9200200000F4010100000044
:10180900E89200200000F40101000000E6920020A7
:101819000000F40101000000E49200200000F4013E
:1018290001000000E793002000C80100E6930020B2
:1018390000C80100E593002000C80100E4930020DE
:10184900006401000A000000E393002000FF01008A
:101859000A000000FF93002000C80100FE93002049
:1018690000C80100FD93002000C80100FC9300207E
:1018790000C80100FB93002000C80100FA93002072
:1018890000C80100F993002000C80100F893002066
:1018990000C80100F793002000C80100A053040804
:1018A900000000000000000000000000000000002F
:1018B900B05304080900000000000000940F002044
:1018C90004000000B85304080900000000000000EB
:1018D900880F002004000000745704080900000064
:1018E900000000007C0F00200400000028510408BB
:1018F9000900000000000000700F00200400000033
:10190900C05304080900000000000000640F002013
:1019190004000000C853040809000000000000008A
:10192900580F002004000000D053040809000000EB
:10193900000000004C0F002004000000D8530408E8
:101949000900000000000000400F00200400000012
:10195900A851040801000000000000000000000078
:1019690000000000000000000D0000000000000061
:101979000000000000000000B0540408000000004E
:10198900000000000000000000000000C05404082E
:101999000500000000000000E092002000000000A7
:1019A900A851040801000000000000000000000028
:1019B90000000000000000000D0000000000000011
:1019C9000000000000000000C854040800000000E6
:1019D900000000000000000000000000AC490408FD
:1019E90000000000000000005C0A00200400000064
:1019F900245104080C000000D92E0308F40F00201C
:101A090000000000945204080C000000512A030849
:101A1900E80F002000000000B85104080C00000085
:101A29001D2A0308DC0F00200000000028530408C9
:101A39000800000000000000D00F00200400000092
:101A4900185304080C000000092A0308C40F0020D9
:101A590000000000D4540408090000000000000040
:101A6900B80F002004000000A4510408030000007E
:101A790059660308A00F002000000000A8510408BF
:101A8900010000000000000000000000000000004C
:101A9900000000000D000000000000000000000030
:101AA90000000000DC5404080000000000000000F1
:101AB9000000000000000000EC5404080C000000C5
:101AC900000000000C10002000000000F45404087D
:101AD9000A00000000000000289400200000000017
:101AE900005504080A00000000000000309400209E
:101AF90000000000085504080A000000000000006A
:101B09003894002000000000105504080800000067
:101B19000000000000100020000000001855040813
:101B2900040000000D33030800000000000000005D
:101B3900A851040801000000000000000000000096
:101B490000000000000000000D000000000000007F
:101B590000000000000000002455040800000000F7
:101B690000000000000000000000000038550408D3
:101B79000C000000000000002410002000000000FC
:101B890048550408040000006931030800000000FA
:101B990000000000505504080C000000000000007F
:101BA900181000200000000064550408040000001B
:101BB900493103080000000000000000A851040892
:101BC900010000000000000000000000000000000B
:101BD900000000000D0000000000000000000000EF
:101BE900000000006C55040800000000000000001F
:101BF90000000000000000008055040807000000F4
:101C09000000000060100020000000008C5504084E
:101C1900080000000000000054100020000000002F
:101C29009855040808000000000000004810002032
:101C390000000000A455040808000000000000008E
:101C49003C10002000000000B05504080800000006
:101C5900000000003010002000000000A851040816
:101C6900010000000000000000000000000000006A
:101C7900000000000D00000000000000000000004E
:101C890000000000BC55040800000000000000002E
:101C9900570A002000000000C85504080B00000086
:101CA90000000000C810002000000000D055040802
:101CB9000B00000000000000BC1000200000000024
:101CC900DC5504080B00000000000000B0100020E3
:101CD90000000000E85504080B00000000000000A7
:101CE900A410002000000000F45504080B000000B7
:101CF90000000000981000200000000000560408B1
:101D09000B000000000000008C1000200000000003
:101D1900085604080B000000000000008010002095
:101D290000000000145604080B0000000000000029
:101D3900741000200000000020560408080000006C
:101D4900000000006810002000000000A8510408ED
:101D59000100000000000000000000000000000079
:101D6900000000000D00000000000000000000005D
:101D7900000000002C5604080000000000000000CC
:101D890000000000000000004056040808000000A0
:101D990000000000F8100020000000004C56040864
:101DA9000800000000000000EC1000200000000006
:101DB900585604080800000000000000E010002048
:101DC900000000006456040808000000000000003C
:101DD900D410002000000000A851040801000000F0
:101DE90000000000000000000000000000000000EA
:101DF9000D000000000000000000000000000000CD
:101E09006C5604080000000000000000540A00207D
:101E1900000000007C5604080B00000000000000D0
:101E29002811002000000000885604080B0000005B
:101E3900000000001C110020000000009456040856
:101E4900070000000000000014110020000000003D
:101E5900A056040807000000000000000C11002033
:101E690000000000AC560408070000000000000054
:101E79000411002000000000A8510408010000001E
:101E89000000000000000000000000000000000049
:101E99000D0000000000000000000000000000002C
:101EA900B85604080000000000000000540A002091
:101EB90000000000C45604080700000000000000EC
:101EC9007411002000000000CC560408070000002F
:101ED900000000006C11002000000000D456040826
:101EE900070000000000000064110020000000004D
:101EF900DC56040807000000000000005C11002007
:101F090000000000E456040807000000000000007B
:101F19005411002000000000EC56040807000000DE
:101F2900000000004C11002000000000F4560408D5
:101F3900070000000000000044110020000000001C
:101F4900FC56040807000000000000003C110020B6
:101F5900000000000457040807000000000000000A
:101F69003411002000000000A851040801000000FD
:101F79000000000000000000000000000000000058
:101F89000D0000000000000000000000000000003B
:101F99000C5704080E00000000000000DD2B0308A8
:101FA900000000007C110020DE92002017000000D4
:101FB900381E0408DD9200200A320100DC9200205C
:101FC90001FA0100D892002000C80100D692002031
:101FD900E803D00701000000504F4449554D4634ED
:101FE90000000000145704080E000000F32B03083A
:101FF900000000001D310308581200201C57040876
:102009000E0000006929030800000000000000001C
:10201900A8120020245704080E000000ED3203081E
:10202900392E0308352E0308841300202C57040881
:102039000E000000152C030800000000000000003D
:1020490038140020345704080E000000A52C03089A
:10205900752C030800000000C41400203C57040834
:102069000E000000212D0308692D0308000000005F
:1020790064150020E8930020010301004857040873
:102089000E000000492C0308252C0308000000005D
:1020990054160020505704080E000000D52C0308E0
:1020A9008931030800000000E01600205C5704088D
:1020B9000E000000992D0308D53103080000000027
:1020C90080170020E29300200103010064570408EF
:1020D90000000000000000000000000000000000F7
:1020E900705704080800000000000000AC18002028
:1020F90000000000785704080700000000000000F5
:10210900A4180020000000008857040807000000F8
:10211900000000009C1800200000000094570408EB
:1021290007000000000000009418002000000000D3
:10213900A05704080C0000000000000088180020C7
:1021490000000000AC5704080300000059660308AA
:102159007018002000000000A851040801000000C8
:102169000000000000000000000000000000000066
:102179000D00000000000000000000000000000049
:10218900B45704080000000000000000000000002F
:1021990000000000C45704080A0000000000000005
:1021A9006421040800000000CC5704080A0000005C
:1021B90000000000E420040800000000D4570408CF
:1021C9000A00000000000000009400200000000048
:1021D900DC5704080A00000000000000B8180020BD
:1021E90000000000A85104080100000000000000E0
:1021F9000000000000000000000000000D000000C9
:10220900000000000000000000000000E45704087E
:1022190000000000000000000000000000000000B5
:10222900F85704080300000059660308F418002051
:102239000000000004580408030000005966030860
:1022490070080020000000000C580408030000007A
:1022590059660308DC18002000000000145804081F
:102269000300000059660308C4180020000000009C
:10227900A85104080100000000000000000000004F
:1022890000000000000000000D0000000000000038
:1022990000000000000000002058040800000000B1
:1022A9000000000000000000000000002C58040895
:1022B9000700000021320308A419002000000000D3
:1022C900F445040803000000596603088C1900202E
:1022D900000000003858040803000000596603088C
:1022E9007419002000000000405804080300000091
:1022F900596603085C1900200000000048580408CA
:1023090007000000053203085419002000000000EE
:10231900B052040803000000596603083C19002064
:10232900000000005458040803000000596603081F
:102339002419002000000000605804080300000070
:10234900596603080C19002000000000A851040870
:102359000100000000000000000000000000000073
:10236900000000000D000000000000000000000057
:10237900000000006C5804080E000000A52B03089B
:102389006D2B030800000000AC19002074580408E4
:102399000E000000092E03080000000000000000E4
:1023A900601A0020805804080E0000000000000098
:1023B9000000000000000000EC1A002090580408FA
:1023C9000E000000E12D03083D3203080000000063
:1023D900781B002098580408000000000000000045
:1023E9000000000000000000884804080300000005
:1023F900596603089C1C002000000000845804084A
:102409000300000059660308841C00200000000036
:10241900A458040803000000596603086C1C002036
:1024290000000000B05804080300000059660308C2
:10243900541C002000000000B858040802000000E5
:10244900716503080000000000000000C05804087E
:10245900020000007165030801000000000000008F
:10246900CC5804080200000071650308020000004E
:1024790000000000000000000D0000000000000046
:10248900000000000000000004030904120100021A
:1024990002020040830440570002010203010000C8
:1024A90009024300020100C03209040000010202CE
:1024B9000100052400100105240100010424020281
:1024C9000524060001070582030800FF090401002D
:1024D900020A000000070501024000000705810209
:1024E90040000000FF000000B9850308F9820308D5
:1024F900295B03080D810308658503081D8103080D
:1025090039810308FD800308ED80030800000000FD
:10251900000000000100000043000000000000006E
:1025290000000000000000000000000000000000A2
:10253900000000000000000043000000000000004F
:102549000000000000000000000000000000000082
:10255900000000000000000043000000000000002F
:102569000000000000000000000000000000000062
:10257900000000000000000043000000000000000F
:102589000000000000000000000000000000000042
:1025990000000000000000004300000000000000EF
:1025A9000000000000000000000000000000000022
:1025B90000000000000000004300000000000000CF
:1025C9000000000000000000000000000000000002
:1025D90000000000000000004300000000000000AF
:1025E90000000000000000000000000000000000E2
:1025F9000000000000000000FDC603083DC50308F7
:1026090000000000F25A0408695304083A24040837
:102619003A2404083A2404083A2404083A24040809
:102629003A2404083A2404083A2404083A240408F9
:10263900FFFFFFFFFFFFFFFFFFFFFFFFFFFF00009F
:102649000100415343494900000000000000000017
:102659000000000000000000000000000000000071
:1026690000004153434949000000000000000000F8
:102679000000000000000000000000000000000051
:1026890000000000681F002000000000000000009A
:102699000000000000000000000000000000000031
:1026A9000000000000000000000000000000000021
:1026B9000000000000000000000000000000000011
:1026C9000000000000000000000000000000000001
:1026D90000000000000000000000000000000000F1
:0C26E900000000000000000001000000E4
:1080000070B4EFF31186502383F31288436B1A6820
:10801000D20720D45D686DB9446A826A944217D051
:1080200081691144D9600ED9A21A5A608462002273
:1080300080F858201A6842F00102F1B21A6081F308
:10804000118870BC704701698A1A5A608562EEE730
:10805000012380F85830F3B283F3118870BC704765
:10806000436A8269D154436A0169426B01338B428E
:1080700028BF00234362002A2FD0EFF31182502340
:1080800083F31288436B1968C9072CD470B45E68F7
:108090006EB9456A816A8D4217D084690C44DC60F0
:1080A0000ED9691A59608562002180F85810196844
:1080B00041F00101D2B2196082F3118870BC70479F
:1080C0000469611A59608662EEE7012380F858302E
:1080D000D2B282F3118870BC7047426DD36843F00E
:1080E0008003D3607047D2B282F31188704700BF1B
:1080F000026B10B462B1836CC2684469D11A013B4F
:10810000615C5DF8044B08BF13468364C8B27047D6
:10811000016A4369C4685B5C0131A14228BF114612
:1081200001625DF8044BD8B2704700BF436B13B1D6
:1081300090F858007047836A406A181AB0FA80F0C5
:1081400040097047416A836A99420AD3CB1A416B4E
:10815000026961B14968501E0B4483420AD2C01AB9
:10816000704702691144CB1A416B0029F2D1501EAD
:10817000C01A704700207047036B43B1826C5B6884
:1081800093422FBF981AC0689B1AC0187047C269E3
:10819000036A9A422FBFD01AC0688018C01A70476D
:1081A0000A4B30B503F1180493F900205D78072AD3
:1081B000C8BF143A811804330D7313F8025C855458
:1081C00013F8012C0A76A342EED130BDCCEB0308A4
:1081D00003682DE9F041DF691FB13B46BDE8F0417E
:1081E0001847002A164611DD04460D460E4400E0ED
:1081F00023689B68204698470028F9D0236815F823
:10820000011B1B6820469847AE42F1D1BDE8F081C2
:1082100010B424212524262200230470417082708A
:10822000C3705DF8044B7047152303701623C370A9
:10823000172383713A2383703B2343713C230372DA
:10824000704700BF30B4846814B12368A5885D838B
:10825000436840F2E93001E0002832D01D8901383E
:1082600015F0020F80B2F7D089B2998140F2E9315E
:1082700001E0002947D01889013910F0010F89B2B7
:10828000F7D0998940F2E93100E059B318890139F2
:1082900010F0020F89B2F8D092B29A8140F2E9321E
:1082A00001E0002A3FD01989013A11F0010F92B282
:1082B000F7D09B8914B12368A2881A83012030BCAF
:1082C000704721498B4204D0A1F574418B42D9D12A
:1082D00002201E4901EB00104189013189B2418120
:1082E0004189CFE7184A934204D0A2F574429342E1
:1082F000E0D10221154B03EB01114B8901339BB2F5
:108300004B814B89D6E71048834203D010498B42FA
:10831000B8D102210D4800EB01114889013080B22B
:1083200048814989AEE708498B4203D0084A934205
:10833000C0D10222054B03EB0212538901339BB2D9
:1083400053815389B6E700BF0030014014AE0020CE
:10835000003C0040002870B51EDB0928044620DDE3
:10836000012303EB83035B00B0FBF3F2092AF8D887
:108370007BB10E4EB4FBF3F00928CCBF572230225C
:10838000A6FB03E5024403FB1044EB0801F8012BB4
:10839000F0D100230B7070BD2D230B7040420131D2
:1083A000DBE7303001F8010BF3E700BFCDCCCCCCDC
:1083B000884230B44FF001042ED301FB04F4B0FB2B
:1083C000F4F58D42F9D284B1AAB901E0B0FBF4F51D
:1083D000092DCCBF572230222A4404FB150003F894
:1083E000012BB4FBF1F4002CF0D100221A7030BC48
:1083F0007047B0FBF4F5092DCCBF372230222A4458
:1084000004FB150003F8012BB4FBF1F4002CF0D1B0
:1084100000221A7030BC70470546002AEBD1D7E71E
:1084200003685A1C02601970704700BF2DE9F047BD
:10843000089C2578002B804689460CBF4FF0200A07
:108440004FF0300A661C35B3002A29DD334601E0BF
:10845000024698B113F8011B501E0029F8D1971E4F
:1084600060B13D46013D51464046C8476B1C002B5C
:10847000F8DC257827EAE770013055B1041B29465E
:108480004046C847301916F8015B002DF7D1BDE80A
:10849000F087BDE8F087002A04DC2846BDE8F087B5
:1084A0000020EBE7571EDCE783684268D0ED037AD3
:1084B00000EB83010133934281ED040A836004BF22
:1084C0000023836000EB830393ED047A036870EE6E
:1084D000277A9A42C0ED037A77EEC77AC0ED037A25
:1084E0000CDA013307EE103AF8EEC76AB7EE007AFD
:1084F00087EEA60A036030EE070A704707EE102ADF
:10850000B8EEC77A87EE870A704700BF90ED057A0C
:1085100090ED004AD0ED066AD0ED014AD0ED047A24
:1085200090ED035AD0ED025AA4EE007AB0EE406A04
:10853000B0EE470AB0EE667AA6EE247A67EEC07A0D
:10854000A0EE457AE6EE257A80ED057AC0ED067A52
:10855000704700BFD0ED057A90ED013AD0ED003ABA
:10856000D0ED064A90ED024A90ED077A90ED035A5D
:1085700090ED086AD0ED045AC0ED067AF0EE406A3C
:1085800027EE830AC0ED056AA3EEA60A80ED087AFD
:10859000A4EE240AA5EE470AA5EEC60A80ED070A56
:1085A000704700BFD0ED007A90ED017A30EE670A97
:1085B000E7EE007AB0EE670AC0ED007A704700BFC0
:1085C000704700BF0A44914214D030B40139551E9F
:1085D00041F2210211F8014F082380EA042004042B
:1085E0004CBF82EA40004000013B80B2F7D18D428F
:1085F000F0D130BC704700BF2DE9F04FDFF8F8C173
:10860000DFF8F8E1BCF80A70DEF80060BCF80C3066
:10861000BCF808A03C028BB0361B4FF00004CDE93B
:108620000034009CBCF806304FEA17654FF0000795
:1086300067EB0507B946B046A4FB06670024CDE901
:108640000634009C002304FB09770024CDE90034A4
:10865000AAFB0823CDE90223039AF30D00930AFB3A
:1086600009230393009B43EA47230093029B4FEAAD
:10867000D31AFB150193039B4AEA436ADDE9002301
:1086800044464D46CDE90845069C12F5FA62A4FB26
:10869000086743F1000304FB0977CDE90623BCF822
:1086A0000440039BBCF802204FEAE31B230C059314
:1086B00023040493340A44EA07643D12DDE90467A5
:1086C0004FEAC23816EB0A0647EB0B0718EB040813
:1086D000DDE906344FEA524949EB0509B3F5FA6F73
:1086E00074F10004B246BB463CDADDE90067BC0029
:1086F000B20044EA9673B41847EB030522463C46A1
:108700002B4602FB04F406FB0344A2FB062323448E
:10871000940844EA83749D105B104FEA3202B8EB70
:10872000040869EB0509BAEB020A6BEB030BDDE900
:108730000623304C4FF0FF35A242AB412CDBDDE984
:108740000856A5FB052305FB06F403EB4403D40FF1
:1087500044EA4304DD17DDE90623121B63EB05033E
:10876000CDE90623DEF80440A4FB082304FB09330B
:10877000540D44EAC3245D15B4EB0A0A65EB0B0BF8
:108780004FEADA3343EA4B4300B1036009B1069B79
:108790000B600BB0BDE8F08F40F6AC52B4184FF050
:1087A000000347EB03052246A2FB022304FB05F46A
:1087B00003EB4403941843EB0305A4185D414FEA0F
:1087C000850CA6004CEA947CB41A6CEB0305DF0020
:1087D000D6006D104FEA340447EA5277921B63EBE0
:1087E0000703B8EB040869EB05091AEB020A4BEB27
:1087F000030BA4E724FAFFFF7C480020CC1F0020D5
:108800004FF40063838270474FF4006383827047A4
:1088100050F8043C012280F84520103803B1184775
:10882000704700BFBFF34F8F0549064BCA6802F47B
:10883000E0621343CB60BFF34F8F00BFFDE700BF83
:1088400000ED00E00400FA05F8B5057B4669036811
:108850001F2D29D9A5F120045F682021A1400F42D6
:108860002A4613D01022A240D960DA605A68E2404A
:10887000D10703D5012202FA04F4DC600446304635
:10888000FFF7BEFB227B23681F2A20D9A2F120001C
:1088900008215A688140114200D0D96004225968E9
:1088A00082400A4221D1F8BD20211C68A9400C4217
:1088B0002A460CD01022AA4099609A601A68EA40B1
:1088C000D207DBD5012202FA05F59D60D6E7082123
:1088D00018689140014200D099600421186801FA9B
:1088E00002F2024203D09A60F8BDDA60F8BDF8BD2A
:1088F00070B4037B04681F2B08D9203B20216268D9
:1089000001FA03F31A421CD170BC7047202122687F
:1089100001FA03F31A42F7D042691449582000FBC8
:10892000021251685689CD680868296821F0010152
:108930002960828992B222EA06028281A36070BC19
:10894000704742690949582000FB02125168568954
:10895000CD680868296821F001012960828992B2F6
:1089600022EA06028281E36070BC7047CCA300203B
:1089700030B4094B1C786CB1084A002502EBC404E2
:10898000116893884D628889083203439BB2A242E2
:108990008B81F5D130BC70478CA6002090A60020BA
:1089A00010B4037B01681F2B09D9203B20224C689F
:1089B00002FA03F31C4214D15DF8044B70472022E5
:1089C0000C6802FA03F31C42F6D00C4A40680024FB
:1089D000147002685DF8044B22F0010202608B60A3
:1089E0007047064A40680024147002685DF8044B22
:1089F00022F001020260CB60704700BF1B8F002095
:108A0000F0B5C40022189200AE498B585B689D8A6D
:108A1000ADB2EEB2F7070A445CD4B70732D5BFF364
:108A20005F8F167EF6B2012E00F0C780A64D1A8B1E
:108A3000BFF35F8F221801EB8202167E022E00F038
:108A4000D580221801EB8202167E032E00F088806A
:108A50009A8895F9086092B242F480629A8022184E
:108A600001EB8202127E013296425BD1AA7A002685
:108A70006E72002A40F09580204401EB80000023B4
:108A80004375F0BD77074ED416F0400600F0C9805C
:108A90008D4D1E8A95F908E0176AF6B207F80E6048
:108AA0005FFA8EFE0EF1010C4FFA8CFC177E85F8F2
:108AB00008C00CF103029742664600F01C812218A0
:108AC00001EB8202127E9445C9D10EF1020676B204
:108AD0002E72C4E71E887C4D26F400663604360CE0
:108AE0001E801E88B6B246F480661E80967E0027E1
:108AF0002F72002E48D06E7A002E42D0221801EB41
:108B000082020126127E6E72022A00F0B9802218BB
:108B100001EB8202927D42F001021A82204401EBB5
:108B20008000037EF0BD684D967E0127AF72002E57
:108B300073D06E7A002E7BD1221801EB8202527E16
:108B4000002A00F0A3801A882E7A92B2013642F4ED
:108B5000007276B21A802E721A88D205FCD47EE793
:108B6000927E002A3FF474AF6A7A002A3FF470AF15
:108B70009A8895F9086022F480621204120C9A8097
:108B80006DE7D27DFF2AB9D0221801EB8202967DD3
:108B900006F0FE061E82D37DFF2BBFD0FF232B7273
:108BA000BCE79A8822F4407212042044120C01EBB4
:108BB00080009A8000234375F0BD927E424D002ACA
:108BC0003FF435AF6A7A002A3FF431AF1A8822F4B5
:108BD00080621204120C1A80BFF35F8F1A8B1A88FE
:108BE000AE7292B242F400721A8031E7927E002A8D
:108BF0003FF427AF6A7A002A3FF423AF1A8895F929
:108C0000086022F480621204120C1A809A8822F4FE
:108C100080621204120C9A8021E76A7A002A8BD0B3
:108C200091E715F0800F284D3AD195F9086016E7C5
:108C3000167ED2F820E01F88022E95F9086045D9EB
:108C400027F480673F043F0C1F801F8AFFB20EF895
:108C500006701F88D2F820E0BFB247F400771F806B
:108C6000F2B21F8A561C76B2FFB20EF806709F88C9
:108C7000961CBAB276B242F480622E729A806BE78A
:108C80001A8892B242F400621A8040E71A8895F975
:108C9000086092B242F4807201271A806F725BE71B
:108CA00095F90870B7F1FF3F2CD0D669F65D1E82AA
:108CB00092F818E001377AB2964516462A727FF488
:108CC000CEAEA3E7AC390020CC1F0020BFB247F4E2
:108CD00000771F801F8AFFB20EF80670F6B21F8A57
:108CE000D2F820E0721C52B20336FFB276B20EF810
:108CF00002702E7230E79A8822F480621204120CFD
:108D00009A80DCE6D77D1F822E72957E1DB9127E79
:108D1000002A7FF403AF9A8822F480621204120CB6
:108D20009A80FBE670B5044682B01430E56D0623E8
:108D30006A464321A847B0B19DF804009DF8006041
:108D40009DF801109DF802509DF803209DF8053014
:108D500041EA062143EA002342EA0522A187E2878D
:108D6000A4F84030012002B070BD00BF70B50446C9
:108D700082B00830656A06236A463B21A847A8B13D
:108D80009DF804009DF800609DF801109DF80250C8
:108D90009DF803209DF8053041EA062143EA0023AF
:108DA00042EA0522E18222836383012002B070BD82
:108DB00000232822036002702922C270012243602E
:108DC0008360827143727047F8B50468C4F30D0480
:108DD00005460E4604B32F682DF060FB092840F0CD
:108DE0008880454C236923F440732361236943F44D
:108DF00000732361236943F0010323613E602DF07A
:108E00004DFB2369092823F00103236171D12B68ED
:108E100004332B600020F8BD384B394A93422BD9DC
:108E200002F58042934226D902F5804293422AD924
:108E300002F58042934228D902F58032934226D926
:108E400002F50032934224D902F50032934222D92E
:108E500002F50032934220D902F5003293421ED926
:108E600002F5802293421CD9B3F1016F1BD3052078
:108E700005F062FAFBE708242DF010FB092814D056
:108E80004FF0FF30F8BD1024F6E71824F4E7202453
:108E9000F2E72824F0E73024EEE73824ECE740241A
:108EA000EAE74824E8E75824E6E7134F3B6923F450
:108EB00040733B613B6943F400733B613B6923F0C2
:108EC000F8033B613B6943F002031C433C613B698F
:108ED00043F480333B612DF0E1FA3B6923F0020358
:108EE0003B613B69092823F0F8033B613FF473AF12
:108EF000C6E76FF00100F8BD003C024000400008EA
:108F0000FF3F0008F8B504460D468E180027B5420D
:108F100001D12069F8BDE368591CE160234415F8CC
:108F2000012B1A720429F2D1206918B9A1682046D0
:108F3000FFF74AFF2061E760E9E700BF70B582B044
:108F400004466946143026F0D3F8B0B19DF8050008
:108F50009DF801609DF802109DF803509DF80420D3
:108F60009DF8063041EA062143EA002342EA052241
:108F7000A187E287A4F84030012002B070BD00BF95
:108F800038B5254B9C68236B73B1636D626BCAB1B6
:108F9000998A1A88C90592B201D5D20700D438BD82
:108FA0004FF6F7721A8038BD636D99891A88890661
:108FB00092B2EBD59206E9D5E26ACAB1988880B23E
:108FC0009047E2E799891A880D0692B2E0D510061B
:108FD000DED5A26A616A8A4219D0A1692569885CD6
:108FE00098800132B2FBF5F105FB1122A262CFE7B6
:108FF0009B88E2696169DBB28B54E269E068636D6A
:109000000132B2FBF0F100FB1122E261BEE7DA6847
:1090100022F08002DA60BBE78439002038B5254BA6
:109020001C68236B73B1636D626BCAB1998A1A882D
:10903000C90592B201D5D20700D438BD4FF6F772F8
:109040001A8038BD636D99891A88890692B2EBD56A
:109050009206E9D5E26ACAB1988880B29047E2E701
:1090600099891A880D0692B2E0D51006DED5A26A5B
:10907000616A8A4219D0A1692569885C98800132A9
:10908000B2FBF5F105FB1122A262CFE79B88E269F2
:109090006169DBB28B54E269E068636D0132B2FB57
:1090A000F0F100FB1122E261BEE7DA6822F08002F3
:1090B000DA60BBE78439002003685B6A03B11847B4
:1090C000704700BF03681B6A03B11847704700BFB1
:1090D00003682DE9F041DF691FB13B46BDE8F0416F
:1090E0001847002A164611DD04460D460E4400E0DE
:1090F00023689B68204698470028F9D0236815F814
:10910000011B1B6820469847AE42F1D1BDE8F081B3
:1091100003689B69184700BF03685B69184700BF75
:1091200003681B69184700BF0368DB68184700BF66
:1091300003689B68184700BF03685B68184700BF57
:1091400003681B68184700BF014B1868F8E700BFA9
:1091500038AA002038B50C46097849B105460134D3
:109160002B6828461B68984714F8011B0029F7D183
:1091700038BD00BF064B53F820302BB11A689B88CE
:1091800051690B4201D1138370475383704700BF6D
:10919000B8B7002003682DE9F04F03F13F4404F510
:1091A0007E04604EA40A0125345D04F01F066409A4
:1091B000032C05FA06F500F0AF80042C00F0A78020
:1091C000022C54D08588B5FA85F0C0F11F0080B21A
:1091D000C40803EB840400F00700266A80000F2710
:1091E000874026EA07062662276A01F0030602FA8C
:1091F00000F0721E3843012AC1F3810CC1F300183C
:109200002062C1F3411137D90024224601274FF0D3
:10921000030E03E0102A04F1020426D007FA02F03C
:10922000A84302F10102F5D1D3F800C00EFA04F010
:10923000C04300EA0C0CC3F800C0D3F8008006FA63
:1092400004FC4CEA080CC3F800C0D3F80CC000EAD8
:109250000C00D860D3F80CC001FA04F040EA0C000E
:10926000102AD86004F10204D8D1BDE8F08F2E4C4A
:10927000666C35436564A5E7002002464FF0010E99
:109280004FF0030904E00132102A00F102003CD043
:109290000EFA02F737EA0504F5D1D3F800A009FA6F
:1092A00000F4E4430AEA040AC3F800A0D3F800B0CB
:1092B00006FA00FA4AEA0B0AC3F800A0D3F808A09D
:1092C00004EA0A0AC3F808A0D3F808B00CFA00FAB6
:1092D0004AEA0B0AC3F808A0D3F804A02AEA070751
:1092E0005F60D3F804A008FA02F747EA0A075F6054
:1092F000DF683C40DC60DF6801FA00F401323C4387
:10930000102ADC6000F10200C2D1BDE8F08F064CEB
:10931000266B3543256355E7034C266C354325649E
:1093200050E700BF8C20040800380240026802F1B8
:109330003F4303F57E032DE9F04F9B0A544DEB5C50
:1093400003F01F055B090124032B04FA05F400F068
:109350009980042B00F09180022B3ED001F003068F
:10936000731E012BC1F3810CC1F300188588C1F372
:10937000411137D90024234601274FF0030E03E0A3
:10938000102B04F1020426D007FA03F0A84303F1DE
:109390000103F5D1D2F800C00EFA04F0C04300EA90
:1093A0000C0CC2F800C0D2F8008006FA04FC4CEAAB
:1093B000080CC2F800C0D2F80CC000EA0C00D06063
:1093C000D2F80CC001FA04F040EA0C00102BD06077
:1093D00004F10204D8D1BDE8F08F2E4B5D6C2C4314
:1093E0005C64BBE7002003464FF0010E4FF0030919
:1093F00004E00133102B00F102003CD00EFA03F719
:1094000037EA0504F5D1D2F800A009FA00F4E443E4
:109410000AEA040AC2F800A0D2F800B006FA00FA7C
:109420004AEA0B0AC2F800A0D2F808A004EA0A0A25
:10943000C2F808A0D2F808B00CFA00FA4AEA0B0AFF
:10944000C2F808A0D2F804A02AEA07075760D2F8A9
:1094500004A008FA03F747EA0A075760D7683C40B8
:10946000D460D76801FA00F401333C43102BD46078
:1094700000F10200C2D1BDE8F08F064B1D6B2C43FA
:109480001C636BE7034B1D6C2C431C6466E700BF39
:109490008C2004080038024010B50409013C032C5C
:1094A00017D80D4B33F8142000F00F0042FA00F3E8
:1094B00013F001030DD0012303FA00F0013810402E
:1094C00032F050FF054A064B125D104403EBC0001A
:1094D00010BD002010BD00BF98200408942004088F
:1094E0002CB600202DE9F04F4A484B494B4B4C4CD1
:1094F0004FF0010A4FF002094FF004084FF0080C3A
:109500004FF0100E20274026802530F8022B12F055
:10951000010F03D01960A3F804A0083312F0020F62
:1095200003D01960A3F80490083312F0040F03D09D
:109530001960A3F80480083312F0080F03D01960F3
:10954000A3F804C0083312F0100F03D01960A3F879
:1095500004E0083312F0200F02D019609F80083316
:1095600012F0400F02D019609E80083312F0800F75
:1095700002D019609D80083312F4807F05D04FF42B
:10958000807B1960A3F804B0083312F4007F05D083
:109590004FF4007B1960A3F804B0083312F4806F15
:1095A00005D04FF4806B1960A3F804B0083312F4AF
:1095B000006F05D04FF4006B1960A3F804B00833B6
:1095C00012F4805F05D04FF4805B1960A3F804B0FB
:1095D000083312F4005F05D04FF4005B1960A3F864
:1095E00004B0083312F4804F05D04FF4804B19605B
:1095F000A3F804B00833D20B04D04FF40042196032
:109600009A80083301F58061A1427FF47EAFBDE806
:10961000F08F00BF98200408000002402CB6002004
:109620000010024000286AD003682DE9F04F03F1D2
:109630003F4404F57E045F4EA40A0125345D04F026
:109640001F066409032C05FA06F559D0042C00F016
:10965000AC80022C59D08588B5FA85F0C0F11F0086
:1096600080B2C40803EB840400F00700266A80007F
:109670000F27874026EA07062662276A01F00306BD
:109680008240701E3A430128C1F3810CC1F30018D7
:109690002262C1F341113DD90024224601274FF037
:1096A000030E03E0102A04F1020426D007FA02F0A8
:1096B000A84302F10102F5D1D3F800C00EFA04F07C
:1096C000C04300EA0C0CC3F800C0D3F8008006FACF
:1096D00004FC4CEA080CC3F800C0D3F80CC000EA44
:1096E0000C00D860D3F80CC001FA04F040EA0C007A
:1096F000102AD86004F10204D8D1BDE8F08F704779
:109700002D4C266C35432564A5E72B4C666C354300
:109710006564A0E7002002464FF0010E4FF00309F8
:1097200004E00132102A00F102003CD00EFA02F7E8
:1097300037EA0504F5D1D3F800A009FA00F4E443B0
:109740000AEA040AC3F800A0D3F800B006FA00FA47
:109750004AEA0B0AC3F800A0D3F808A004EA0A0AF0
:10976000C3F808A0D3F808B00CFA00FA4AEA0B0ACA
:10977000C3F808A0D3F804A02AEA07075F60D3F86B
:1097800004A008FA02F747EA0A075F60DF683C4076
:10979000DC60DF6801FA00F401323C43102ADC602F
:1097A00000F10200C2D1BDE8F08F034C266B3543B7
:1097B000256350E78C20040800380240002855D06B
:1097C000026802F13F4303F57E032DE9F04F9B0A47
:1097D000544DEB5C03F01F055B090124032B04FAD5
:1097E00005F444D0042B00F09780022B44D001F004
:1097F0000306731E012BC1F3810CC1F30018858889
:10980000C1F341113DD90024234601274FF0030E37
:1098100003E0102B04F1020426D007FA03F0A8435A
:1098200003F10103F5D1D2F800C00EFA04F0C043F1
:1098300000EA0C0CC2F800C0D2F8008006FA04FC62
:109840004CEA080CC2F800C0D2F80CC000EA0C00C8
:10985000D060D2F80CC001FA04F040EA0C00102BE2
:10986000D06004F10204D8D1BDE8F08F70472E4BD0
:109870001D6C2C431C64BAE72B4B5D6C2C435C6461
:10988000B5E7002003464FF0010E4FF0030904E056
:109890000133102B00F102003CD00EFA03F737EA37
:1098A0000504F5D1D2F800A009FA00F4E4430AEA6D
:1098B000040AC2F800A0D2F800B006FA00FA4AEA98
:1098C0000B0AC2F800A0D2F808A004EA0A0AC2F8FB
:1098D00008A0D2F808B00CFA00FA4AEA0B0AC2F85B
:1098E00008A0D2F804A02AEA07075760D2F804A01B
:1098F00008FA03F747EA0A075760D7683C40D46084
:10990000D76801FA00F401333C43102BD46000F116
:109910000200C2D1BDE8F08F034B1D6B2C431C63CA
:1099200065E700BF8C2004080038024038B50446C3
:1099300090F8590000285AD104F11405236E8022B2
:109940006B2128469847642005F0A2F9236E072270
:10995000682128469847642005F09AF9236E002272
:109960006B2128469847642005F092F9236E012266
:109970006B21284698470F2005F08AF994F8532068
:10998000236E032A8CBF1A2218221B2128469847CF
:109990000F2005F07DF9236E18221C2128469847D8
:1099A0000F2005F075F9236E94F852201A212846ED
:1099B00098470F2005F06CF9236E94F85420192174
:1099C00028469847642005F063F9236E102237215A
:1099D000284698470F2005F05BF92846236E0122A0
:1099E000382198470F20BDE8384005F051B9FFF7FE
:1099F00053FD0546D0B1202300218371C171FFF7CB
:109A0000DDFE21460F4B41F8103F284625F006FBAE
:109A1000AB88B3FA83F3C3F11F03012212FA03F3F5
:109A20008AD009490A6813430B6085E70146FFF7AE
:109A3000C5FE2146034B41F8103F284625F0EEFABB
:109A40007AE700BF11880008003C014010B10368AC
:109A500082885A83704700BF10B1036882881A83D6
:109A6000704700BF18B10368828809B95A837047EC
:109A70001A83704710B40A4B0A4A1C7801238340AA
:109A8000234052F8200029B9B3FA83F149095DF85F
:109A9000044BE7E7191C18BF01215DF8044BE1E70F
:109AA000B4B70020B8B7002030B1036882881B69C2
:109AB0001A4214BF01200020704700BF2DE9F04179
:109AC0000B4E346873691C400FD0DFF828800127E3
:109AD000B4FA84F3C3F11F0307FA03F558F823001F
:109AE00003689847AC437561F2D1BDE8F08100BFCF
:109AF000003C0140887A00202DE9F0410B4E34688B
:109B000073691C400FD0DFF828800127B4FA84F372
:109B1000C3F11F0307FA03F558F8230003689847B9
:109B2000AC437561F2D1BDE8F08100BF003C01405B
:109B3000887A00202DE9F0410B4E346873691C408F
:109B40000FD0DFF828800127B4FA84F3C3F11F0394
:109B500007FA03F558F8230003689847AC4375618A
:109B6000F2D1BDE8F08100BF003C0140887A0020BE
:109B70002DE9F0410B4E346873691C400FD0DFF8BB
:109B800028800127B4FA84F3C3F11F0307FA03F511
:109B900058F8230003689847AC437561F2D1BDE8DB
:109BA000F08100BF003C0140887A00202DE9F0419F
:109BB0000B4E346873691C400FD0DFF828800127F2
:109BC000B4FA84F3C3F11F0307FA03F558F823002E
:109BD00003689847AC437561F2D1BDE8F08100BFDE
:109BE000003C0140887A00202DE9F0410B4E34689A
:109BF00073691C400FD0DFF828800127B4FA84F382
:109C0000C3F11F0307FA03F558F8230003689847C8
:109C1000AC437561F2D1BDE8F08100BF003C01406A
:109C2000887A00202DE9F0410B4E346873691C409E
:109C30000FD0DFF828800127B4FA84F3C3F11F03A3
:109C400007FA03F558F8230003689847AC43756199
:109C5000F2D1BDE8F08100BF003C0140887A0020CD
:109C6000084A094808B5536C43F480435364002103
:109C7000402234F0F6FE054B4FF0FF321A60C3F875
:109C8000032008BD00380240887A0020C87A0020EE
:109C900003685B6A184700BF2DE9F0410446184687
:109CA0000D461646984631F0B3FE2768E672284402
:109CB000A07229467D69434632462046AC46BDE83F
:109CC000F0416047036810B504461B689847236855
:109CD00020469B689847A37B0133A37310BD00BF48
:109CE00010B5036804469B689847FF2301226373FD
:109CF000227310BD08B5FFF7CFFB38B12C2282715B
:109D00000022C2712021BDE8084057E508BD00BF10
:109D100040F2E93300E0A3B10289013B12F0020FE7
:109D20009BB2F8D089B2818140F2E93300E043B1BF
:109D30000289013B12F0010F9BB2F8D08089C0B2BA
:109D40007047094A904205D0084B984201D0FF2045
:109D500070470223064A02EB03135A89013292B27A
:109D60005A815889C0B2704700300140003C004021
:109D700014AE002010B5014600BF074C2368986858
:109D8000FFF764FE23685868FFF7C2FF23689868EE
:109D9000FFF762FE00BF10BD1C7B0020144B9842F1
:109DA00024D003F58063984220D0028822F040023C
:109DB0001204120C0280028822F038031B041B0CD0
:109DC00059B141F48071002991FAA1F2B2FA82F1FD
:109DD00008BF4FF0FF310139C9000B439BB203802C
:109DE00003889BB243F04003038070474908DCE7D7
:109DF0000038004010B5802104468069FFF7CEFF8F
:109E0000012004F0EBFE2046FFF790FD10226A21AE
:109E100004F11400FEF716FA642004F039FFA0697B
:109E20000421FFF7BBFF0120BDE8104004F0D6BEBF
:109E3000F0B484894FF6FF764FF47A7443B3002967
:109E400038D00F78013101E0B4421AD00589013CC5
:109E500015F00205A4B2F7D0BCB284814FF47A7435
:109E600002E0BCB2B4420CD0058915F0010504F142
:109E7000FF37F6D08589ADB20AB115700132013BCA
:109E8000DCE70D4B984207D0A3F57443984202D00B
:109E90000120F0BC70470225084B03EB05156B89C8
:109EA00001339BB26B81688980B2003018BF0120FA
:109EB000F0BC7047FF27C9E70030014014AE002016
:109EC00070B50546806810B104688088608341F0F1
:109ED0008001686840F2E93400E0E4B10689013CA1
:109EE00016F0020FA4B2F8D089B2818140F2E931B4
:109EF00000E009B30489013914F0010F89B2F8D0E8
:109F000081890021FFF794FFAB6813B11A689B8821
:109F10001383012070BD1049884204D0A1F574411B
:109F20008842EED102240D4901EB0414618901310C
:109F300089B261816189E4E7074CA04203D00849F6
:109F40008842DED10221054C04EB01114C89013419
:109F5000A4B24C814989D4E70030014014AE0020FE
:109F6000003C0040F8B5654C0601A7190546387A53
:109F700031F0C6F83B7A03F01F015B090122032B85
:109F800002FA01F26DD0042B66D0022B5CD0A3192B
:109F900001351879FFF780FAEDB2074610B11223A8
:109FA000C5718371A3195879FFF776FA10B113239D
:109FB000C5718371A3199879FFF76EFA10B1142354
:109FC000C5718371A5190A21EA793846FFF72AFB82
:109FD0006879FFF761FAEA790A21FFF723FBA8798C
:109FE000FFF75AFAEA790A21FFF71CFBA359444A02
:109FF000934247D0434A934250D0434A934259D068
:10A00000424A934262D0424A93426BD0414A9342C1
:10A010002CD03444227BE2B901200222198801F4B9
:10A02000415141F445710A4302431A809A8B22F44C
:10A0300000621204120C07219A8319821A8892B2C4
:10A0400042F040021A80F8BD334B596A0A435A6203
:10A050009DE700200246E1E72F4B19690A431A6188
:10A0600095E72D4B196A0A431A6290E702F564429C
:10A070004FF40010536A43F4001353622CF008F9B4
:10A08000A359C6E702F584324FF48050536A43F473
:10A09000805353622CF0FCF8A359BAE702F5003262
:10A0A0004FF48040136A43F4804313622CF0F8F8B5
:10A0B000A359AEE702F5FE324FF40040136A43F4B1
:10A0C000004313622CF0ECF8A359A2E702F58232A8
:10A0D0004FF40050536A43F4005353622CF0D8F805
:10A0E000A35996E702F568424FF48010536A43F48F
:10A0F000801353622CF0CCF8A3598AE714AE0020E9
:10A100000030014000380040003C00400034014075
:10A11000005001400054014000380240427A02B928
:10A12000704710B504460368406804F10A01984777
:10A130000023637210BD00BF437A5A1C0344D2B29D
:10A1400042729972037A934200D802B9704710B5EF
:10A1500004460368406804F10A01984700236372CB
:10A1600010BD00BF302827D0312827D0322827D073
:10A17000332827D0342827D0352827D0202827D0A7
:10A18000212827D0102827D0112827D0122827D0FF
:10A19000132827D0142827D0152827D0162805D013
:10A1A000172808BF0F2202D0002070470E22104B44
:10A1B00003EB4203587E70470022F8E70122F6E7DE
:10A1C0000222F4E70322F2E70422F0E70522EEE799
:10A1D0000622ECE70722EAE70822E8E70922E6E799
:10A1E0000A22E4E70B22E2E70C22E0E70D22DEE799
:10A1F000CCEB030870B5448806460D46C4F30B0447
:10A2000022460021284634F02CFC3369094A934247
:10A2100009D3094A934206D2224628461946BDE888
:10A22000704032F09DB923B121462846BDE8704008
:10A23000184770BD2406000829070008064B074987
:10A240008B4202D30023184670471A88C2F30B02D0
:10A250009042F8D01433F3E7880100082406000880
:10A26000024A136823EA000010607047249400201B
:10A27000F8B5174D2B78A32B28D16B78BE2B25D1A1
:10A28000022229464FF6FF70FEF79CF9114FAC1CD5
:10A2900022884AB1A618BE4218D2052A16D92146EC
:10A2A000FEF790F93446F3E721460222FEF78AF9D9
:10A2B0000222A118FEF786F90634074B641B1C80A6
:10A2C00041F60F53C31A58425841F8BD0020F8BD5B
:10A2D0000040000800800008E23F00202DE9F04F18
:10A2E000DFF84C914D4F8BB00326A7EB09071822DE
:10A2F000002104A834F0B5FB494BCDF81090059728
:10A300001A69002A04DA474A5A6002F188325A6010
:10A3100001228DF82420F322DA60434B434C1B8842
:10A32000ADF800300222694604A8FEF7EBFD0222D8
:10A3300069464FF6FF70FEF745F9DFF8F8A0804652
:10A340004FF0000B544539D30AAC002524F8245DA6
:10A350000222214604A8FEF7D5FD022221464046EE
:10A36000FEF730F940BAC043ADF80800022202A956
:10A3700004A8FEF7C7FD079878B106ABC0F1040248
:10A380002946184434F06DFB089818B9069904A8BA
:10A39000FEF71AFD0023089007939DF82430089AD1
:10A3A00023B11F490B6943F000430B61013E2DD0DF
:10A3B000002A9CD1FFF75CFF50B32CE065888DF834
:10A3C0000DB0C5F30B05AB1DADF808302388C3F302
:10A3D0000B02ADF80A201B0B062202A904A88DF877
:10A3E0000C30FEF78FFD062202A94046FEF7EAF880
:10A3F000616880462A4604A8FEF784FD61684046ED
:10A400002A46FEF7DFF8143480469BE7002AD1D0B5
:10A41000052003F091FF0BB0BDE8F08F008000082D
:10A42000003C02402301674504EC03088801000852
:10A4300000400008240600080378202B024600F1A3
:10A440000100F9D0092BF7D02D2B2CD02B2B03BFDB
:10A450005378B7EE000A0246B7EE000AA3F13001C6
:10A46000C8B209289FED467A10D8F2EE046A07EECA
:10A47000901AF8EEE77A12F8013FE7EE267AA3F198
:10A480003001C8B20928B0EE677AF0D92E2B4CD033
:10A4900003F0DF03452B0BD0F7EE007A67EE276A57
:10A4A00020EE260A70475378BFEE000A0246D5E731
:10A4B00010B451782D2959D02B290ABF9178501CFE
:10A4C000901C0024A1F13003092B53D8002303EB87
:10A4D000830301EB430310F8011FA1F13002092AA5
:10A4E000A3F13003F3D9B3F59A7F28BF4FF49A73E1
:10A4F000072B42D9DFED236A1A46F7EE007A083AB5
:10A50000072A67EEA67AFAD803F007032BB1F2EE1A
:10A51000046A013B67EEA67AFBD124B3C7EE276A33
:10A520005DF8044B20EE260A70475378A3F1300102
:10A53000C8B2092802F10102AAD8F2EE046AF0EECC
:10A54000665A07EE901AF8EEE77A12F8013F87EEA6
:10A55000A66AA3F13001C8B2092866EEA56A37EEF3
:10A56000067AEED994E767EE276AD9E7901C9178CE
:10A570000124A7E7F7EE007ACFE7F7EE007AC5E708
:10A580000000000020BCBE4CB5EEC00ADFED317A01
:10A59000F1EE10FACCBF30EE270A30EE670ADFED9D
:10A5A0002E7A20EE270A30B5FDEEC07A87B017EE7E
:10A5B000904A054684EAE470002303A9A0EBE47006
:10A5C00001930093029323F021FD002CACBF2023C4
:10A5D0002D2303A88DF8003031F01AFA012803A9C1
:10A5E00024D002282DD0032805BF302368466846B2
:10A5F0008DF8013034F05BFA684631F009FA03381F
:10A60000C4B222466946284634F0AFFA00232B55DF
:10A61000284631F0FDF92E22431C2A540DEB04018B
:10A62000E81834F061FA284607B030BD3023684698
:10A630008DF801308DF802308DF8033034F037FAA0
:10A64000DAE7302368468DF801308DF8023034F0B7
:10A650002EFAD1E76F12033A00007A442DE9F04157
:10A66000064615460846B6FBF2F43CB905FB1464F1
:10A67000124B1B5D00F8013BBDE8F081B4FBF2F723
:10A6800067B90E4B05FB174705FB1464DA5D00F84C
:10A69000012B1B5D00F8013BBDE8F081B7FBF2F830
:10A6A000B8F1000F02D04046FFF7D8FF05FB18783D
:10A6B000024B13F8082000F8012BE3E7A020040860
:10A6C00030B402681146531C036011F8024B01605C
:10A6D000D31C517803609378151D05601B0443EA71
:10A6E0000123D078234343EA006030BC704700BFA9
:10A6F0000368591C1A46016012F8021B0260587860
:10A7000041EA0020704700BF03685A1C02601878B5
:10A71000704700BF38B504460068154631F020FF89
:10A7200022682A44226038BD036810B40A0E5C1CFB
:10A7300004601A7003680A0C5C1C04601A700368D9
:10A740000A0A5C1C04601A7003685A1C02601970C3
:10A750005DF8044B704700BF036810B40A0A5C1C24
:10A7600004601A7003685A1C026019705DF8044B8B
:10A77000704700BF03685A1C026010B41970036868
:10A780000A0A5C1C04601A7003680A0C5C1C0460F2
:10A790001A700368090E5A1C026019705DF8044BA8
:10A7A000704700BF03685A1C026019700368090AE9
:10A7B0005A1C0260197070472DE9F047002488B0D8
:10A7C00080460F461E46A14605AD531C03931178E3
:10A7D00039B3252933D1931CCDF8109003935078C9
:10A7E00030284ED04FF0000AA0F13003DBB2092B25
:10A7F00042D96C2819D0642800F0938024D82528E9
:10A800001CD063D9582876D063281BD131784046B4
:10A81000B847039A531C0393117804360134002976
:10A82000D7D1204608B0BDE8F087039B5A1C03929D
:10A830001B78642B7CD02AD8252B54D12521404667
:10A840000134B847039AC0E7732833D044D9752838
:10A850004FD106F1040E30682B4600220A217646BD
:10A86000FDF7A6FD049A0095534639464046FDF78C
:10A87000DDFD039A0444A8E704AA03A923F0A2FB80
:10A88000B7E7D31C039390784FF0010AACE7732B22
:10A8900010D05BD9752B3AD0782B96D1A3F1580202
:10A8A000B2FA82F2306852092B4610210436FDF7C5
:10A8B0007FFDD7E73368049A00933946002340466A
:10A8C000FDF7B4FD04360444039A7EE70028B9D1AD
:10A8D000204608B0BDE8F0876E28B3D1039A3368EC
:10A8E00004361C6071E72AD9582BD7D0632B8DD042
:10A8F0006BE77828A6D1A0F15802B2FA82F230684C
:10A9000052092B461021FDF753FD0436AAE706F144
:10A91000040E30682B4600220A217646FDF748FDDA
:10A92000A0E7331D306829461E46FDF713FD99E761
:10A93000331D306829461E46FDF70CFD92E7002BBB
:10A940007FF443AF204608B0BDE8F0876E2BC6D039
:10A950003BE700BF0EB400B584B005AB019053F8DF
:10A96000042B0649039301A8FFF726FF019B002251
:10A970001A7004B05DF804EB03B07047218400083E
:10A980000FB430B583B006AB0A490B4853F8042B1B
:10A99000096800680193FFF70FFF084C054620681F
:10A9A000FEF7BAFB0028FAD0284603B0BDE83040D5
:10A9B00004B07047783900207C39002038AA002084
:10A9C000DFED2B7AB4EEE70AF1EE10FA4ADDDFEDA7
:10A9D000296A9FED297A01E0B0EE670AB4EEC70A52
:10A9E000F1EE10FA70EE667AF6DC9FED247AF4EE62
:10A9F000C77AF1EE10FA38D5DFED1E6A9FED207AA6
:10AA000001E0F0EE407AF4EEC77AF1EE10FA37EE9C
:10AA1000A60AF6D4DFED1B7AB4EEE70AF1EE10FADF
:10AA200014DDDFED137A37EEC00A60EE006A9FEDA9
:10AA3000166A9FED167ADFED167AA6EE867A20EE7C
:10AA4000266AE6EE877AA6EE270A7047DFED117ACE
:10AA5000B4EEE70AF1EE10FA44BFDFED087A37EE04
:10AA6000C00AE2E7F0EE407ABFE7B0EE670AD1E74E
:10AA7000DB0F4940DB0FC940E4CB1641DB0F49C077
:10AA8000E4CB16C1DB0FC93F92E741B99730083CD0
:10AA900015A82ABEDB0FC9BF80EAE073A3EBE07301
:10AAA0008B4205DB002801DD401A704702D1704758
:10AAB000002070470844704709B909E0194690FB27
:10AAC000F1F301FB13030846002BF7D1084670474A
:10AAD0000146FBE7F0EEC07AB0EEE07AB4EEE77A3A
:10AAE000F1EE10FAB4BFB0EE676AB0EE476AB5EEA9
:10AAF000406AF1EE10FA46D0B4EEE77AF1EE10FAC1
:10AB00008CBFF0EE675AF0EE475AC5EE866A9FEDAD
:10AB10001F3A9FED1F6A9FED1F4A9FED1F5ADFED01
:10AB20001F3ADFED1F4ADFED1F5AA6EEC36AE6EEBD
:10AB3000A34AA6EE864AB7EE006AA6EE845AA6EEAF
:10AB4000A46AE6EE855AC5EE866AB4EEE77AF1EEBF
:10AB500010FA48BFDFED147AF5EEC00A48BF77EE71
:10AB6000E66AF1EE10FA48BFDFED107AB5EEC00AE2
:10AB700048BF77EEE66AF1EE10FA48BFF1EE666A7A
:10AB8000B0EE660A7047DFED076ADEE739094E3D31
:10AB9000E3B59E3E88FA163E45FE7F3F99FB243F73
:10ABA00069A2163EA7DFA834DB0FC93FDB0F49407F
:10ABB000DFED317A30EE277AFDEEC76A16EE903A75
:10ABC0002033402B02D99FED2D0A7047B4EEE70ADF
:10ABD000F1EE10FA4DDD9FED2A6ADFED2A6A01E001
:10ABE000B0EE677AB4EEE67AF1EE10FA77EE467AD6
:10ABF000F6DC9FED257AF4EEC77AF1EE10FA35D542
:10AC0000DFED1F6A9FED217A01E0F0EE407AF4EE6D
:10AC1000C77AF1EE10FA37EEA60AF6D4DFED167A0F
:10AC2000B4EEE70AF1EE10FA1BDCDFED197AB4EEB0
:10AC3000E70AF1EE10FA44BFDFED137A37EEC00AEF
:10AC400060EE006A9FED136A9FED137ADFED137AD1
:10AC5000A6EE867A20EE266AE6EE877AA6EE270A28
:10AC60007047DFED0F7A37EEC00AE9E7B0EE670A0A
:10AC7000D4E7F0EE477ABCE7DB0FC93F00000000E5
:10AC8000DB0FC940E4CB1641DB0F49C0E4CB16C152
:10AC9000DB0FC9BF92E741B99730083C15A82ABE1F
:10ACA000DB0F4940FDEEC07A17EE903A2033402B7F
:10ACB00051D8DFED2D7AB4EEE70AF1EE10FA50DD4F
:10ACC000DFED2A6A9FED2A7A01E0B0EE670AB4EE62
:10ACD000C70AF1EE10FA70EE667AF6DC9FED257A7F
:10ACE000F4EEC77AF1EE10FA38D5DFED206A9FED69
:10ACF000227A01E0F0EE407AF4EEC77AF1EE10FA33
:10AD000037EEA60AF6D4DFED1D7AB4EEE70AF1EECF
:10AD100010FA1BDCDFED1A7AB4EEE70AF1EE10FA56
:10AD200044BFDFED147A37EEC00A60EE006A9FED93
:10AD3000156A9FED157ADFED157AA6EE867A20EE7C
:10AD4000266AE6EE877AA6EE270A7047DFED067AD6
:10AD500037EEC00AE9E79FED0E0A7047B0EE670ACA
:10AD6000D1E7F0EE407AB9E7DB0F4940DB0FC9408D
:10AD7000E4CB1641DB0F49C0E4CB16C1DB0FC93F62
:10AD8000DB0FC9BF92E741B99730083C15A82ABE2E
:10AD90000000000010B507EE901A2DED028BB8EE02
:10ADA000678ADFED217A28EE008A044628EE278A9A
:10ADB000B0EE480A31F094FDF0EE408AB0EE480A59
:10ADC00031F0F0FCF7EE007A9FED187AF0EE675A5A
:10ADD000E8EE875A0023A361B0EE676AC7EEA56A62
:10ADE00063612362E361A8EEC76ABDEC028B77EE74
:10ADF000C07AB6EE007AF8EE005A27EE877A20EE97
:10AE0000250A27EE267A26EE266A67EEA67A20EE37
:10AE1000260A84ED046AC4ED017A84ED007A84ED9B
:10AE2000027A84ED030A10BD27D4D236F304353FED
:10AE300010B44C09012250F8243001F01F0102FA2D
:10AE400001F10B4340F824305DF8044B704700BF1C
:10AE50004B0901F01F0150F82320012303FA01F1EF
:10AE6000114214BF18460020704700BF074A084B24
:10AE700010781B78074A834296BFC31AC3F1800338
:10AE80000020126818441044704700BF34AA002004
:10AE9000B1A90020F8470020064A074B10781B781C
:10AEA00083428ABFC3F18003C01AC018C0F17F007B
:10AEB000704700BF34AA0020B1A9002030B5144C5F
:10AEC000237883B01BB90120237003B030BD052265
:10AED00000238DF800208DF8013000BF0D4D2B6848
:10AEE0009868FEF7B3FD2B6801AA6946586830F0F0
:10AEF0001BFA2B689868FEF7AFFD00BF9DF8053080
:10AF000003F0010383F00100237003B030BD00BFE4
:10AF10002E7B00201C7B002070B5064C0646256861
:10AF200003E023685B1BB34203D8FFF7C7FF002889
:10AF3000F7D070BD0CAE00202DE9F04F89B0B2F112
:10AF4000000A02900491039340F3B0800B46002264
:10AF500001EB8A0153F8040B8B420244FAD1039BA4
:10AF60000592002B00F09A80059B002B6AD0544B71
:10AF7000059A1B68DFF85C9100920099DAB25118CB
:10AF8000B1F5807F8CBFC2F58072009A01924D4A64
:10AF900092689A426DD9190C1A0A4FF002040620E1
:10AFA0008DF81F308DF81E208DF81D108DF81C4077
:10AFB000FFF7B2FF0620FEF7DDFE434A01231370C0
:10AFC00000BFD9F800309868FEF740FDD9F800308E
:10AFD00007A95868002230F05FF90024049D029E02
:10AFE000019FA34629684FEA840800220B460134DA
:10AFF00071B1B9422AD2D9F8000031684068FEF731
:10B0000017FF2A68336813443360BF1AC5F800B0CD
:10B01000A24505F1040506F10406E3D1D9F8003094
:10B020009868FEF719FD00BF254B019900981B6831
:10B03000421A0092224A0B441360039A32B3009AD8
:10B04000002A9AD1059809B0BDE8F08F029CD9F882
:10B05000003054F80810586800223B46FEF7E8FE1E
:10B0600054F808202B683A44DF1B44F808202F606E
:10B07000D4E70598009C1549154A001B05900598D2
:10B0800000230B70137009B0BDE8F08F059B009A88
:10B090009B1A0593059809B0BDE8F08FFFF70EFFE6
:10B0A00000287FF461AF039B0593CBE7039C1CB999
:10B0B000FFF704FF0594C5E700230593C2E700BF2F
:10B0C000F8470020740300202E7B002034AA0020C3
:10B0D000B1A900201C7B002070B5104D104E2B78BC
:10B0E00031788B4284B016D00E4A03921A440292F1
:10B0F0008CBF0C46CA1A04A98CBFC3F1800200247D
:10B10000012341F8102D02A802220194FFF714FF39
:10B11000002333702B7004B070BD00BFB1A90020B4
:10B1200034AA0020B4A9002070B5194C194D237819
:10B130002978994284B027D0174A03921A44029280
:10B1400034BF0E46CA1A04A934BFC3F180020026D8
:10B15000002341F8102D02A802220196FFF7ECFE11
:10B1600023781844C0B203062B7848BF80F08000D3
:10B170008342207002D0002004B070BD0023012063
:10B180002B70237004B070BD012004B070BD00BFEF
:10B19000B1A9002034AA0020B4A9002008B545F2C6
:10B1A0000820FFF7B9FE0620FEF7E4FD064B01225A
:10B1B000C7201A70FEF7DEFD04480549054A002342
:10B1C00003700B70136008BD2E7B002034AA002092
:10B1D000B1A90020F84700202DE9F04182B00346D4
:10B1E000060C050A032406208DF80730884617460A
:10B1F0008DF805608DF806508DF80440FFF78CFE41
:10B20000C0B100BF0D4C23689868FEF71FFC23688F
:10B2100001A95868002230F03FF823684246002117
:10B2200058683B46FEF704FE23689868FEF714FC56
:10B2300000BF384602B0BDE8F08100BF1C7B002093
:10B24000F0B5124B9D6885B00DB905B0F0BDED0AA3
:10B2500014D0002704AE7C196410E0021022694665
:10B26000FFF7BAFF0F2809DD6B4653F8042B0132B4
:10B270000AD1B342F9D12546AF42ECDBFFF72CFFF0
:10B28000034BED021D60E0E7671CF5E77403002047
:10B29000F84700200C4B984213D0A3F580639842E6
:10B2A0000FD003F5804398420BD003F5806398429A
:10B2B00007D003F58063984203D0044B1868400818
:10B2C0007047024B1868704700040140E0A200205C
:10B2D000F0B5774B774A87B01968914200AF00F01C
:10B2E000DB800023744A3B607B60136843F4803347
:10B2F000136003E03B68B3F5A04F09D0136803F473
:10B3000000337B603B6801333B607B68002BF1D0EE
:10B31000694B1B6813F4003318BF01237B607B6803
:10B32000012B7BD0654D644B654AEA606549586FD7
:10B33000654A0860AA605E6B644C654A654826F001
:10B3400080065E635E6F46F080765E67196B0C4325
:10B350001C63596B5963996B9963196C41F05B518C
:10B3600041F47B1141F41F6141F00F011964596CE4
:10B3700007F118040A4348F2FF715A6444F8101D9B
:10B38000002621460123FB733E737E73BE732AF0B1
:10B390004BFE21464FF6FF734F48BB602AF044FE38
:10B3A0004FF6FF7321464D48BB602AF03DFE214613
:10B3B0004B482AF039FE21464A482AF035FE2146FC
:10B3C00049482AF031FE214648482AF02DFE214600
:10B3D00047482AF029FE214646482AF025FE204605
:10B3E0002BF014F8444B454C1B68BA684448454957
:10B3F000A4FB03439B09A0FB0202013B920CB3F1A7
:10B40000807F0A6007D2404AF0200721536085F808
:10B410002300966011601C37BD46F0BD264B3B4DA6
:10B420001A6C3B4842F080521A642C68426881686A
:10B4300044F440442C609C689C609C6844F4004444
:10B440009C609C6844F4A0549C600068120642EA28
:10B45000801242F48002490842F00802013942EAAF
:10B4600001425A601A6842F080721A601A689201AA
:10B47000FCD52849104A40F205700860996821F00F
:10B4800003019960996841F002019960936803F0A3
:10B490000C03082BFAD145E700221A6062B61E4B56
:10B4A0001B6883F308881D4B1B689847FEE700BFA5
:10B4B000FCFF0120EFBEADDE0038024000ED00E0F1
:10B4C0000005FA054C6D002000000008FF916700A0
:10B4D000335F070000000240000402400008024001
:10B4E000000C02400010024000140240001802400C
:10B4F000001C024000200240E0A20020D34D621058
:10B5000083DE1B4310AE002010E000E0007000401E
:10B5100000000020003C02400000FF1F0400FF1F4D
:10B5200008B5054B1B6803B19847044B044A1A60E1
:10B5300072B6FDF777F900BF20430020FCFF012021
:10B54000EFBEADDE08B5034B1B6803B1984772B67A
:10B55000FDF768F920430020084B10B507281B6849
:10B56000C8BF143818440C46007EFDF795FF20B183
:10B570002146BDE81040FEF775BA10BDF47A0020F0
:10B5800030B50446406D61718389A26823F400538D
:10B590001B041B0C838185B0A379009213F0040275
:10B5A00030D04FF4805213F00203ADF804205CD188
:10B5B000ADF806304FF480630022ADF8083011F08A
:10B5C0000103ADF80C2028D1ADF80A3008238D070F
:10B5D000694648BFADF80A301DF0BCFDA279636D25
:10B5E000D10724D412F0080F9A8A1BD122F0080246
:10B5F0001204120C9A829A8992B242F400529A81F1
:10B6000005B030BD13F00203ADF804202AD04FF48A
:10B6100000551346ADF80650CEE70423ADF80A30C6
:10B620000C23D4E792B242F008029A82E3E7104971
:10B630008B4215D0A1F548418B420FD001F58061B6
:10B640008B4209D00B498B42CCD105200121FFF759
:10B6500083FFA279636DC5E70320F7E70220F5E7D2
:10B660000020F3E7ADF80630A6E74FF400539FE75C
:10B67000001001400014014010B50446406DA16067
:10B68000838923F400531B041B0C8381A37984B0AA
:10B6900013F00402009135D04FF4805213F00203EE
:10B6A000ADF804205CD1ADF806304FF480636279C8
:10B6B000ADF80830D1074FF00003ADF80A30ADF80F
:10B6C0000C3045BF0423ADF80A3008230C2369462B
:10B6D000920748BFADF80A301DF03CFDA279636DBA
:10B6E000D1071FD412F0080F9A8A16D122F008024F
:10B6F0001204120C9A829A8992B242F400529A81F0
:10B7000004B010BD13F00203ADF8042025D04FF4AF
:10B7100000511346ADF80610C9E792B242F0080294
:10B720009A82E8E710498B4215D0A1F548418B4237
:10B730000FD001F580618B4209D00C498B42D1D1E9
:10B7400005200121FFF708FFA279636DCAE70320F6
:10B75000F7E70220F5E70020F3E7ADF80630A6E7AB
:10B760004FF400539FE700BF001001400014014058
:10B7700038B50C4B07281B68CCBFA0F11404044655
:10B7800023440546187EFDF787FE50B10134272279
:10B79000C47182712FF020FD28460021BDE8384099
:10B7A000DAE638BDF47A002070B50F4C0F4DC0EBCF
:10B7B000C00004EB8004286B26693043286382B004
:10B7C0009209667BA1600025012101A863618DF8C3
:10B7D00004608DF805208DF806508DF807101DF0D7
:10B7E00081FC02B070BD00BFB401002000380240EF
:10B7F000074BC0EBC00030B403EB8000054C05697B
:10B80000236B2B4323630176427630BC704700BF25
:10B81000B4010020003802402DE9F04F5B4C54F891
:10B82000204083B0002C00F0AC80E66D002E00F0CC
:10B83000AA809046564A35692260994604F26222EF
:10B8400004F162036361A2614FF400737268A16046
:10B850000746E36023616265A246B5B14D4B002007
:10B860005A68954203F11C0376D001301028F7D1B5
:10B8700000207A1CD2B20C21FFF7BAFF636DB168C9
:10B88000326922630433A1632365F068E8B1414B58
:10B8900000215A68904203F11C035BD0013110294A
:10B8A000F7D100257A1CD2B20B212846FFF7A0FF62
:10B8B0002346F27F38492846FFF776FF636DB1686B
:10B8C000F26862630433E163E36494F86100FDF7B6
:10B8D000E3FD054694F86000FDF7DEFD8346307F0A
:10B8E00000284BD119F0080F38D118F0020F09D0F9
:10B8F00045B10B227B1CAA71EB712846727F222175
:10B90000FDF790FE18F0010F15D1A36B7BB996F8E7
:10B910002020B17F8DF8063001A8930901228DF80F
:10B9200005308DF804108DF807201DF0DBFB504624
:10B9300003B0BDE8F08FBBF1000FE6D001370C2358
:10B940008BF807708BF806305846727F2221FDF77E
:10B9500069FEDAE7CDB2A5E7C0B28AE70137FFB2E8
:10B9600015B10B23EF71AB7119F0100F284614BFFE
:10B9700002211221727FFDF755FEC6E72FF0C0FBB2
:10B98000B0E7A246D3E7B246D1E700BF8439002032
:10B9900008EC0308B4010020498800080348D0F8E7
:10B9A000AC3113B100F5D27018477047B4010020D4
:10B9B0000348D0F8903113B100F5C47018477047B0
:10B9C000B40100200348D0F8743113B100F5B6700B
:10B9D00018477047B40100200348D0F8583113B11C
:10B9E00000F5A87018477047B40100200348D0F84C
:10B9F0003C3113B100F59A7018477047B40100202C
:10BA00000348D0F8203113B100F58C701847704707
:10BA1000B40100200348D0F804310BB1FC301847C2
:10BA2000704700BFB40100200348D0F8E8300BB1E4
:10BA3000E0301847704700BFB40100200348D0F839
:10BA4000CC300BB1C4301847704700BFB4010020A0
:10BA50000348D0F8B0300BB1A8301847704700BF8A
:10BA6000B40100200348D0F894300BB18C30184753
:10BA7000704700BFB40100200248836F0BB17030E3
:10BA800018477047B40100200248C36D0BB1543011
:10BA900018477047B40100200248036C0BB13830DE
:10BAA00018477047B40100200248436A0BB11C30AC
:10BAB00018477047B40100200248836803B1184753
:10BAC000704700BFB4010020431C00F00E812DE937
:10BAD000F04F4FEAC00808EB00039B00DFF8E8A234
:10BAE0005AF803B087B00AEB0304BBF1000F00F073
:10BAF000F98014330AEB03010022DBF804704AF8E2
:10BB000003204A608A60CA600346A5680190013339
:10BB1000D4F80C90DBB2002D00F0E8801522EB7118
:10BB2000AA71B9F1000F00F0FA80162289F80620F8
:10BB300089F807309BF80E002FF0E2FABB8823F457
:10BB400040731B041B0CBB802846FDF785FF48464D
:10BB5000FDF782FF11212846FDF7E8FB1121484639
:10BB6000FDF7E4FB0826642403E03CB12FF0E6FA7D
:10BB7000013C2846FDF798FF0028F6D02846FDF73F
:10BB800065FF2FF0DBFA2846FDF766FF2FF0D6FAA7
:10BB9000013EEED14846FDF759FF2FF0CFFA284677
:10BBA000FDF754FF2FF0CAFA2846FDF755FF2FF096
:10BBB000C5FA4846FDF750FF019B08EB03040AEB6A
:10BBC00084042846637C002B0CBF122132210422FE
:10BBD000FDF728FD637C002B0CBF12213221484663
:10BBE0000422FDF71FFD704B9F4200F0B7806F4BA2
:10BBF0009F4200F0BD806E4B9F4200F0A580BB8845
:10BC000001996C4A6C4C23F440731B041B0CBB80E1
:10BC10003B8888440AEB880A9BB243F001039AF8F8
:10BC200010103B80BD8802A8002918BF14462AF0D6
:10BC3000EDFB049A6148B2FBF4F325F03F05A0FB4D
:10BC400002122D04900C2D0C0543BD805C4C3988EC
:10BC50004FF4967202FB00F284FB02409BB2D217B3
:10BC6000002BC2EBA01221F0010108BF012309043F
:10BC7000013243F40043090C92B239803A84BB8309
:10BC80003B889BB243F001033B803B8823F48163F4
:10BC900023F002031B041B0C43F480634FF4804227
:10BCA0003B803A813B8823F080031B041B0C3B80C4
:10BCB0009BF810308DF808300024012302A88DF87D
:10BCC0000B308DF809408DF80A401DF00BFA9BF8F7
:10BCD0000F308DF8083002A88DF809408DF80A4021
:10BCE0001DF026FA07B0BDE8F08F7047B9F1000FDC
:10BCF00048D0162289F8073089F806209BF80E00F4
:10BD00002FF0FEF9BB8823F440731B041B0C28465C
:10BD1000BB80FDF7A1FE4846FDF79EFE1EE79BF89F
:10BD20000E002FF0EDF9BB8823F440731B041B0CAD
:10BD3000BB802846FDF790FE4846FDF78DFE112199
:10BD40002846FDF7F3FA0DE71E4A136A43F4000391
:10BD500013624FF400002AF0A3FA50E7194A136A5D
:10BD600043F4001313624FF400102AF099FA46E7E7
:10BD7000144A136A43F4800313624FF480002AF0DC
:10BD80008FFA3CE79BF80E002FF0BAF9BB8823F43A
:10BD900040731B041B0C4846BB80FDF75DFE484604
:10BDA000FDF75AFEDEE600BF005400400058004098
:10BDB000005C0040009F2400804F120083DE1B4384
:10BDC000D34D621000380240AC390020F8B54FEA7C
:10BDD000C00E274F069C0EEB000507EB85056E682D
:10BDE000002E42D04900C9B2A9754FF0000C0121C4
:10BDF000EA7585F819C0A9762B76697585F814C09F
:10BE0000B3882C629905EC6114D43388DA050CD41C
:10BE10004FF4805401E0013C1ED033889B05FAD4D6
:10BE200033889BB243F480733380B3889BB243F46E
:10BE30004073B3800EEB000107EB81024FF4805496
:10BE400001E0013C08D0537D002BFAD107EB8107BC
:10BE50003C7D84F00100F8BD064A138801339BB293
:10BE60001380FFF731FE2046F8BD3046F8BD00BF15
:10BE7000AC390020E03F002070B590F904506C1CF4
:10BE800082B00AD0032D08DC16460A464179009696
:10BE90002846FFF79BFF02B070BD002002B070BDC6
:10BEA00000B50378012B83B004D1032301AA00213C
:10BEB000FFF7E2FF9DF805309DF804209DF806008D
:10BEC0001B0243EA0243184303B05DF804FB00BFC2
:10BED00008B5FFF7E5FF014B586008BDCC1F0020F7
:10BEE00008B5FFF7DDFF014B186008BDCC1F00202F
:10BEF000F0B585B002AB04460093032206231E2151
:10BF00000020FFF763FF00283CD09DF808509DF803
:10BF100009109DF80A709DF80B209DF80C609DF8A3
:10BF20000D3041EA052142EA072243EA062309B21D
:10BF300012B21BB2144D06EE901A07EE102A07EE4D
:10BF4000903AF8EEE66A95ED035AD5ED055A95ED6F
:10BF5000046AB8EEC77AF8EEE77A66EE856A27EEED
:10BF6000257A67EE867AFDEEE66ABDEEC77AFDEECB
:10BF7000E77A16EE901A17EE102A17EE903A218003
:10BF8000A280638005B0F0BD0000002000B583B042
:10BF9000002000920A466821FFF718FF03B05DF801
:10BFA00004FB00BFF0B5C60033189B00254DEA58CE
:10BFB0005468A28A83B092B20192019A2B4412F47F
:10BFC000706F1CBF01221A75019B13F4E06F0746C6
:10BFD0000CD1A38A3E4423F4706305EB86051B0451
:10BFE0001B0C0022A3826A7503B0F0BD238BA388CB
:10BFF00023F480631B041B0CA380019B9B05E8D4E6
:10C0000023889805E5D42388D9050ED52388DA0539
:10C01000FCD423889BB243F40073238023889B05C0
:10C02000FCD43846FFF750FDD3E723889BB243F496
:10C0300000732380A38823F440731B041B0CA3808C
:10C04000C7E700BFAC390020F0B583B0441C8DF8C1
:10C05000073001D0032802DD002003B0F0BDC70087
:10C06000244E3B1806EB83035D68002DF4D0490095
:10C07000C9B2997501240021DA755C7699761C762F
:10C080005C751975A9880DF107028905DA611A62D4
:10C0900014D42B88DA050CD44FF4805401E0013C11
:10C0A0001ED02B889B05FAD42B889BB243F4807357
:10C0B0002B80AB889BB243F44073AB80074406EB04
:10C0C00087024FF4805401E0013C09D0537D002BDE
:10C0D000FAD106EB87073C7D84F0010003B0F0BD88
:10C0E000054A138801339BB21380FFF7EDFC20460D
:10C0F000B3E700BFAC390020E03F00202DE9F0435A
:10C10000322083B002F0C4FD0022104611231E210C
:10C11000FFF79AFF602301221E210020FFF794FF02
:10C12000642002F0B5FD6846FFF7E2FE0024DFF868
:10C130005481254626460A27012302221E2100207B
:10C14000FFF782FF322002F0A3FD6846FFF7D0FE22
:10C15000BDF902E0BDF90410BDF900208E4573461B
:10C16000A8BF0B469342A8BF134643454FF00100BA
:10C1700075440C44164479DBFCF7FCFF013FDBD12E
:10C180004FF001090022104612231E21FFF75CFF29
:10C19000DFF8F0800A27012302221E210020FFF78A
:10C1A00053FF322002F074FD6846FFF7A1FEBDF98F
:10C1B00002E0BDF90410BDF900208E457346A8BF0A
:10C1C0000B469342A8BF134643454FF00100A5EB31
:10C1D0000E05A4EB0104A6EB02064ADBFCF7CAFF3E
:10C1E000013FD8D107EE906AF8EEE76A07EE905A61
:10C1F000B8EEE77A07EE904ADFED1F5A9FED1F5A1F
:10C200001F4EF8EEE77A85EEA66A002210467023EC
:10C210001E21C5EE876A85EE277AB0EEC66AF0EE7B
:10C22000E66AF0EEC77A86ED036AC6ED046AC6EDEB
:10C23000057AFFF709FF202301221E210020FFF7C6
:10C2400003FF0023184602221E21FFF7FDFE642093
:10C2500002F01EFDB9F1000F04D14FF07E53F360E0
:10C2600033617361012003B0BDE8F0834FF0000932
:10C2700088E74FF00009B5E700406F4601C05E4611
:10C280000000002001F0FFFF0378012B00D0704771
:10C29000417990F904005822D6E600BF0378012BBB
:10C2A00000D07047417990F904004822CCE600BFE5
:10C2B000134600200A466821C6E600BF0220FCF7AC
:10C2C0009FBB00BF02206DE60120FCF799BB00BFB9
:10C2D000012067E60020FCF793BB00BF002061E669
:10C2E0001549164B16480A6810B48C681549B2FBFC
:10C2F000F4F203FB02F30360D1F88820124B134CD5
:10C3000042F47002C1F888201A68002042F001024D
:10C310001A6098601A6822F0847222F480321A60DF
:10C320005C601A684FF0006422F480221A60D860C2
:10C330008C605DF8044B70470000002040420F0005
:10C34000E0A2002000ED00E00038024010300024A0
:10C35000044B4FF4F0700A21022283E80700FFF734
:10C36000BFBF00BF0000002038B50B4C23688BB165
:10C370005A68821A002A054604DA0CE05A68AA1A9A
:10C38000002A07DB9A68226018461A6890472368DB
:10C39000002BF3D138BD38BD944B00200B4B00224D
:10C3A00010B4027203F58474032102E0072A09DC49
:10C3B0009979890702D51979815401329C4203F198
:10C3C0001803F3D15DF8044B704700BF8C180408C4
:10C3D0002E230370704700BF012233230270437085
:10C3E000704700BF2322032302704370704700BFD1
:10C3F0002DE9F0410B78047BDB43DEB200F1100243
:10C4000000F1380342F8044F9342FBD1DFF89CC09F
:10C4100000F16001002243F8042F8B42FBD14FF062
:10C42000140E0521002546FA01F303F00103002B49
:10C430001D4414BF4FF019084FF00A0811F0010F06
:10C44000EDB214BF2746002700220EEB02039BB279
:10C4500000EB8303013242455F61F6D1013A92B2AB
:10C46000013201390EEB02034A1C9BB201D09E46F9
:10C47000D9E715F0010F14BF19250A2500215A1814
:10C4800092B200EB82020131A9425461F7D10B4410
:10C490009BB21A1D00EB8202013300219BB2516056
:10C4A000ACF800300361BDE8F08100BFE01F002060
:10C4B000254B5B880B332DE9F04F8A4601F1060BC3
:10C4C0001FFA83F94FF00108002100271AF801EB49
:10C4D0003E464C460122A4F10B039BB207E0013318
:10C4E0009BB2B0F80CC0C5F814C09C420AD000EB57
:10C4F0008305002AF3D100EB830501339BB29C42F4
:10C500006A61F4D1231D00EB83030136092FF6B2D3
:10C5100059600CD0092E14D008FA07F313EA0E0F55
:10C5200014BF012200220C34A4B20137D3E709F171
:10C530007809DA451FFA89F9C7D1034B5980BDE85C
:10C54000F08F0022EFE700BFE01F00202DE9F04749
:10C55000DFF85C80B8F8043004338A461FFA83FCA5
:10C5600001F109094FF0010E1AF8017B644600261B
:10C57000231F0EFA06F29BB23A40BAB1818900EB52
:10C58000830501339BB29C426961F6D101360434C4
:10C59000082EA4B2ECD10CF1200CCA451FFA8CFC79
:10C5A000E2D10023A8F80430BDE8F0871146E6E7A1
:10C5B000E01F002010B4037B01681F2B09D9203B2A
:10C5C00020224C6802FA03F31C4214D15DF8044B9C
:10C5D000704720220C6802FA03F31C42F6D00C4A82
:10C5E00040680024147002685DF8044B22F00102D8
:10C5F00002608B607047064A40680024147002682D
:10C600005DF8044B22F001020260CB60704700BF6E
:10C61000EC81002008B520F037FDFEF793FF00BF46
:10C62000024A034B1278197825F034BFBC2200204F
:10C63000BD220020038A2DE9F0478589ADB21D4057
:10C6400029D00F4606464FF000484FF00009B5FAD2
:10C6500085F328FA03F2D24391B21B3B1540318295
:10C66000042B16D8DFE803F03129211903007B6A77
:10C67000002B32D003F1FF3A1FFA8AFAC7F8249050
:10C680003C6A34B123682046514698476468002CC0
:10C69000F8D1002DDBD1BDE8F0873868716B0368F5
:10C6A00089B29847002DD2D1F5E77868B16B03685D
:10C6B00089B29847002DCAD1EDE7B868F16B0368DD
:10C6C00089B29847002DC2D1E5E7F868316C03685C
:10C6D00089B29847002DBAD1DDE7F36A1FFA83FAD1
:10C6E000CEE700BF2DE9F04F2DED028BA0F10A033C
:10C6F00089B00C46E72B00F23787DFE813F01C0106
:10C700003507350735073507350735073507350749
:10C710003507350735073507350735073507350739
:10C7200035073507350735073507350735078001E4
:10C7300035073507350771013507350735076401BA
:10C74000350781023507690235073902350731029D
:10C7500035070C023507E001350735073507DA01E3
:10C76000D3013507C70535073507BF0535079605DA
:10C770003507350735077905350735073507350797
:10C78000F6023507FC003507F305CF0535073507F9
:10C7900035073507350735073507DD0635079506B3
:10C7A0003507600635070B063507200735073507BF
:10C7B000350735072805ED04E604C502E800AB049B
:10C7C0009704CF048B043507540438043507350724
:10C7D000350735072D04350735070C0435073507B0
:10C7E0003507FE03E703AC036A0335073507350752
:10C7F0005B03440335031503350735073507350754
:10C800003507350735073507350735073507350748
:10C810003507350735072805350735073507350747
:10C820003507350735073507350735073507350728
:10C8300035072D0135073507350735073507350726
:10C840003507350735073507350735073507350708
:10C8500035073507350735073507350735073507F8
:10C8600035073507350735073507350735073507E8
:10C8700035073507350735073507350735073507D8
:10C8800035073507350735073507350735073507C8
:10C8900035073507350735073507350735073507B8
:10C8A00035073507350735073507350735073507A8
:10C8B0003507350735073507350735073507350798
:10C8C000350735073507350735079E01A901AE4EF7
:10C8D000337853B1AD4F002537F8021F2046FDF7DE
:10C8E00061FF33780135AB42F6DC012009B0BDECC5
:10C8F000028BBDE8F08FA44E3378002BF5D0A44F07
:10C900000025B846236817F81520591C21601A70B5
:10C9100098F8011001EB810101EB810101F2EE2198
:10C9200089B22046FDF73EFF33780135AB4208F16E
:10C930000208E7DCD9E7974D28462FF069F8002870
:10C94000D3DD2B460544226813F8011B501C9D4281
:10C9500020601170F7D1C8E70B68DFF870C2591C6E
:10C960009CF8002021601A709CF80030002BBCD08D
:10C97000894E8A4D8A488B490023226816F8017F28
:10C9800002F1010EC4F800E01770226815F8017F6B
:10C9900002F1010EC4F800E01770226810F8017F60
:10C9A00002F1010EC4F800E01770226811F8017F4F
:10C9B00002F1010EC4F800E017709CF8002001336A
:10C9C0009A42DADC91E70B68774A581C11782060AC
:10C9D000197023685278591C216001201A7085E76C
:10C9E000724D08462988FDF7DDFEA9882046FDF72F
:10C9F000D9FE20462989FDF7D5FE012076E76C4D4A
:10CA000005F1500628782BF017FB2368027A591C91
:10CA100021601A7023686A78591C21601A70236893
:10CA2000AA78591C21601A702368EA780435591CC9
:10CA3000AE4221601A70E5D157E75E4D0846E9899C
:10CA4000FDF7B0FE2046A989FDF7ACFE01204DE7B9
:10CA5000594B03F1700522681978501C2060117041
:10CA600022685978501C2060117022689978501CF7
:10CA7000206011702268D978501C206011702268E3
:10CA80001979501C2060117022685979501C20605F
:10CA90001170226899790733501C9D4220601170F3
:10CAA000D9D122E70B6801229918216010461A702B
:10CAB0001CE708460021FDF75DFE012016E73F4D0B
:10CAC00005F1380703E00835AF423FF40EAF95F9A2
:10CAD0000260304611F0A0F90028F4D023685A1CF7
:10CAE00022601E7029882046FDF75CFE2368EA78E4
:10CAF000591C21601A7023682A79591C21601A7008
:10CB00002368AA79591C21601A7023686A79591C14
:10CB100021601A70D7E72A4B03F15A052268597928
:10CB2000501C2060117022681978501C2060117010
:10CB300022685978501C2060117022689978501C26
:10CB4000206011702268D978501C20601170226812
:10CB500019790633501C9D4220601170DED1C4E665
:10CB60000B68184A591C527D216001201A70BDE6DD
:10CB7000154D05F1800655F8041F2046FDF7FAFD16
:10CB8000AE42F8D1B1E600BF28920020AA79002079
:10CB9000AC4D00203842002093510020A3510020CA
:10CBA000C3510020B3510020FC470020243A00204C
:10CBB00000480020FC4C0020485500205C8D0020DF
:10CBC0001C41002070A80020148E002091510020EC
:10CBD000AB4D05F14006B5F880102046FDF7E2FDAB
:10CBE000236895F88220591C21601A70236895F8F3
:10CBF00083200435591CB54221601A70EBD174E6CC
:10CC0000A04D0B682A7A591C21601A70A98B204606
:10CC1000FDF7C8FD298B2046FDF7C4FD698B204632
:10CC2000FDF7C0FD2368EA7C591C21601A70A98CAD
:10CC30002046FDF7B7FDE98C2046FDF7B3FD2368DC
:10CC4000AA7F591C21601A70236895F82020591C6E
:10CC500021601A70698C2046FDF7A4FD2368EA7AEA
:10CC6000591C21601A70E9682046FDF783FD23688E
:10CC70002A7C591C21601A70236895F82120591CC0
:10CC8000216001201A7031E67F4D804E9FED808A31
:10CC9000DFF83082DFED7F8A05F120070EE0FCEE41
:10CCA000E77ACDED017ABDF8041020460435FDF792
:10CCB00079FDBD4206F118063FF417AE717C0029DC
:10CCC000F3D0754BD5ED007A1B78012BE7D1734B70
:10CCD0001B68DB0440F1EB84F5EE407AF1EE10FACC
:10CCE00040F0158540F2DC51DFE70B686C4D591CB4
:10CCF0002A7921601A7023686A79591C21601A7098
:10CD000029882046FDF74EFD2368AA79591C216029
:10CD10001A7069882046FDF745FD2368EA79591C99
:10CD2000216001201A70E1E50B685E4F591C3A78CA
:10CD300021601A703B78002B3FF4D7AD0025EEB28E
:10CD400030461CF053FF23684278591C216030465E
:10CD50001A701CF04BFF01892046FDF723FD3B783C
:10CD60000135AB42EBDCC0E54F4B5049B3F9003025
:10CD700081FB0321DB17C3EBA101204689B2FDF73C
:10CD800011FD0120B2E50A68494B501C197820605A
:10CD9000117022685978501C2060117022689978AF
:10CDA000501C206011702268DB78511C216001202A
:10CDB00013709BE53F4D0846298AFDF7F3FC698A0D
:10CDC0002046FDF7EFFC2046A98AFDF7EBFC012089
:10CDD0008CE5DFF8F4E00027FEB2714600232268FC
:10CDE000501C206016702268501C2060137022684E
:10CDF00011F8010F0133551C062B25601070EED180
:10CE00000137062F0EF1060EE6D12B4900232268CA
:10CE1000501C206017702268501C2060137022681C
:10CE200011F8010F0133551C0B2B25601070EED14A
:10CE30002368134A581C07212060197023680021B9
:10CE4000581C20601970236892F8F020591C21604A
:10CE500001201A704AE50B68184A19491078124ADD
:10CE60005D1C2560187023688978581C2060197033
:10CE700023689278591C216001201A7036E500BFA2
:10CE8000188E002070A80020FC420020E4A20020A0
:10CE90000000404200E08244C8A30020F8A6002021
:10CEA000E05B0020D54E00206C4800206766666677
:10CEB00078510020A4A30020FB8E0020D4A60020DF
:10CEC000FC4C0020DB9B9141D78E00200A68B14BBF
:10CED000B1491878551C2560107022685878551C87
:10CEE0002560107022689B78501C206013702046CB
:10CEF000C988FDF757FC0120F8E4A74D08462988AA
:10CF0000FDF750FC69882046FDF74CFCA9882046B7
:10CF1000FDF748FCE9E4A14D05F16006A98820462B
:10CF2000FDF740FCE9882046FDF73CFC29892046B6
:10CF3000FDF738FC2368AA7A591C21601A7023680F
:10CF4000EA7A591C21601A7055F80C1B2046FDF72F
:10CF500011FCAE42E2D1C8E4914952232268501C30
:10CF60002060137011F8013F002BF7D1BDE48D480C
:10CF700000232268056803EB4301561C6D5C2660A4
:10CF80001570026825680A446E1C527826602A7063
:10CF9000026825680A4401339278691C0A2B2160D3
:10CFA0002A70E6D1A1E4804D0B682A68591C1278DA
:10CFB00021601A702B6822689978531C2360002323
:10CFC00011702A6821681A4401335279481C032BD6
:10CFD00020600A70F5D123682A68591C127A2160F2
:10CFE0001A7023682A68591CD27821601A70236845
:10CFF0002A68591C127921601A702B6820465989B9
:10D00000FDF7D0FB2A682368527A591C21601A70F8
:10D010002A68DEE4654B08461968FDF7ABFB644BF4
:10D0200020461988FDF7BEFB01205FE4614B0846EE
:10D030001988FDF7B7FB604B20461988FDF7B2FB56
:10D040005E4B22681B78511C03F001032160012014
:10D0500013704BE45A4B0A681B785A4D511C03F06D
:10D0600002032160137023682A7D591C21601A7005
:10D0700029682046FDF77EFB69682046FDF77AFBAC
:10D0800029892046FDF78EFBE9892046FDF78AFBBA
:10D090002046298AFDF786FB012027E44A4D0846F1
:10D0A0002988FDF77FFB69882046FDF77BFBB5F9F2
:10D0B0000430464AD91782FB0323C1EBA301204663
:10D0C00089B2FDF76FFB012010E4084610224049A9
:10D0D000FDF720FB012009E43E4B9B8AB3F5006F6E
:10D0E00000F2FA82B3F5806F00F20F83B3F5007F90
:10D0F00034BF01270227384D05F10C0655F8041BF3
:10D1000091FBF7F1204689B2FDF74CFBAE42F5D119
:10D11000324D334F05F10C06B5EC010AD7ED087A14
:10D1200080EE270A2FF090FB81B22046FDF73AFBF4
:10D13000B542F1D12B4D05F10C0655F8041B2046E4
:10D1400089B2FDF72FFBB542F7D1FFF7CEBB002523
:10D150008146DFF89480DFF894B005950495069534
:10D16000079501214FF6FF7A05E001350B2D00F000
:10D17000FE8118F9011F4F1C4AFA05F3F5D0DE07AE
:10D18000F3D5BBF800302B41D807EED506A8FDF744
:10D190004FFEEAE7E04D0020C45B00205C5C00200D
:10D1A00030EC030800920020D4AD002038AD002000
:10D1B0002CAD0020A8500020AA5000205C50002078
:10D1C0005CAD002060AD00203CAD00206766666667
:10D1D000EC420020E4AC00201CAD0020ECA60020B6
:10D1E00044AE0020DC91002060EC03084A8F002050
:10D1F000FDF764FE2368A44D002803F101010CBF74
:10D200000222032221601A7029882046FDF7B2FA13
:10D21000A9682046FDF7AEFAFDF728FE0146204634
:10D22000FDF7A8FA0120FFF761BB0B68974A984DFC
:10D230001178984A581C2060197011682046FDF733
:10D2400099FA2368944A591C127A21601A70298825
:10D250002046FDF7A7FAA9882046FDF7A3FA2989F9
:10D260002046FDF79FFA00212046FDF79BFA204655
:10D270000021FDF797FA0120FFF738BB0846082286
:10D280008549FDF747FA0120FFF730BB0B68834A59
:10D29000581C917820601970FFF79BBB0B68804E7B
:10D2A00001255A1C0A601D700B68B278591921605B
:10D2B0001A7016F0B3F823687A4A7B495F19276021
:10D2C0001870B1F90010B2F90000FDF7F5FB236802
:10D2D0005A192260187031882046FDF763FA2846F3
:10D2E000FFF704BB0B6800255A1C0A601D700B6811
:10D2F0005A1C0A601D700B685A1C0A602046294699
:10D300001D70FDF737FA20462946FDF733FA012054
:10D31000FFF7ECBA00212046FDF744FA0021204631
:10D32000FDF740FA00212046FDF73CFA23685F4DE7
:10D3300000265A1C22601E7023682A68591C92F825
:10D340002C2021601A7023682A68591C92F8362014
:10D3500021601A7023682A68591C92F837202160CE
:10D360001A7023685A1C22601E7023685A1C22609F
:10D370001E7023685A1C22601E702B682046598F2D
:10D38000FDF710FA2B682046198FFDF70BFA23687A
:10D390002A68591C92F82E2021601A7023685A1CA2
:10D3A00022601E702B682046598EFDF7FBF92B6812
:10D3B0002046998EFDF7F6F90120FFF797BA3C4E0B
:10D3C0000B687279394D591C21601A702B68204600
:10D3D000198CFDF7E7F92B682046D98BFDF7E2F9A8
:10D3E00071892046FDF7DEF9B1892046FDF7DAF9AB
:10D3F0002B682046598CFDF7D5F92B682046998C6F
:10D40000FDF7D0F9F1892046FDF7CCF9318A2046A5
:10D41000FDF7C8F92A68236892F82620591C216074
:10D4200001201A70FFF762BA214EF378002B00F04A
:10D4300047810B680822591C21601A702368012259
:10D44000991821601A7023681A4D591C2A79216095
:10D450001A702368AA78591C21601A7029882046FE
:10D46000FDF7A0F9E9892046FDF79CF92368F279D8
:10D47000591C21601A702368EA78591C2160012028
:10D480001A70FFF733BA00BF74030020FC47002076
:10D49000243A00202494002070A80020F8AD002039
:10D4A0000A9400207246002074460020009200205A
:10D4B000D4A60020A4A3002024F0D0FFFF28064615
:10D4C00000F00C8108A9002501F8125D0DF10D0096
:10D4D0008DF80D5024F0A2FF08A800F8115D24F08B
:10D4E00091FF08A800F8105D24F080FF08A820F83C
:10D4F000085D24F06FFF23685A1C22601E702368A9
:10D500009DF80D20591C21601A7023689DF80E208B
:10D51000591C21601A7023689DF80F20591C216046
:10D520001A7023689DF81020591C21601A7020463B
:10D53000BDF81810FDF736F90120FFF7D7B90B68D1
:10D54000924A9349D078934A5D1C256018702368ED
:10D550004979581C206019702368D278591C2160C1
:10D5600001201A70FFF7C2B90020FFF7BFB9DFF83A
:10D570004CA200254FF008080135C5F1200208FA39
:10D5800002F2A5F120032AFA05F6164328FA03F35E
:10D590001E43252D06F001024FF000030BD013436C
:10D5A000EAD0E8B22DF02EFA0028E5D0294606A8E8
:10D5B000FDF73EFCE0E7784B1B78DA0700F1958039
:10D5C0000025764E2F4602E00135252D0DD0294647
:10D5D0003046FDF73DFC0028F6D0294606A8FDF7A9
:10D5E00037FC00285ED10137EEE76D4B6D4DB3F887
:10D5F00050102046FDF7D6F86B4B1988204689B2AB
:10D60000FDF7D0F8694B19684B0103F02002C1F314
:10D6100040031343C1F3800243EA4203C1F3C00253
:10D6200043EA8203C1F3401243EAC20301F010014E
:10D6300019432046FDF7B6F804A904222046FDF759
:10D6400069F8236829785A4A581C20601970118893
:10D650006429A8BF64212046FDF7A4F8B9F1960F0C
:10D6600048D000212046FDF79DF82168B7F1190345
:10D6700048BFA7F11203A3F3C4034A1C226020464B
:10D680001A460B7005A9FDF745F82368494A581C4E
:10D6900010212060197020461188FDF76BF80120D9
:10D6A000FFF724B9394604A8FDF7C2FB9BE7F4EE67
:10D6B000C87AF1EE10FA47DA4FF47A71FFF7F5BA4B
:10D6C0000B68B1783C4A581C2060197023681278A6
:10D6D000591C21601A70B6E608270CE523685A1C0D
:10D6E000226001201E70FFF701B9069B43F0010381
:10D6F000069365E723680322591C21601A7023688A
:10D700006A78591C21601A70AFE70427F3E4F4EE3D
:10D71000C87AF1EE10FA3FF5E5AAF4EEE87AFDEEEC
:10D72000E77AF1EE10FA17EE901A20D86FF4F97339
:10D73000303903FB01F140F2E73391FBF3F101F2E1
:10D74000DB5189B2FFF7B1BAFDEEE77A40F2E7327A
:10D7500017EE903A303B02FB03F388FB0312D91714
:10D76000C1EB622101F2E93189B2FFF79EBA40F2C2
:10D77000F313A1F5836103FB01F140F2E73391FB61
:10D78000F3F101F2DD5189B2FFF78FBAFC4C0020B2
:10D79000BC9100206C480020644F0020B0AA0020FB
:10D7A0008C030020F1910020E03F002058AD0020C4
:10D7B000E43F0020788F0020905A002090E33FF44F
:10D7C0001C4C08B501210220FCF754F9237803F022
:10D7D0000502052A29D003F00903092B08D00021EE
:10D7E0000120FCF747F900210846FCF743F9FEE762
:10D7F000114A124B11681A680B68114C23F001038F
:10D800000B601388206823F001031B041B0C13809A
:10D8100018B1292200238271C37109224A21FBF722
:10D8200001FF2068FCF712F9D9E71FF0BFFC23784D
:10D83000D1E700BF80390020B83A0020BC3A002070
:10D84000C03A0020022828BF022010B4084C094B1F
:10D85000207000EB8002C0EBC20207495DF8044B68
:10D86000013003EB4203C0B20B6011F0FFBD00BFFB
:10D87000F1910020EE9200200092002008B518F0EF
:10D8800035FCFCF72BFDBDE8084018F017BC00BFC5
:10D8900038B5484B5A899989914224BF00225A8150
:10D8A000198ADA89914224BF0022DA81DA78CAB172
:10D8B000072A41496AD091F85700404D01240021C0
:10D8C0000A282C709C70D9715DD00C2807D0002AD2
:10D8D0006CD0DFED3B7A072A0ED00A2862D0DFED4C
:10D8E000397A09E0344A92F857000A2856D00C28B1
:10D8F0005BD1D979DFED347A344C9FED350AA278CB
:10D90000002918BFF0EE407A062A04D8314901EB0D
:10D91000820191ED0F0A217979B1013A032A0BD8DE
:10D92000F7EE007A87EE800A2EF08EFF2388984269
:10D9300028BF1846208038BD38BD9B781F4A07EEA7
:10D94000103A1178B8EEC77A67EE277A07EE101A08
:10D95000B8EEC77A27EE277AB4EEC70AF1EE10FACE
:10D96000EADD80EE277AFDEEC77A17EE903A102BAB
:10D97000A8BF1023012BB8BF0123DBB28B4238BFF5
:10D980000B46137038BDDFED147AA4E791F8570009
:10D990000A2803D00C28ACD0D9799AE7D979DFEDE1
:10D9A0000E7AA9E7DFED0D7AA6E7D979DFED047AE3
:10D9B000A2E700BFD4A6002044AE0020905A002069
:10D9C0006F1203396F12833A0AD7A339A4A3002038
:10D9D0006F12033830EC03085304E9380F506E3AE5
:10D9E00038B50C4C0C4DAC4206D26168204614345C
:10D9F000FCF700FCAC42F8D3084A094B094C146010
:10DA0000002209491A705A7008480860BDE8384079
:10DA10001DF0D6BD880100082406000800920020F1
:10DA2000F1910020EE920020D4AD0020049200205D
:10DA300008B5FFF7D5FF18F059FBFCF74FFCBDE820
:10DA4000084018F03BBB00BFF0B50C2934D8DFE824
:10DA500001F0893333335E333333343333330700E8
:10DA6000048C9689B2F802E01788734D24F4805430
:10DA70002404240C0484038C8488818B23F40053B5
:10DA800021F4E6411B0409041B0C46EA0E06090CAE
:10DA900043EA063341EA0721A8429BB2A4B289B205
:10DAA00000F09E8005F58065A84200F0998092689C
:10DAB0008480818302640384F0BD048C9589B2F86C
:10DAC00002C0B2F800E05C4F24F480742404240CFB
:10DAD0000484038C8688818B23F400731B0421F05B
:10DAE00073011B0C45EA0C04090443EA0423090CE6
:10DAF000B8429BB2B6B241EA0E015CD04F4CA04294
:10DB000059D0926886808183C2630384F0BD048CFF
:10DB10009589B2F802C0B2F800E0474E24F0100434
:10DB20002404240C0484038C8788018B23F02003B5
:10DB300021F4E6411B0409041B0C45EA0C04090C02
:10DB400043EA041341EA0E21B0429BB2BFB289B24C
:10DB50005DD03A4CA0425AD092688780018382639C
:10DB60000384F0BD048C9789B2F802E01688324D28
:10DB700024F001042404240C0484038C8488018B85
:10DB800023F002031B0421F073011B0C47EA0E076C
:10DB900009043B43090CA8429BB2A4B241EA060126
:10DBA00025D005F58065A84221D092688480018344
:10DBB00042630384F0BDD589148A578A23F4006335
:10DBC00043EA05254FF6FF332B40958826F440564F
:10DBD0003C4343EA052346EA04169BB2B6B290E7FB
:10DBE000158A24F4804444EA8514A4B25FE7D689F8
:10DBF000158A578A23F00803334324F44074968827
:10DC00003D4323F004032C433343A4B2CDE7D4892E
:10DC1000158A568A23F0800343EA04134FF6BF7433
:10DC20001C40938827F44067354344EA031347EACE
:10DC300085079BB2BFB28FE700000140000401409E
:10DC40002DE9F04FC822002183B08B488B4CDFF8C0
:10DC500050928B4D8B4E8C4FDFF8488230F001FF95
:10DC60008A488B49DFF840E2DFF840C200221359AE
:10DC7000834200F0D680B3F1804F00F0DD80AB42EC
:10DC800000F0E580B34200F0E480BB4200F0E380A6
:10DC9000734500F0E280634500F0E180434500F009
:10DCA000E080DFF80CA2534500F0DD800AF5806AC1
:10DCB000534500F0DA800AF5806A534500F0D780BA
:10DCC000AAF5983A534500F0D4800AF5806A534586
:10DCD00000F085800AF5806A534508BF0D237FD088
:10DCE0001832B2F5907FC2D1644C6A4E6A4F6B4DC8
:10DCF00004F5907802E01834A0456DD0A379002B8C
:10DD0000F9D023794FEA131909F1FF39B9F1030F5B
:10DD100003F00F03EFD836F8190040FA03F2D207E8
:10DD2000E9D54FF0010A0AFA03F3013B18402EF03F
:10DD300019FB17F80930184415EBC002DBD055F871
:10DD40003000DFF870E1217A00F13F4303F57E03F4
:10DD50009B0A1EF8033003F01F0E5B09032B0AFA1F
:10DD60000EFA60D0042B69D0022B07D1DFF820E136
:10DD7000DEF844304AEA0303CEF844309388009337
:10DD8000B3FA83F3C3F11F039BB2DA0800EB8202FC
:10DD900003F00703D2F820E09B004FF00F0C0CFAC1
:10DDA00003FC2EEA0C0EC2F820E0D2F820E001FAC3
:10DDB00003F343EA0E031362694600230222183478
:10DDC0008DF804208DF805308DF806308DF8073079
:10DDD00028F02AF9A04591D103B0BDE8F08F0C23BB
:10DDE00009EBC3034FF0010A93F85C3003F01F0BFB
:10DDF0005B09032B0AFA0BFA09D0042B0CD0022B77
:10DE00007FF46EAF4B6C4AEA03034B6468E70B6C1C
:10DE10004AEA03030B6463E70B6B4AEA03030B63F1
:10DE20005EE70023DCE7DFF868E0DEF840304AEA2E
:10DE30000303CEF84030A1E70123D1E7DFF850E03B
:10DE4000DEF830304AEA0303CEF8303096E702239A
:10DE5000C6E70323C4E70423C2E70523C0E706237C
:10DE6000BEE70723BCE70823BAE70923B8E70A237C
:10DE7000B6E70B23B4E700BF307B00208C18040802
:10DE80000004004000080040000C00400000014079
:10DE90000038024098200408942004082CB6002082
:10DEA00030EC030800040140001000400014004062
:10DEB000004001408C20040801490248FEF7BABB2B
:10DEC000D07B00200018004001490248FEF7B2BB99
:10DED000A87B00200004014001490248FEF7AABBCC
:10DEE000A87B00200004014001490248FEF7A2BBC4
:10DEF000807B0020000C004001490248FEF79ABBDD
:10DF0000587B00200004004002494FF08040FEF79B
:10DF100091BB00BF307B0020F0B50468474DA30AD9
:10DF2000AB426ED009D8B3F5801F66D0023DAB423C
:10DF300058D14FF0480E012608E0414DAB4264D065
:10DF40003B35AB424FD14FF0980E03264779B000D6
:10DF50004FEA970C00295CD063460227A5899F40B1
:10DF600083190CEB43032F4303F1040C354DBFB26F
:10DF700045F8231045F82C20A781EFF3118150229A
:10DF800082F31288821905EBC202136963B313622C
:10DF90000433821905EBC202576917B11F60536938
:10DFA0000433821905EBC202976917B11F609369A8
:10DFB0000433821905EBC202D76917B11F60D36918
:10DFC00004330027CAB21F6082F31188304405EB86
:10DFD000C000036A5BB9A38923F001031B041B0C77
:10DFE000A381F0BDF0BDF0BD05EB0E03D1E7A38921
:10DFF0009BB243F00103A381F0BD4FF0200E002639
:10E00000A4E74FF0700E0226A0E74FF0C00E0426E2
:10E010009CE70223BF0803FA07F7A389094D9BB2C7
:10E0200023EA070387190CEB470CA3810CF10403C7
:10E0300045F82C1045F823209FE700BF030010008F
:10E0400006001000307B002010B5036883480139BA
:10E05000834282B089B200F0CB80A0F58060834219
:10E0600000F0C68000F58040834200F0B88000F5E3
:10E070008060834200F0B38000F58060834200F04E
:10E08000AE80774C188824686408B4FBF2F4013C35
:10E09000A4B282B2B3F1804F0AD07248834207D053
:10E0A00000F58060834203D000F58060834202D196
:10E0B00022F0700292B26C48834200F0A28000F518
:10E0C0008060834200F0A78022F4407200F56C402B
:10E0D00092B283421A80D9621C854FD05F4A934224
:10E0E0004CD001229A821A8892B242F001021A8020
:10E0F000B3F1804F00F099805A4A934200F0978024
:10E1000002F58062934200F0948002F580629342AF
:10E1100000F0918002F58062934200F08E8002F55B
:10E120008062934200F08B8002F57042934200F0CF
:10E13000888002F57052934200F0858002F580627B
:10E14000934200F0828002F5806293427FD0A2F574
:10E15000983293427DD002F5806293427BD002F5E3
:10E160008062934208BF0D2215D002A84FF0012310
:10E1700040F8043D1AF0B6FF02B010BD01220021A4
:10E1800019869A821A88394892B242F00102834273
:10E190001A80ADD10A46364B03EBC20301A893F8AF
:10E1A0005D408DF80440012300228DF805308DF884
:10E1B00007308DF806201AF095FF1B2C08D02E2C66
:10E1C000DAD12C4B019301A81AF08CFF02B010BDDC
:10E1D000294B019301A81AF085FF02B010BD204C15
:10E1E00018882468B4FBF2F4013CA4B282B251E76F
:10E1F0001B4C18882468B4FBF2F4013CA4B282B230
:10E2000056E701201A80D9621C8598821A8892B23A
:10E2100002431A8070E701201A80D9621C85988217
:10E220001A8892B202431A8062E70122B3E70222FF
:10E23000B1E70322AFE70422ADE70522ABE70622F0
:10E24000A9E70722A7E70822A5E70922A3E70A22F0
:10E25000A1E70B229FE70C229DE700BF00040140CD
:10E26000E0A2002000040040001000400000014037
:10E2700030EC03082C010001190100012C4B9842DD
:10E280003DD0B0F1804F3CD0A3F57C4398423AD0CA
:10E2900003F58063984238D003F58063984236D006
:10E2A00003F58063984234D003F58063984232D0FE
:10E2B00003F57043984230D003F5705398422ED046
:10E2C00003F5806398422CD003F5806398422AD0EE
:10E2D000A3F59833984228D003F58063984207D07D
:10E2E00003F58063984208BF0D2202D000207047DA
:10E2F0000C22104B03EBC20393F85C007047002222
:10E30000F7E70122F5E70222F3E70322F1E704220F
:10E31000EFE70522EDE70622EBE70722E9E708220F
:10E32000E7E70922E5E70A22E3E70B22E1E700BF7E
:10E330000000014030EC03082DE98048013085B031
:10E34000C3B203938A4D8B4F8B4C8C4E0A2302939E
:10E35000DFF82C9220F0CEFC4FF4FA7A4FF0100C3C
:10E360004FF47A70D9F80430C3F30803002B40F05F
:10E37000C180EFF31183002B40F0BC802968A268B4
:10E3800000BF2B689942F9D1D7F800E000FB0EF3EB
:10E390009B1AB3FBFEF300FB01314FF0010E01911C
:10E3A000D9F80430C3F30803002B40F08780EFF363
:10E3B0001183002B40F082802B68A16800BF2A687F
:10E3C0009342F9D1D7F800B000FB0BF2521AB2FB1E
:10E3D000FBF200FB0323019A9B1AB3F57A7FDFD38C
:10E3E000BAF1010ABED1039B002B40F0BD804FF46F
:10E3F0007A7ADFF88C9150464FF0100CD9F804303F
:10E40000C3F30803002B40F09280EFF31183002B3D
:10E4100040F08D802968A26800BF2B689942F9D12D
:10E42000D7F800E000FB0EF39B1AB3FBFEF300FBF2
:10E4300001314FF0010E0191D9F80430C3F3080304
:10E4400003BBEFF31183EBB92B68A16800BF2A6807
:10E450009342F9D1D7F800B000FB0BF2521AB2FB8D
:10E46000FBF200FB0323019A9B1AB3F57A7FE3D3F7
:10E47000BAF1010AC2D1029B013B02937FF468AF5B
:10E48000FDF74EF8EFF311888CF31288A16823682A
:10E49000DB0344BFC6F800E0A1682B6832685FFA6E
:10E4A00088F888F31188D7F800801A4400FB08F335
:10E4B0005B1AB3FBF8F300FB0233D4E7EFF31188E8
:10E4C0008CF31288A1682368DB0344BFC6F800E020
:10E4D000A1682B6832685FFA88F888F31188D7F84A
:10E4E00000801A4400FB08F35B1AB3FBF8F300FB4F
:10E4F000023370E7EFF311828CF31288D4F808E04E
:10E500002368D90303D501233360D4F808E02B68CE
:10E510003168D2B282F311883A68194400FB02F3E1
:10E52000A3EB0E03B3FBF2F300FB013135E7EFF38E
:10E5300011828CF31288D4F808E02368D90303D53C
:10E5400001233360D4F808E02B683168D2B282F33B
:10E5500011883A68194400FB02F3A3EB0E03B3FBE6
:10E56000F2F300FB013164E718462CF043FF3EE76D
:10E570000CAE002010AE002010E000E008AE00203D
:10E5800000ED00E02DE9F047AC4FAD4E17F0AEFDC9
:10E59000BE421ED2DFF83483DFF834934446258828
:10E5A00062197DB14A450DD2052D0BD9338861889A
:10E5B000C3F30B03994200F0EE80144625886219DC
:10E5C000002DEFD1716830461436FBF713FEBE42C2
:10E5D000E4D39C4A1378A3F1170102290FD99A4971
:10E5E00011F83300002840F01B81D800014449781D
:10E5F00029B1964911F833300BB918231370944C94
:10E600006378022B84BF002363702378022B84BFBE
:10E61000002323708F4B9A78042A00F0F88032B9D7
:10E620001A88B2F5F07F84BF4FF4F0721A808A4DD9
:10E630008A4A2B681A40002A00F0FB80D80700F1B4
:10E64000E180590400F1D9801A0700F1D1809B04C0
:10E6500000F1C780824D2B685A8C998C914224BF5F
:10E6600000225A84FFF714F926F07CFD002800F000
:10E67000B4804FF40070FBF7F3FD4FF48020FBF7FC
:10E68000EFFD4FF00070FBF7EBFD4FF08060FBF704
:10E69000E7FD6378022B06D8724A734903EB430304
:10E6A00002EB83030B602378022B07D803EB830173
:10E6B0006E4AC3EBC10302EB43032B602CF01AFA42
:10E6C000002130226A4830F0CCF928681EF090F919
:10E6D000684B2D6803F1500102E0043399427AD06F
:10E6E0001A78002AF9D19C78D8788442F5D2624908
:10E6F000624B0A7028461D6023F004FE604B614A9D
:10E700001E7961496148624B1160C825642212FB81
:10E710000652604C406B31F8061C5A600022218082
:10E720009A60DA601A615A619A61DA6183F820208E
:10E7300083F8212008B117F001FB574B9FED575A82
:10E740001B88574A9FED576A557B574C5749584885
:10E75000086006EE903AF8EEE66A1389C5EE265A8E
:10E7600007EE103A5389127BC4ED005A07EE903A37
:10E77000B8EEC77A4F4BF8EEE77A1D725A7227EE61
:10E78000067A67EE867ABDE8F04783ED017AC3ED3D
:10E79000007A17F093BC63799B077FF40EAF716822
:10E7A00094F804A03046FBF725FD3388BAEB133FFD
:10E7B00004D01436BE42FFF4F1AE0AE773887068E5
:10E7C000AA1FC3F30B039A4204F10601A8BF1A461D
:10E7D0002DF0C6FEEDE7012289E737480FF0D2F8A9
:10E7E00047E73648FBF73CFD4020FBF739FD31E7B2
:10E7F0003348FBF735FD2B6829E73248FBF730FD3E
:10E800002B6821E73048FBF72BFD2B6819E79A8A24
:10E81000B2F57A7FBFF40BAF4FF47A729A8206E7B3
:10E82000D8000C186468002C7FF4E0AE1724147034
:10E83000DCE643F008032B6000E700BF2406000875
:10E8400088010008FC4700202C12040890100408DE
:10E85000F1910020A4A3002024940020096000026C
:10E860000092002004920020D4AD0020EE920020FF
:10E870008824002000480020F41D0020BC24002033
:10E88000E05B002088AA0020024D0020E4AC0020BC
:10E89000548F00208C4C0020144E0020C0C9FB482F
:10E8A000E01F002017B7D138184E00201054002068
:10E8B0003661023DEC5300205C8D002009400002CF
:10E8C0000160000209200002086000020240000806
:10E8D0000080000808B517F009FCFBF7FFFC17F0F3
:10E8E000EDFBFFF74FFE0120BDE8084010F0BEBD74
:10E8F0002DE9F04F013085B0C3B203930B4602916E
:10E900008B4C8C4E002B00F099808B4D8B4FDFF899
:10E91000309220F0EFF94FF4FA7A4FF0100C4FF4E8
:10E920007A70D9F80430C3F30803002B40F0DE807E
:10E93000EFF31183002B40F0D9802968A26800BF53
:10E940002B689942F9D1D7F800E000FB0EF39B1A2F
:10E95000B3FBFEF300FB01314FF0010E0191D9F83A
:10E960000430C3F30803002B40F08780EFF31183DA
:10E97000002B40F082802B68A16800BF2A68934278
:10E98000F9D1D7F800B000FB0BF2521AB2FBFBF240
:10E9900000FB0323019A9B1AB3F57A7FDFD3BAF108
:10E9A000010ABED1039B002B40F0BD804FF47A7A60
:10E9B000DFF88C9150464FF0100CD9F80430C3F3B7
:10E9C0000803002B75D1EFF31183002B71D1296857
:10E9D000A26800BF2B689942F9D1D7F800E000FB8C
:10E9E0000EF39B1AB3FBFEF300FB01314FF0010E57
:10E9F0000191D9F80430C3F3080313BBEFF311837B
:10EA0000FBB92B68A16800BF2A689342F9D1D7F8F7
:10EA100000B000FB0BF2521AB2FBFBF200FB032327
:10EA2000019A9B1AB3F57A7FE3D3BAF1010AC4D1F4
:10EA3000029B013B0293002B7FF467AF05B0BDE85A
:10EA4000F08FEFF311888CF31288A1682368DB0341
:10EA500044BFC6F800E0A1682B6832685FFA88F806
:10EA600088F31188D7F800801A4400FB08F35B1A7A
:10EA7000B3FBF8F300FB0233D2E7EFF311888CF31A
:10EA80001288A1682368DB0344BFC6F800E0A168D0
:10EA90002B6832685FFA88F888F31188D7F800800D
:10EAA0001A4400FB08F35B1AB3FBF8F300FB0233D4
:10EAB00070E7EFF311828CF31288D4F808E0236832
:10EAC000D90303D501233360D4F808E02B683168FB
:10EAD000D2B282F311883A68194400FB02F3A3EB27
:10EAE0000E03B3FBF2F300FB01317FE7EFF311827A
:10EAF0008CF31288D4F808E02368D90303D50123E6
:10EB00003360D4F808E02B683168D2B282F3118800
:10EB10003A68194400FB02F3A3EB0E03B3FBF2F3D4
:10EB200000FB013118E718462CF064FC3EE700BFFB
:10EB300010E000E008AE00200CAE002010AE002077
:10EB400000ED00E0204B5B68C3F3080330B4BBB9B1
:10EB5000EFF31183A3B91D4B1D4C1868A16800BFCA
:10EB60001A689042F9D11B4B1C684FF47A7202FB71
:10EB700004F3591AB1FBF4F130BC02FB00107047EA
:10EB8000EFF31182102383F3128811498C680B680C
:10EB900013F4803F104B02D0012018608C680B49A1
:10EBA000D2B20D68186882F311880A4B19684FF4C5
:10EBB0007A72284402FB01F31B1B30BCB3FBF1F358
:10EBC00002FB0030704700BF00ED00E00CAE0020FB
:10EBD00010E000E010AE002008AE00202DE9F84F54
:10EBE0008046FFF7AFFF254E2549DFF8A0E0254A14
:10EBF000254D844610274FF47A740120DEF8043046
:10EC0000C3F30803D3B9EFF31183BBB90B68D2F890
:10EC100008A000BFD1F800904B45F7D1D6F800B05E
:10EC200004FB0BF9A9EB0A09B9FBFBF904FB0393FD
:10EC3000A3EB0C034345E1D3BDE8F88FEFF3118A52
:10EC400087F31288D2F808B01368DB0344BF28604A
:10EC5000D2F808B00B68D5F800905FFA8AFA8AF308
:10EC60001188D6F800A0994404FB0AF3A3EB0B0328
:10EC7000B3FBFAF304FB0933DAE700BF10AE002060
:10EC80000CAE002010E000E008AE002000ED00E037
:10EC90002DE9F04FDFF830C1474A4849484E494D09
:10ECA0008046102718F1FF38C0F08480DCF804306B
:10ECB000C3F30803002B5CD1EFF31183002B58D171
:10ECC0000B68946800BF08688342F9D1D6F80090B9
:10ECD0004FF47A7000FB09FEAEEB040EBEFBF9FEAA
:10ECE00000FB03EEDCF80430C3F308034FF47A743E
:10ECF0000120FBB9EFF31183E3B90B68D2F808A048
:10ED000000BFD1F800904B45F7D1D6F800B004FB16
:10ED10000BF9A9EB0A09B9FBFBF904FB0393A3EB7D
:10ED20000E03B3F57A7FBDD2DCF80430C3F30803D9
:10ED3000002BDFD0EFF3118A87F31288D2F808B0E6
:10ED40001368DB0344BF2860D2F808B00B68D5F81D
:10ED500000905FFA8AFA8AF31188D6F800A09944E5
:10ED600004FB0AF3A3EB0B03B3FBFAF304FB093335
:10ED7000D5E7EFF3118487F31288D2F8089013686F
:10ED8000D80303D501232B60D2F808900B682868BC
:10ED9000E4B284F31188D6F800A04FF47A7400EB43
:10EDA000030E04FB0AF3A3EB0903B3FBFAF304FB22
:10EDB0000E3E97E7BDE8F08F10E000E00CAE0020BB
:10EDC00010AE002008AE002000ED00E030B4EFF3FC
:10EDD0001183102282F312880649074C0A680748FB
:10EDE000013200250A602560DBB2026883F31188D6
:10EDF00030BC70470CAE002008AE002010E000E0F0
:10EE00000F4B1B88014643B90E4B0F4A1B78106805
:10EE10000BB981F00101FAF725BE0C4B5A691AB102
:10EE200018B91A68106058747047094A1868118830
:10EE3000084A92FBF1F2012102605974704700BF49
:10EE4000C4B70020C6B70020C8B70020CCB7002048
:10EE5000E4B7002020A1070038B5254B5C69236B7F
:10EE600073B1636D626BCAB1998A1A88C90592B28F
:10EE700001D5D20700D438BD4FF6F7721A8038BDDD
:10EE8000636D99891A88890692B2EBD59206E9D505
:10EE9000E26ACAB1988880B29047E2E799891A88F5
:10EEA0000D0692B2E0D51006DED5A26A616A8A42EA
:10EEB00019D0A1692569885C98800132B2FBF5F10F
:10EEC00005FB1122A262CFE79B88E2696169DBB290
:10EED0008B54E269E068636D0132B2FBF0F100FB34
:10EEE0001122E261BEE7DA6822F08002DA60BBE755
:10EEF0008439002038B5254BDC68236B73B1636D12
:10EF0000626BCAB1998A1A88C90592B201D5D20733
:10EF100000D438BD4FF6F7721A8038BD636D9989F9
:10EF20001A88890692B2EBD59206E9D5E26ACAB18F
:10EF3000988880B29047E2E799891A880D0692B2C4
:10EF4000E0D51006DED5A26A616A8A4219D0A169AD
:10EF50002569885C98800132B2FBF5F105FB11222E
:10EF6000A262CFE79B88E2696169DBB28B54E269F8
:10EF7000E068636D0132B2FBF0F100FB1122E26147
:10EF8000BEE7DA6822F08002DA60BBE7843900204D
:10EF90002DE9F04F2DED028B95B0804621F0A2FFB8
:10EFA0008E4B1D7825B115B0BDEC028BBDE8F08FFE
:10EFB0008B4B1B685905F6D58A4BDFF880B21B686E
:10EFC0006BB1894ADBF800101368CB1A7C2B06D989
:10EFD000864811600378013303702AF055FA844B98
:10EFE0001B78002B6DD0834C834AD4F81031A8EBEA
:10EFF0000303934201F2278394F81891B9F1000FAB
:10F0000032D17E4F3868FAF797F8C0B201280FD98D
:10F0100002287B4E42F013803378002B42F00881A7
:10F02000D4F81C31A8EB0303B3F57A6F82F0CE82DB
:10F03000D4F82031002B44D094F81831BBB9714B6F
:10F040001B689B7801211E3B00228B4284F818111B
:10F0500084F82C2142F26C823868022104302AF0B4
:10F06000C5F994F8243110E0D4F820314BB3D4F82A
:10F07000283140F6B732A8EB0303934221D994F824
:10F080002431002B01F0D9865C4F013BDBB284F8C0
:10F090002431002B01F00A84D4F8206194F82C214B
:10F0A00016F8011B94F82D313868C4F820610A4421
:10F0B000013384F82C2184F82D31FAF741F8C4F893
:10F0C0002881514BDBF800601B7843B14F4F386803
:10F0D00028B14F4B1B78013B012B41F2F6834D4B7E
:10F0E0001B786BB14C4F3B6853B1DBF80030414C9F
:10F0F00003931A46D4F84431D31A632B01F2938157
:10F10000464F3B78022B01F078863D4E96F87430DE
:10F11000032B01F0B683424B1B7873B1414D2B6832
:10F120005BB1344CFFF70EFDD4F85031039044F638
:10F130001F62C31A934200F231813B4B1B78002BB4
:10F140007ED13A4B1B7843B12A4CD4F8A03203F558
:10F15000C333A033984581F03782354B1B78002BA1
:10F160003FF421AF234E334C334D06F2C1272068C4
:10F17000F9F7E2FF00283FF416AF2068F9F7D4FF53
:10F180002B7880465A1E33B120682A70F9F7D4FFD5
:10F190000028F2D107E703223946781E2FF047FCFA
:10F1A00096F8C03296F8C12286F8C38283F47F4372
:10F1B00083F0FF039B1A1FFA88F89BB2B8EB132F5A
:10F1C000D5D196F8C222DBB29A42D0D1781E1AF07D
:10F1D00087FD2B7818442870C9E700BF68530020CA
:10F1E000F8A6002014AB002034AD002030AD002084
:10F1F00016900020F81F00203F0D0300DCAC00201B
:10F2000028000020E0AC00201890002018AB00205F
:10F210002090002028900020D4AC00205E4C0020DC
:10F220003090002034900020A0900020B190002069
:10F230003A90002040900020449000200CAE002026
:10F24000484C2278A2B1484B9B7A53B1FFF77AFC25
:10F25000464B1B68C31AA3F57A73B3F5FA6F07D848
:10F260002278434B43491868F9F732FF0023237093
:10F27000414CD4F8983203F5C333A0339845FFF4DA
:10F2800060AF3E4DC4F898822B78002B41F0108778
:10F290003B4D2B78002B41F06B8694F89C2239492A
:10F2A0008D5CEA0702F10780AF0701F1C7876807A5
:10F2B00001F188872A0748D5334B344E0D9314AAA1
:10F2C0001146A3F13D0241F8202D0020A3F1400298
:10F2D0000D4603F8400C05910223112151709370E3
:10F2E00028463168FBF720FA28467168FBF71CFABC
:10F2F000F389274903EBC3039B00053381FB0321FB
:10F30000DB17C3EBA101284689B2FBF725FA338A44
:10F3100003EB8303590089B22846FBF71DFA1D4B06
:10F32000059D1B789B0743BF318901F57A7189B22E
:10F330004FF47A712846FBF70FFA0C9B327D591C6B
:10F340000C9128461A7021F05DFD134A94F89C3206
:10F350001178013393FBF1F201FB123384F89C32F4
:10F36000EFE600BF0890002070A80020CC4B0020E2
:10F37000A4900020C88F0020F81F0020A890002033
:10F38000A9900020AC900020C88F002060AD002024
:10F39000676666665CAD0020B090002094F8563138
:10F3A000002B41F0CB85D34B1A6802F00803002BE9
:10F3B00048F603414AF60B404BF60F4349F6074621
:10F3C00004BF03460E4612F0040F4FF0190118BF98
:10F3D0001E46970684F8561103D546F4804646F03B
:10F3E0002006C54B5F79C6F30909002F42F013814F
:10F3F0009B79002B42F01E821F4664204FF0FF3A9B
:10F400004FF0000E0C960D96ADF83E70ADF83CE056
:10F41000CDF842E0CDF846E0CDF84AE0CDF838909E
:10F42000ADF840A08DF84E000CAE0FCEB34F84F86F
:10F4300005E00FC796E80F0007C727F8023B3946DB
:10F440004FF0010E1B0CFE261F20C82201F81E39AA
:10F45000A670A27184F807E0E07094F8660120714C
:10F4600080F0F10383EA0313DAB2130983F0E703B0
:10F4700043EA022383EAC2031BB283EA0312D2B235
:10F48000C3F3072383EA121343EA022383EAC20386
:10F490001BB283F0C80282EA0212D2B2C3F307237E
:10F4A00083EA121343EA022383EAC2031BB283EA0C
:10F4B0000E0686EA0616F6B2C3F3072282EA161291
:10F4C00042EA062200EB0E0382EAC60607EB0E00B4
:10F4D00084F86631268011F8013B734083EA0313F8
:10F4E000DBB21A0982EA162242EA032282EAC30345
:10F4F0001BB29EB281422680EDD183F07C0383EA69
:10F500000313DBB24FEA131E8EEA162E8EEA032E89
:10F510008EEAC30E0FFA8EFE1FFA8EFC784FA4F807
:10F5200000C05FFA8EFE4FEA1C2C84F828C084F8D5
:10F5300027E007F5C77904F1220A38687968BA68C4
:10F54000FB684E460FC610375745B146F5D13868AF
:10F5500030606C4E3B7989F8043006F1270784F857
:10F56000B5E184F8B6C116F8011F2868F9F7E8FD7F
:10F57000B742F8D194F85731002B41F0E484624946
:10F58000DBF8002009780A2084F85701002901F0EF
:10F5900000865E4E01293088079042F251817088C2
:10F5A0000690022902F04F80B0880590032902F0EE
:10F5B0005E81F0880490042902F054810529308985
:10F5C00002F04C810629B6F80A9002F0448107291E
:10F5D000B6F80CC000D0F38994F866110C920F466F
:10F5E00087F0300282EA0212D2B21609484908971F
:10F5F00086F07A0646EA02260988277186EAC20260
:10F60000444EC1EB012186FB017A079E4FF0000EAC
:10F6100066F30F0E069E12B266F31F4E8A44059ED5
:10F62000CDF834E0C917C1EB6A2A002782EA02113B
:10F63000C9B266F30F07C2F30722002682EA11124D
:10F6400060F30F06002007926CF30F00049A8DF808
:10F6500045A063F31F40079B109062F31F4769F3B7
:10F660001F464FF000090E970F968DF8449043EA1D
:10F6700001220DF1300E82EAC106BEE80F0036B25B
:10F6800086F0C80C8CEA0C1C1C4F84F805905FFABD
:10F690008CFCC6F307260FC786EA1C1646EA0C2325
:10F6A0009EE8030083EACC031BB283F0230247F8F1
:10F6B000040B82EA0212D2B2C3F30723089E83EA44
:10F6C0001213384643EA022383EAC20206F1010E0E
:10F6D00020F814194FF0230C1621FE26C82384F8B5
:10F6E00066E102372280E17084F807C0A670A3713A
:10F6F000114611E058AD002044AD0020002000204C
:10F70000FA1F00208721002028920020AC790020D9
:10F71000488F00200308208010F8013B4B4083EA0B
:10F720000313DBB21A0982EA112242EA032282EAB7
:10F73000C3031BB299B2B8422180EDD183F0F40328
:10F7400083EA0313DBB24FEA131E8EEA112E8EEA10
:10F75000032E8EEAC30E0FFA8EFE1FFA8EF7C84EE6
:10F7600027804FEA172C5FFA8EFE84F81EE084F89B
:10F770001FC07168B2683068F36806F5C7770FC7B5
:10F7800030697169B26904F28F1607C704F2AD17C8
:10F7900084F8ADC184F8ACE116F8011F2868F9F7C8
:10F7A000CFFCB742F8D194F85A31002B41F0DB83FB
:10F7B000B44B06931B681922980684F85A2140F12D
:10F7C000EA82B14BB14E1B78990741F12187337D15
:10F7D000042B8CBF03270227FFF7B4F9338A328941
:10F7E0000C9003EB83035B00ADF84A304FF47A7062
:10F7F00033688DF84C700E93F18996F814E07368B5
:10F800008DF84DE000FB02F24FF0000C0CAF4FF012
:10F81000FF30CDF834C010920F93ADF8481011901E
:10F82000BE46BEE80F000597994F0FC79EE80F0030
:10F8300007C73A46182122F81C39E17194F866117D
:10F8400084F805C081F0780383EA0313D8B2030972
:10F8500083F0F60343EA002383EAC0031BB283EA82
:10F860000310C0B2C3F3072383EA101343EA002353
:10F8700083EAC0031BB283F0C80080EA001E5FFA6F
:10F880008EFEC3F3072080EA1E1040EA0E2080EAB5
:10F89000CE0000B280F0180383EA0313DBB2C0F39A
:10F8A000072080EA131040EA032080EAC30301F135
:10F8B000010EFE204FF01E0C4FF0C809A070023759
:10F8C000217184F866E1238084F803C084F80690EF
:10F8D000184612F8011B414081EA0111C9B20B0917
:10F8E00083EA102343EA012383EAC10109B288B203
:10F8F000BA422080EDD181F0180181EA0111C9B22C
:10F900000A0982EA102383EA012383EAC1031BB2B6
:10F910009AB25B490491DBB24FEA122C2280079322
:10F9200084F827C084F826300F4601F5C77A04F121
:10F93000220938687968BA68FB68D646AEE80F00D5
:10F9400010374F45F246F4D13868CEF80000DFF8A2
:10F950004C919DF81C3084F8B43109F1260784F8E5
:10F96000B5C1CA461AF8011F2868F9F7E9FB5745DF
:10F97000F8D1FFF7E7F8069B71681B68328906919A
:10F9800013F0140F4FF47A71D6F800E001FB02F186
:10F9900041F00B860E4694F866A10C908AF06A003E
:10F9A0003C4B3D4FB3F90420CDF834E080EA001021
:10F9B000C0B2030983F0D50343EA002383EAC003FE
:10F9C0001BB283EA0310C0B2C3F3072383EA101308
:10F9D00043EA002383EAC0031BB287FB0207D21766
:10F9E0004FF0000CC2EBA7020698DDF814E0109669
:10F9F00083F0C8070E900F91ADF84A20ADF844C0CF
:10FA0000ADF846C0ADF848C087EA0717FFB2C3F3A8
:10FA10000726BEE80F0086EA171646EA072686EA9A
:10FA2000C7071B4E84F804A03FB20FC687F021031E
:10FA30009EE8070083EA0313DBB2C7F3072787EAD0
:10FA400013170AF1010E47EA032786E8070087EA41
:10FA5000C30384F866E14FF0210A4FF0FE0E1C2725
:10FA6000C8220C3684F805C084F807A084F802E0A8
:10FA7000A6F11C01E7701846A271238010E000BFB8
:10FA8000FA1F002058AD00205CAD002060AD0020C2
:10FA9000002000203CAD00206766666687210020BC
:10FAA00011F8012B424082EA0212D2B2130983EA12
:10FAB000102343EA022383EAC20212B290B2B14297
:10FAC0002080EDD182F0680282EA0212D2B24FEABF
:10FAD000121A8AEA102383EA022A8AEAC20A0FFA71
:10FAE0008AFA1FFA8AF3D74E23804FEA132C5FFA63
:10FAF0008AFA04F1220384F825C084F824A006F5CC
:10FB0000C77E0693F36830687168B26877460FC79E
:10FB1000069B10369E42BE46F4D13388CA4E3B80C7
:10FB20004F4684F8B2A184F8B3C117F8011F2868C2
:10FB3000F9F706FBBE42F8D194F866E1C34AC44E19
:10FB400084F804E08EF0EB0383EA0313D9B20B09C7
:10FB500083F0C50343EA012383EAC1031BB283EAAE
:10FB60000310C0B2C3F3072181EA101141EA00215A
:10FB700081EAC0010CCA09B281F0C80787EA0717F9
:10FB8000FFB24FF0000C0C92C1F30721059A0D93C0
:10FB9000CDF838C081EA171343EA072307CA83EA7E
:10FBA000C7031BB283F0310786E8070087EA07170F
:10FBB000FFB2C3F3072383EA171343EA072383EA59
:10FBC000C703277A607AA17AE27A267B84F805C097
:10FBD0001BB25F4087EA0717FFB2C3F3072383EA2C
:10FBE000171343EA072383EAC7031BB2584080EA8E
:10FBF0000010C0B2C3F3072383EA101343EA0023C3
:10FC000083EAC0031BB2594081EA0110C0B2C3F3BA
:10FC1000072181EA101141EA002181EAC00109B2FD
:10FC20004A4082EA0212D2B2C1F3072383EA1213D6
:10FC300043EA022383EAC2031BB25E4086EA061649
:10FC4000F6B2C3F3072383EA161343EA0623607B65
:10FC5000A17BE27B277C94F811C083EAC6031BB228
:10FC6000584080EA0010C0B2C3F3072383EA1013A0
:10FC700043EA002383EAC0031BB2594081EA011121
:10FC8000C9B2C3F3072383EA111343EA012383EACA
:10FC9000C1031BB25A4082EA0212D2B2C3F3072355
:10FCA00083EA121343EA022383EAC2031BB25F40D2
:10FCB00087EA0717FFB2C3F3072383EA171343EA60
:10FCC000072383EAC7031BB28CEA030C8CEA0C1CE3
:10FCD0005FFA8CFCC3F3072383EA1C1343EA0C236B
:10FCE00083EACC03A17CE27C5A4F1BB2594081EAE3
:10FCF0000111C9B2C3F3072383EA111343EA0123B5
:10FD000083EAC1031BB25A4082EA0212D2B2C3F3A1
:10FD1000072383EA121343EA022383EAC2031BB2D6
:10FD200083F0270686EA0612D2B2C3F3072686EAD4
:10FD3000121646EA022686EAC20636B20EF1010320
:10FD4000B2B231204FF0FE0C0C2184F86631C8238A
:10FD50004FEA122E5FFA86FA2280E07184F802C020
:10FD6000E170A371049E84F814A084F815E0716812
:10FD7000B268F3683068B6F810C00FC727F803CB35
:10FD800084F8A3E184F8A2A119F8011F2868F9F703
:10FD9000D7F94F45F8D194F85E71002F41F0DE801D
:10FDA0002D4B94F866E1B3F90010B3F90220B3F9D2
:10FDB00004309FED2A6A677107EE103ADBF80030D5
:10FDC0000C938EF06A0383EA031306EE901AD9B2FD
:10FDD0000B0983F0D50343EA012383EAC1031BB275
:10FDE00083EA03115242C9B207EE902AC3F30723F4
:10FDF00083EA111343EA0123F8EEE77AF8EEE66AA4
:10FE0000B8EEC77A83EAC1031BB267EE867A66EE64
:10FE1000866A27EE067A002083F0C80CCDED0E7AB4
:10FE2000CDED0D6A8DED0F7A1090119012908CEA45
:10FE30000C160DF13009F6B2C3F3072CB9E80F0028
:10FE40000EE000BFFA1F0020AB210020A0500020D0
:10FE500000200020882100203CAD002088C3E43A27
:10FE60008CEA161C4CEA062C8CEAC60CD04E0FFA13
:10FE70008CFC0FC68CF01E0799E8070087EA07176D
:10FE8000FFB2CCF3072383EA171343EA072386E87C
:10FE9000070083EAC707C8214FF005094FF01E0C81
:10FEA000FE231C200EF10102A17184F85E9184F8FA
:10FEB00007C0A370E070A6F1100184F804E00C36CE
:10FEC000278084F8662111F8013B7B4083EA031305
:10FED000DBB21A0982EA172242EA032282EAC3034A
:10FEE0001BB29FB2B1422780EDD183F0270383EA92
:10FEF0000313DBB24FEA131E8EEA172E8EEA032E8F
:10FF00008EEAC30E0FFA8EFE1FFA8EFCA94FA4F8DC
:10FF100000C05FFA8EFE4FEA1C2C84F825C084F8DE
:10FF200024E007F5C77904F1220A38687968BA68CD
:10FF3000FB684E460FC610375745B146F5D19E4E69
:10FF40003B88A9F8003006F1240784F8B2E184F870
:10FF5000B3C116F8011F2868F9F7F2F8B742F8D1D3
:10FF600094F85F91B9F1000F40F0F287934B1B6852
:10FF7000052284F85F219A0641F11581904ADFED50
:10FF8000917AD18907EE101AB8EEC77A13F0140FE0
:10FF900027EE277A01F071838B4BDFED8A6AD3ED70
:10FFA000007AF8EEE77A67EEA67A94F866C1874B96
:10FFB000874AB3F90410B2F90620864E86488DEDC3
:10FFC0000D7A8CF0220383EA0313DFB23B0983F03E
:10FFD000590343EA072383EAC703B2F5FA6F1BB25A
:10FFE000A8BF4FF4FA6283EA0317FFB2B2F57A7F33
:10FFF000C3F3072383EA1713B8BF4FF47A724FF0A5
:020000040801F1
:10000000640E43EA0723A2F57A720EFB02F283EA3A
:10001000C70786FB02E680FB01E03FB2C917D21793
:10002000C2EBA612C1EBA0034FF0000A0CA987F0A7
:10003000C806CDED0E7AADF84220ADF84030CDF8CF
:1000400030A0CDF83CA08E4686EA0616F6B20591A1
:10005000C7F30727BEE80F0087EA161747EA062707
:1000600087EAC606524FDEF800E084F804C00FC7E6
:1000700036B286F04A0383EA0313DBB2C6F30721E4
:1000800081EA13113A4641EA03210CF1010C81EA9D
:10009000C303142042F810E9FE264FF04A0E002157
:1000A00084F866C14FF0C80CE0702380043784F8F0
:1000B00007E0A670617184F806C0184612F8011BAB
:1000C000414081EA0111C9B20B0983EA102343EAD6
:1000D000012383EAC10109B288B2BA422080EDD17E
:1000E00081F0140181EA0111C9B24FEA111E8EEAB2
:1000F000102E8EEA012E8EEAC10E2E4B0FFA8EFEC6
:100100001FFA8EF61F464FEA162C5FFA8EFE84F811
:100110001CE084F81DC0386859689A68DB68B7F835
:1001200018A0049726803E4607F5C7770FC73069A9
:10013000716903C704F28F16A7F800A0374684F848
:10014000ABC184F8AAE104F2AB1A17F8011F2868C2
:10015000F8F7F6FFBA45F8D1204B214A1B78127800
:10016000013B12F00100DBB214BFC0214021172B6C
:1001700003D81C4A134493F830901B4B1A889707F6
:100180001ABF002341F01001012312F4027F18BFAF
:10019000022312F0100F18BF062312F0200F18BF11
:1001A0001023002841F008824FF0030C1EE000BF2E
:1001B00000200020FA1F00208721002058AD0020D9
:1001C00060AD00200AD7233C38AD00203CAD0020B4
:1001D000AC790020D34D621067666666FC4700204C
:1001E000644F0020F8EC03084A8F002094F866E181
:1001F0000C938EF0460383EA0313DAB2130983F0FB
:10020000920343EA022383EAC2031BB283EA031088
:10021000C0B2C3F3072282EA101242EA002282EA45
:10022000C00212B282F0C80787EA0717FFB2C2F312
:10023000072282EA171200238DF837C0032042EA12
:10024000072C059A8DF834908DF835308DF83610DE
:100250008DF8380007CA8CEAC70C0FFA8CFCD04F17
:10026000E3718CEA0C1903C75FFA89F9CCF3072C08
:100270008CEA191C4CEA092181EAC90994F808C0E2
:100280003A700FFA89F98CEA090C8CEA0C1C5FFAB7
:100290008CFCC9F3072282EA1C1242EA0C22607A23
:1002A000A17A94F80B90637182EACC0212B25040AA
:1002B00080EA001C5FFA8CFCC2F3072080EA1C1065
:1002C00040EA0C2080EACC0000B2414081EA0111F2
:1002D000C9B2C0F3072282EA111242EA012282EA7D
:1002E000C10212B289EA020989EA09195FFA89F999
:1002F000C2F3072282EA191242EA092294F80CC0DA
:10030000607BA17B84F804E082EAC90212B28CEA25
:10031000020C8CEA0C1C5FFA8CFCC2F3072282EA06
:100320001C1242EA0C2282EACC0212B2504080EA4D
:100330000010C0B2C2F3072282EA101242EA002281
:1003400082EAC00212B2514081EA0111C9B2C2F37D
:10035000072282EA111242EA012282EAC102E17B0B
:1003600094F8109013B281EA030282EA0212D2B228
:10037000C3F3072383EA121343EA022383EAC20387
:100380001BB289EA030282EA0212D2B2C3F3072344
:1003900083EA121343EA022383EAC2031BB283F007
:1003A000320282EA0212D2B2C3F3072383EA1213A3
:1003B00043EA022383EAC2031BB29AB24FF0FE0C57
:1003C0005FFA83FB0920C8210EF1010E84F802C0F8
:1003D0004FEA122CE070A17184F866E1228084F863
:1003E00012C084F811B0049B186859689A68B3F871
:1003F0000CA007F5C07EAEE8070007F5C8778EF8B9
:100400000290AEF800A084F8A0C184F89FB116F85D
:10041000011F2868F8F794FEB742F8D1039BC4F88F
:100420005031FEF78ABEDFF898A15E4EDFF8949156
:10043000412028F087FFBAF9023086FB0320DB1742
:10044000C3EBA00080B228F061FFBAF9003086FB50
:100450000320DB17C3EBA00080B228F057FFBAF9E6
:10046000043086FB0320DB17C3EBA00080B228F02A
:100470004DFF99F800103868F8F762FE94F848A12B
:100480001AF0010600F0F784474B06931B689A06A2
:1004900073D5464B464E1B789B0741F15180337D07
:1004A000042B8CBF4FF0030A4FF0020A472028F0BC
:1004B00049FF306828F0F6FE706828F0F3FE3D4AE8
:1004C000F3893868A2FB0323C3F347131946049347
:1004D000F8F736FE069B99F800101A68049B12F094
:1004E000140F83EA010389F8003040F067863389EE
:1004F000642000FB03F028F0D5FE367D38684AEA18
:100500008606F6B23146F8F71BFE99F800303868D7
:100510005E40314689F80060F8F712FE94F848A171
:10052000BAF1000F29D1244E4F2028F00BFF30687C
:1005300028F0B8FE706828F0B5FE504628F0B2FEEC
:1005400001213868F8F7FCFD184A99F80030167850
:10055000386806F00106314683F0010389F800305F
:10056000F8F7EEFD99F8003038685E40314689F8BA
:100570000060F8F7E5FD94F848A1039B0F4AC4F822
:1005800044310AF10103DBB2A2FB0312D20802EBF1
:100590008202A3EB420384F84831FEF7B1BD00BFED
:1005A000002000206766666658AD00205CAD002024
:1005B00060AD00201F85EB51A0500020CDCCCCCCED
:1005C0003CAD0020D8AC002094F8A432C24AC4F854
:1005D000A08202EB8302926C42B314AD04F2AB230F
:1005E000BE4E45F8203D002104F2BD2331800D931D
:1005F00080211523A52784F8AA32284684F8A91259
:1006000084F8A872904728463188FAF7CBF80C9DF9
:10061000B34804F52A716D1A152DA8BF15252A4671
:100620002BF09EFFAF4A94F8A4321570AE4A013306
:1006300082FB0312A2EBE37202EB42029B1A84F8E4
:10064000A432FEF78ABDA94AA94BD4F81411DBF8ED
:1006500000001B88D77AA74A401A4FF47A71DEB29D
:1006600001FB07F11B0A9677167588424FF00006CA
:10067000D37753759670167180F0D1849E4E9F4B40
:10068000D6F800C01B689E4E9E48DFF8989201681D
:100690008068DFF894E286FB0376DB17C3EB661312
:1006A00003F5FA739BB293761B0AD37689FB017329
:1006B000C917C1EBA30189FB00791177C017091293
:1006C000C0EBA90051778E4982F820000CF5EA436F
:1006D000001281FB0C71303382F821004FEAEC707C
:1006E0001B12C0EB6110884E9EF800E082F82330A8
:1006F0007830864B82F824000CF13001307D039075
:100700001EF0020F82F82210987600F08584D6F849
:1007100000E07F4AD6F804A07E48DFF810C282FBD2
:100720000E194FEAEE7182FB0A72C1EBA9514FEA32
:10073000EA79C9EBA25200FB01E900FB02A009EB38
:10074000490900EB40004FEA49094000049207467E
:100750008CFB0920801405908CFB072CF089049AEF
:100760003689079702EB820206F5FA7600EBC000A5
:1007700002EB8202B6B204960892059E82000992AC
:1007800001EB81014FEAE972B01A01EB8101624E7F
:1007900006910246039906FB1292069E40B2052975
:1007A00000EB86004FEAE7714FEAAC4C5A4E0590D9
:1007B000ACEB0100014606FB1070089E504FDFF8BD
:1007C00070C14FEADA7A49B201EB86014FEADE7E68
:1007D00087FB006983F80EA087FB026A099F83F8F4
:1007E00009E0DFF850E13E468EFB066EBCF8006083
:1007F00003969DF810605E75049EBDF814C083F8E2
:100800000AC04FEA162689B204964FEAE2724FEA0E
:10081000E777424ED973C2EB6A12C7EBAE174FEAC5
:100820001C2A4FEA112E4FEAE0700399368883F8AC
:100830000BA0C0EB691083F810E04FEA22291A736D
:100840009DF810209A754FEA202CC7F3072A4FEA2B
:10085000112134BF4FF0320E4FF0330E9DF80C20B3
:1008600083F80D90587483F812C0DF7183F808A0E4
:10087000DA74197583F81BE01E77C4F81081FEF74F
:10088000BBBBDFF8B490D9F80000F8F745FC0028AE
:100890003EF441ACD9F800000121F8F739FC0222FE
:1008A000002386F874203B70FEF735BC94F82C11B9
:1008B00094F82D3138684A1C013384F82C2184F8CF
:1008C0002D31F8F73DFCFEF7FABB154CDFF86C90C4
:1008D0004FF0000A3FE000BFF8EC0308848F0020CF
:1008E000B4490020C949002056555555E04F002015
:1008F000D84F0020489000202CAD002038AD0020BB
:100900001F85EB5120AB002060AD002074900020CB
:100910006BCA5F6B806967FF40420F00AA500020DE
:10092000F81F0020676666665CAD002083DE1B430F
:10093000A8500020D34D6210604D002028000020F8
:100940001B2B00F06F820D2B00F04B814FF0010349
:1009500089F801303868F8F7EFFB002839D038689B
:10096000F8F7E2FB83B27E2BDBF800202AD099F85F
:1009700001100029EED194F82E21002AE0D07D2B21
:1009800000F0368294F83CE1BEF1000F04D080F014
:100990002003DBB284F83C11511CC9B2224409295E
:1009A00084F82E1182F8303100F016820829D1D84F
:1009B000B4F83A21134403EB132303F0FF03A4F824
:1009C0003A31C7E784F82EA184F82FA189F801A055
:1009D000C0E794F83D3133B194F8313184F83D01EA
:1009E000302B00F0C18594F82F21C54BC549DFF8A5
:1009F00050A3DFF850E391464A46002A3EF46FAB1D
:100A0000DBF80020921B012A24D894F83E21002A0A
:100A100040F01E8294F83FC133F81C00F8B94FF043
:100A2000010284F83F210A689706E5D59AF800206C
:100A30009007E1D5B44EB549F2894FF4F36303FB57
:100A400002F381FB0321DB17C3EB61114FF4036059
:100A500028F0B2FC002384F82F31FEF740BB0CF1E4
:100A6000010C5FFA8CFCB0F5E06F84F83FC100F038
:100A700098801BD8B0F5047F00F0238135D8B0F5FD
:100A8000887F00F0CD80B0F5007F00F0B380B0F536
:100A9000807FB1D10A685207AED59D4B196828F006
:100AA0008BFC002384F82F31FEF719BBB0F5026FE1
:100AB00000F05A816AD8B0F5E46F00F08180B0F59B
:100AC000006F00F0D680B0F5E26F95D1914BDA6BF4
:100AD000998A642303FB02F393FBF1F128F06CFC89
:100AE000002384F82F31FEF7FABAB0F5826F00F0D8
:100AF0005181B0F5C06F00F02781B0F5806F7FF4B1
:100B00007BAF94F840310133DBB2032B00F2AD81AF
:100B100042F2107184F8403101FB03F17E4B1B88D7
:100B2000002B40F0A08101317C4B1B78DB077C4B14
:100B30001B8848BF0431DF0748BF0A31980748BF08
:100B400014311A0648BF2831DF0548BF283158073D
:100B500048BF64311A0748BFC8319F0548BF01F537
:100B6000C871980648BF01F57A71DA0648BF01F5E9
:100B7000FA615F0648BF01F57A614FF4806028F0A2
:100B80001BFC002384F82F31FEF7A9BAB0F5046FDF
:100B90001AD0B0F5116F52D0B0F5036F7FF42CAFBF
:100BA00041E75C4B91469A6B998A642303FB02F3FD
:100BB00093FBF1F128F000FC84F82F91FEF78FBA37
:100BC000544B91461A6CEFE7564BB3F9041001EB06
:100BD00081019146490028F0EFFB84F82F91FEF740
:100BE0007EBA4FF0010184F82E1184F83031A4F858
:100BF0003A21AFE69EF80620002A3FF4FDAE4A4BAC
:100C00004A491B6881FB0321DB17C3EBA1014FF4A9
:100C1000007028F0D1FB002384F82F31FEF75FBA73
:100C20000A6852077FF5E8AE414B4FF488701968A7
:100C300028F0C2FB002384F82F31FEF750BA9EF84B
:100C40000520002A3FF4D8AE3A4A107800283FF435
:100C5000D3AE394B1B8803EB8303590091FBF0F1B2
:100C60004FF4116028F0A8FB002384F82F31FEF721
:100C700036BA0A6897067FF5BFAE9AF8002090074B
:100C80007FF5BAAE1CF0010F1F4E204900F05C84C6
:100C9000726882EAE273A3EBE27303EB5303A1FBF6
:100CA0000331C908002AACBF41F0004141F0404186
:100CB0004FF4006028F080FB002384F82F31FEF70A
:100CC0000EBA9EF80520002A3FF496AE194A107815
:100CD00000283FF491AE194B5B7B002B00F094840D
:100CE000154B1B8893FBF0F000EB800041004FF4A4
:100CF000047028F061FB002384F82F31FEF7EFB970
:100D0000F8EC030858AD002060AD00201F85EB51C2
:100D100038AD0020E4AC0020788F0020644F002024
:100D20004A8F00203CAD002020AB0020676666663D
:100D30002CAD0020EE4F0020D84F0020E04F0020C7
:100D40005CAD002044AD00209EF80620002A3FF450
:100D500053AEC34B4FF4C060996828F02DFB0023BD
:100D600084F82F31FEF7BBB90F68BF067FF544AE9C
:100D70009AF800C01CF0020F3FF43EAEB94E338922
:100D80006421914601FB03F128F016FB84F82F91B2
:100D9000FEF7A5B90A68900640F1F180B24BB14E5A
:100DA0001878317D00F00203002B0CBF00234FF4B4
:100DB0007A7340F6B83208BF4FF4FA6210F0010FB0
:100DC00018BF134619444FF4826028F0F5FA002347
:100DD00084F82F31FEF783B9B4F83A21C2F1FF024B
:100DE00093427FF4B3AD4FF0010384F83D31ADE59C
:100DF0004FF0010384F83C31ACE5FDF7A3FE9B4BBB
:100E00001B68C01A40F6B833984200F21E81DFF822
:100E10009CA29AF804303A2B00F0BA8200233B706F
:100E2000FEF779B93868F8F787F900287FF48EADB6
:100E30004FF0010384F82F318CE5C4F8203184F899
:100E400018318B4F28F006FB94F82431FEF71DB9BA
:100E50008849062018F0CEFF002384F83E0184F86C
:100E60002F31FEF73CB902315EE6012384F84031B0
:100E700042F2107152E6804B1B88D80513D4D90674
:100E800000F17A839A0600F1F183580600F1F383AA
:100E9000190700F1F983DA0700F1148413F0020F47
:100EA0000CBF04260C26754B754A1B78D27803F0CC
:100EB00001030AB143F002035320049328F042FADD
:100EC000704A128802EB820202EB8202900080B22A
:100ED00028F01CFA002028F019FA6B4A6B49128896
:100EE0003868C2EBC212520081FB023111444FEA52
:100EF000E27ACAEB612A5FFA8AFA5146F8F720F9DA
:100F000099F80020049B38681E438AEA020A0021EF
:100F100089F800A0F8F714F931463868F8F710F9A5
:100F200099F8003038687340DBB2194689F8003010
:100F3000F8F706F994F848A1FFF7F2BA013B84F8F4
:100F40005631FEF717BB013B84F85731FEF72BBC37
:100F500009F1FF3984F85F91FFF760BA013F84F827
:100F60005E71FEF7FDBF013B84F85A31FEF713BFF7
:100F700047493A2018F03EFF2870FEF7E2B8454A8C
:100F80001268120600F1FA82434A127B002A3FF4EB
:100F900033AD94F84111032900F28A83DFE801F0B0
:100FA000322819023D4B1B6859799A79DB7901F196
:100FB000407101EB022101EB0341002384F8413130
:100FC0004FF4826028F0F8F9002384F82F31FEF7FF
:100FD00086B8334B1A68137A507992781B0403EB66
:100FE000002313444A1C84F8412103EB0161E7E725
:100FF0002B4B1A68D379107952781B0403EB00232A
:101000001344EFE7264B1A689379D07812781B04C3
:1010100003EB00231344E5E72D22DA762DE4214B80
:10102000DBF800101B78C4F81411013B012B3FF6CC
:1010300025AB1021022391701371FFF71FBB28F01D
:10104000F9F901233370FDF7F3BF174AB2F84A31BB
:1010500000210133A2F84A313970FEF75CB800BFB5
:1010600020AB002060AD00205CAD0020644C00206F
:10107000DCAC0020B19303084A8F0020644F0020AD
:10108000548F0020D84F0020488F00200308208074
:10109000650E0308F8A60020E04F0020D4AD002024
:1010A00000920020508F0020F81F00204C4C0020A0
:1010B000A64EA74B00930024A6F13F01A54BA64ADC
:1010C0000A9106F8404CA5490B960CA8F9F742FC8A
:1010D0000A9E731C0A9334700A9B2922591C0A9198
:1010E0001A700A9BEA22591C0A911A700A9BC8229C
:1010F000591C0A910CA81A702AF08AFC471C0CA9EA
:101100003A460A982BF02CFA0A9AD31901330A931B
:10111000D4550A9B5A1C0A921C700A9B5A1C0A92AC
:101120001C700A9B5A1C0A921C700A9B5A1C0A9239
:101130001C700A9B5A1C0A921C700A9B5A1C0A9229
:101140001C700A9B5A1C0A921C700A9B5A1C0A9219
:101150001C700A9B5A1C0A921C700A9B5A1C0A9209
:101160001C700A9B5A1C0A921C700A9BFF22591C75
:101170000A911A700A9B0122991814A80A911A70F0
:1011800050F8283D9B1B33701FF03CFE2C70FDF780
:10119000D8BF8C468946084604910591069107916F
:1011A0000B46FEF719BA9FED6E7A13F0140F08BFC5
:1011B000F0EE477A7EF4F0AEFEF7F7BE694B1868A2
:1011C000FFF799B9684A614B12680D93A3F1400784
:1011D000002103F8401C2123D100BB7040F13A826A
:1011E00062490326624B1B885A0500F12982D80701
:1011F00000F13E8203F002035E4A002B1CBF03266F
:101200001146DFF88891324648462BF0A9F906EBE3
:10121000090314A80133A9F1020140F8203D00227E
:101220005B1A06F809207B701FF0ECFDFEF742B850
:10123000C4F81C8186F80090FDF7FABE434A4E4B75
:101240000D9214AEA2F13D0046F8200D19884B4FC7
:10125000A2F1400300204FF00A0E02F8400C0822D1
:1012600083F801E030469A70F9F776FA3B68444912
:10127000DA1781FB0313C2EBA30399B23046F9F7E7
:101280006BFA09F03DFDBF680C9B3A0C591C0C91A0
:101290001A700C9B3A0A591C0C911A700C9B5A1C20
:1012A0000C921F700C9B5A1C0C92187030461FF049
:1012B000A9FDFDF7FCBF334F9FED338AB7F902203C
:1012C00022480D9007EE902AF8EEE77A14AE67EE0A
:1012D000887AA0F13D01FDEEE77A46F8201D00F87E
:1012E000403C0823CDED037A00F83F3C1E23BDF8B7
:1012F0000C1000F83E3C3046F9F72EFAB7F90030F2
:1013000007EE903AF8EEE77A304667EE887AFDEE1F
:10131000E77ACDED037ABDF80C10F9F71DFAB7F9AD
:10132000043007EE903AF8EEE77A304667EE887AB6
:10133000FDEEE77ACDED037ABDF80C10F9F70CFA63
:1013400030461FF05FFDFDF7AFBF00BFC88F002024
:10135000F7910020E4200408EC200408F820040899
:101360000000000038AD002060460020D0200408B6
:101370004A8F0020E0200408D84F002020AB002036
:10138000676666663CAD002058A08B418B8F0020BD
:101390009AF80240C4B1013CE4B2013454445146CD
:1013A000002211F8013B534083EA0313DBB2120A17
:1013B000DE0042EA03228C4286EA131382EA030229
:1013C000EFD1002A7FF42AADC04AC14EC14B12882A
:1013D000C149C24CF261DFF838931A6809689B680A
:1013E000F262B4F84A21F066F364D9F80000F163C0
:1013F000F265F6F7C1FE039000287DF487AE022166
:10140000D9F80000F7F784FE94F84C319AF80320DD
:101410000492642B4FF0040286F8742040F07C8123
:1014200094F84D31072B04BF9DF80C3084F84D31F2
:1014300094F84D31079306EB031ADAF80410039180
:1014400008462AF0E5FADAF8081006915FFA80FA01
:1014500008462AF0DDFAC0B205900AEB0002079BAD
:101460009F48039903900832C27123F00F02864609
:101470008272059803F00F0300EBCA008EF80D305E
:1014800052468EF80E000EF10F002BF069F8954BC6
:10149000059A06990AF1090018442BF061F803989F
:1014A000C37903F1010ACBB1013B5FFA83FC0CF174
:1014B000080CDFF860E284440023073010F8011BB9
:1014C00059408B00CA0883EA410302F018024B40DE
:1014D0004EFA02F253408445DBB2EFD1814A0498C0
:1014E0000AF802301DF054F994F84D31002201330E
:1014F00084F84D3184F84C21039BDDF80CA09B78D7
:101500005BB11AF80510D9F80000F7F719FE01359C
:101510009AF80230EDB2AB42F3D894F84C31032282
:10152000013384F84C3186F874203A70FFF7ABB978
:1015300002213868F7F7ECFD94F82431FDF7A5BDDA
:101540004FF0010AFEF7B2BF326882EAE273A3EB02
:10155000E27303EB5303A1FB0331C908002AB8BFB0
:1015600041F08041FFF7A4BB5F49881F27F0A6FD2B
:1015700084F83E01FFF737BA342694E4102300269E
:10158000042218460CA98DF830308DF831208DF8E2
:1015900032608DF833608DF834608DF8356027F057
:1015A000EBFE84F82F61FDF79ABD4B4B1E6806EBEE
:1015B00086067600FEF7EFB94C4AD278002A0CBFB7
:1015C0004FF0040C4FF0050CFEF710BE01233868F5
:1015D0003370F7F7A9FD06463868F7F7A5FD7206E0
:1015E0007DF426AD8A2851D08E287DF421AD94F863
:1015F0001831002B7DF438AD3D4BC4F820312D233C
:1016000084F82431FDF71BBD304B1888FFF76CBB05
:101610000127FEF7E1B82D499A790B8803EB830384
:1016200003EB83039F00BFB2002A00F01181294B16
:101630001B680FFA83FA09F063FB40B2FDF7E0BEC6
:1016400003262C49DDE59C469946184604930593EC
:10165000FDF7C2BF284B294A1B68294903F48003C0
:10166000002B16BF114604260326BBE524261AE4E8
:1016700024490426C5E5102615E4138907EE903A9F
:10168000F8EE677AFEF791BC20260CE41E4B1B682F
:101690009B067DF5CDAC94F81831002B7DF4E4ACBD
:1016A0001A4BC4F820312D2384F82431FDF7C7BC30
:1016B0004B1CDBB2042B84F841314FEA01613FF44B
:1016C0007CAC7DE40826FFF7EEBB00BFD84F0020BE
:1016D0002800002020AB002038AD0020F81F00209B
:1016E000C4750020CA75002030210020548F0020CE
:1016F00048900020D4200408F8A60020D020040838
:10170000C8200408D820040858AD00207490002098
:10171000604D00200007090E96F875A05749059501
:101720001AF00F0F04BF0AF1010A5FFA8AFABAF140
:10173000070F28BF4FF0010A4FEA0A1C06EB0C0303
:10174000187C4F4B03930A18002392F824104C4A3C
:1017500093725FFA8CF31A464A4B964606EB0C02DC
:101760004EEA000001291870D26803F101000CD97B
:101770000239C9B28D1C1D44034603F8012BAB424C
:101780004FEA1222F9D101310844B44422F0600337
:101790000AF1010A9CF811205FFA8AFA1343BAF1A0
:1017A000080F037000F1010340D04FEA0A1C06EB5A
:1017B0000C01344A087C314901449A1A91F82410EA
:1017C00055180EF1100E132D5FFA8EFEC6DD059D25
:1017D0000398DFF8BCE0D2B2931DDBB243F04001C6
:1017E000C17103F1010CCBB10532D3B20833C31878
:1017F00005930EF10100002310F8011B59408B00E6
:1018000083EA4103CA084B401F4902F0180241FA1B
:1018100002F25340059A8242DBB2EDD104980CF8F3
:101820000E3086F875A01CF0B3FF65E6154A059DDD
:101830009A1ACDE7154B6420B3F900A0FDF7E0BD7F
:101840009C4699461846049305930693FDF7C4BE3B
:101850004FF0FF33EDE69C46FDF7BEBE9C46994631
:10186000FDF7BABE9C4699461846FDF7B5BE9C46A4
:10187000994618460493FDF7AFBE00BFF8EC030885
:10188000C4750020D17500200007090E20AB002090
:10189000CA7500202DE9F04F95B0B0F908500D81C0
:1018A000EDB2442D00AF0C46904600F03182064662
:1018B00043D9812D00F0728200F29880542D00F0FF
:1018C000CC8040F2BD816E2D00F0F081802D40F083
:1018D000D080AA4B93F800A00AF1020A1AF0FF0A7E
:1018E00000F09780A64BDFF8D482A64EDFF8D0B286
:1018F0009A4403F101090A2516E0322D00F00C8309
:10190000A5F13C00C0B2132840F20C8300232268EA
:10191000511C216015702268D14502F1010121603E
:10192000137076D019F8015B0A2DE6D1BBF80030B0
:10193000FF2BA8BFFF23DBB2E9E7052D00F0D6811E
:1019400020D8022D00F0818040F26781032D00F045
:10195000A381042D40F08D808B4920462A46F8F75C
:10196000D9FE00212046F8F71DFF22680021531CF4
:101970000125236028462B46543711706381BD46EC
:10198000BDE8F08F242D5ED040F2D980282D00F0E4
:10199000C781382D6DD10A687C4B0125511C21600F
:1019A00015702268052150192060117022680A21E3
:1019B00050192060117022680021501920601170A8
:1019C00022681978501920601170226859785019CE
:1019D0002060117022689978531923602B4611708A
:1019E000284654376381BD46BDE8F08FA02D18D03E
:1019F00040F2E880B82D00F0CF81FE2D39D1644D42
:101A000005F1080635F8021B2046F8F7CBFEAE427A
:101A1000F8D101252B46284654376381BD46BDE8E1
:101A2000F08F5C4B08461968F8F7A4FE5A4B204625
:101A30001968F8F79FFE594B196820460125F8F7F9
:101A400099FE2B46E7E7564BF6E704225549204618
:101A50000125F8F75FFE2B46C2E70B6800215A1CF0
:101A60002260197022680125531923602B461170DA
:101A7000B6E721462846FAF735FE03460028C8D1C6
:101A8000742D00F0FB80772D0DD132687168914282
:101A90001EBF531C33601178434A08BF19462046C5
:101AA00026F076FAB5E7F52D01F0AB83762D00F040
:101AB000DD81472D00F0888271683368292DA1EB04
:101AC000030200F0558340F25D82392D00F03E8321
:101AD000532D40F06F83591C31601978032900F2AF
:101AE000E0854B1E314D3248DBB203EB430305EB7F
:101AF000430301705D7800298BD0531EDBB2AB42EB
:101B000040F0CF850022C0F80620C0F80220827283
:101B10005BB1591C33680144421C0133336013F834
:101B2000010C02F8010F8A42F7D1224B1B78002BDF
:101B30003FF46FAF01251EF05BFA2B4650E7202DD6
:101B400097D10B681C4D591C6A7821601A70236864
:101B50002A78591C21601A702368AA78591C2160C0
:101B60001A7029892046F8F71DFE23686A79591CE6
:101B700021601A702268A979F9E600BFD54E0020CD
:101B80004CED0308F0260020F7910020D9920020A8
:101B9000F84E0020107AFF1F147AFF1F187AFF1FDB
:101BA000249400206421040889720308A0F3030828
:101BB000F0810020603A002044AD00206766666630
:101BC00018270020822D7FF454AF0B68BB4ABC4D10
:101BD0001178BC4A581C2060197011892046F8F70A
:101BE000E1FDB94B22681B88FF2B02F10101A8BF60
:101BF000FF2321601370A96881F3100189B2204688
:101C0000F8F7D0FD296801F30F0189B22046F8F7F3
:101C1000C9FDAE4B22681978A9E6012D7FF429AFE2
:101C20000B680022591C21601A7023685A1C22601C
:101C30001D7022682421531C23602B461170CFE6AF
:101C4000522D7FF416AF0A68A14D531C0321236067
:101C500005F10C0E11702B46062001212268561C3E
:101C6000266011702268734502F101012160107035
:101C700000F0DD809979D8790633EFE73268716832
:101C800091421EBF531C33601178924A08BF194617
:101C9000204626F07DF9BCE60B685A1C0A601D70D0
:101CA0000B680222591C21601A705EE6864B0A6896
:101CB0001B88834DFF2BA8BFFF23511C216013708D
:101CC000A96881F3100189B22046F8F76BFD824BB9
:101CD00020461988F8F766FD296801F30F0189B2DB
:101CE00020460125F8F75EFD2B4679E60B227B495D
:101CF0002046F8F70FFD082279492046F8F70AFD3B
:101D00000125072277492046F8F704FD2B4667E6B0
:101D1000002A3FF47EAE744B136001252B465FE62C
:101D20000B68DFF8E891714E591C022221601A708D
:101D300023684FF006085A1C226083F8008023684D
:101D40000A22591C21601A70236801255A19226041
:101D50001D70B9F800102046F8F724FDB9F80210FC
:101D60002046F8F71FFD23685A19226083F8008087
:101D700023685022591921601A70236800225919CA
:101D800021601A7031882046F8F70CFD71882046D2
:101D9000F8F708FD2B4623E6554B4DE6554B1E78CC
:101DA000033616F0FF063FF434AE534BDFF8608184
:101DB0001E4403F1010A4FF00A0920E0B9F1500F67
:101DC00000F0A880B9F1320F00F0C180A9F13C0009
:101DD000C0B2132840F2BE800025294623685A1C51
:101DE0002260204683F80090F8F7DCFC2946204664
:101DF000F8F7D8FC56453FF40CAE1AF8019BB9F140
:101E00000A0FDBD13D4B9D68196805EB85054FF640
:101E1000FF736D009D42A8BF1D469942A8BF194699
:101E200025EAE57521EAE171ADB289B2D6E7344B16
:101E300021681A78481C20600A70002A3FF4E9AD36
:101E4000013AD2B202EB420205EB42025578002D74
:101E50003FF4DFAD01351D440133226813F8011F43
:101E6000501C9D4220601170F7D1D2E53268511CA0
:101E700031601278002A01F0A682102A07BF214B98
:101E800093E842001E46314625686B1C23602046BD
:101E90002A70F8F76FFC31462046F8F76BFC1A4BB6
:101EA00020461968F8F766FC20460021F8F77AFC0E
:101EB00000212046F8F776FC57E500BFEE4F0020E2
:101EC00020AB002044AD0020D84F0020508F0020D0
:101ED000A0F30308317E0308488F00206C2104081A
:101EE000782104088421040815C60008D82600209B
:101EF00010410020D54E00205CED0308A4260020F0
:101F0000F0810020C0240020084E00207C4E0020DC
:101F1000E8260020A24B76E73388FF2BA8BFFF23DB
:101F2000DBB2F4E417F062FE00283FF4EFAC037874
:101F30000A2B25D8B0F9023088FB0312DB17C3EB5C
:101F4000A2039BB2FF2BA8BFFF23DBB2DFE498E81C
:101F500022005AE717F04AFE00283FF43DAF03780D
:101F60000A2B3FF639AFB0F90430B0F9061003EB95
:101F7000830383F3500521EAE171ADB289B22DE705
:101F80000023E2E7212D40F015811A46591C3160EB
:101F9000844D12F8021B697032605A782A70DA1C7C
:101FA00032609B78AB703046F8F7A2FB336828812B
:101FB000591C1A46316012F8021B697132605B7855
:101FC000AB7101252B460BE5726835687B623046A4
:101FD000551BF8F775FB052D38627B6A01F2D0813D
:101FE0008026B346012594E80600521A103AB24200
:101FF000B8BF1FFA82FB6C4A396A92683A61521A7A
:102000009345396A7B622046FA6088BF1FFA82FBDB
:10201000F8F7B0FB7B6A002B01F09181002D41F0B5
:102020004D812368C7F800D05D71C0B00533C7F893
:1020300008D0FB61BBF1000F01F026823B6A3A69D0
:10204000934281F02682AA463E6A7D627C608025AA
:102050005446FB681C1B544BB4F5807F28BF4FF4DB
:1020600080749B6832199A4288BF9C1BF9F734F838
:102070002246BC6830462146F9F7AEF8F969B861E6
:1020800004EB000C0B787B6164452ED2DFF81C91C9
:102090000CF1FF3C04F1FF3E1EF8013F09EB830207
:1020A00019F823405688ECB100234FF4004204F1A4
:1020B000FF3816424FEA520202D0087828430870CF
:1020C0006D0806D10AF1010A4D701FFA8AFA013132
:1020D0008025D34503D8F44532D8984530DC013308
:1020E0009C42E6D1F445D7D1F9617B6ABA691344C1
:1020F0009BB2D3457B6206D97B6A3A6A1C46D618E6
:102100003B699E42A5D37C68802D1CBF0AF1010368
:102110001FFA83FA0AF1020189B22046F8F742FB5E
:102120002368796A01255A19226020461D70F8F744
:1021300039FB2368534423602B46D7F800D04FE483
:10214000FB697C681A463B7D1370DDE75A1C3260E0
:102150001A780A2A01F028813046F8F7D5FA304675
:10216000F8F7D2FA01253046F8F7CEFA2B4637E4D5
:102170005A1C32601B780A2B01F00F81502B41F062
:1021800038803046F8F7B4FADFF82480A8F8000069
:102190003046F8F7ADFA0125A8F802002B461FE4F7
:1021A000DC26002044AD0020740300206CED030801
:1021B000D82600200B3DEF2D00F2738201A050F8CD
:1021C00025F000BF1D2E0108A3260108A326010843
:1021D000A3260108A3260108A3260108A3260108B7
:1021E000A3260108A3260108A3260108A3260108A7
:1021F000A3260108A3260108A3260108A326010897
:10220000A3260108A3260108A3260108A326010886
:10221000A3260108A3260108A3260108A326010876
:10222000A3260108772E0108A3260108552E0108D0
:10223000A3260108F32D0108A3260108A3260108FF
:10224000A3260108CB2D0108A32601087730010839
:10225000A326010845300108A32601081F30010804
:10226000A32601080D300108A3260108B52F010897
:10227000A3260108352F0108A3260108A32601087B
:10228000A3260108A3260108131A0108A3260108A2
:10229000E52E0108A3260108A3260108CB2E01087C
:1022A000A3260108A9310108A3260108A3260108D5
:1022B000A3260108A32601089D310108A3260108D1
:1022C000A3260108A32601081F310108A32601083F
:1022D000D1300108A3260108A32601085F310108B7
:1022E000A3260108A3260108A3260108A3260108A6
:1022F000A3260108A3260108A3260108F72C01083C
:10230000A3260108832C0108A3260108112C01082B
:10231000A3260108232B0108A3260108FB2A010894
:10232000C12A0108A3260108A3260108A326010843
:10233000A3260108A3260108A3260108A326010855
:10234000A3260108A3260108A3260108A326010845
:10235000A3260108A3260108A3260108A326010835
:10236000A3260108A3260108A3260108A326010825
:10237000A3260108A3260108A3260108A326010815
:10238000A3260108A3260108A3260108A326010805
:10239000A3260108A3260108A3260108A3260108F5
:1023A000A3260108A3260108A3260108A3260108E5
:1023B000A3260108A3260108A3260108A3260108D5
:1023C000A3260108A3260108A3260108A3260108C5
:1023D000A3260108A3260108A3260108A3260108B5
:1023E000A3260108A3260108A3260108A3260108A5
:1023F000A3260108A3260108A3260108A326010895
:10240000A3260108A3260108A3260108A326010884
:10241000A3260108A3260108A3260108A326010874
:10242000A3260108A3260108A3260108A326010864
:10243000A3260108A3260108A3260108A326010854
:10244000A3260108A3260108A3260108A326010844
:10245000A3260108A3260108A3260108A326010834
:10246000A3260108A3260108A3260108A326010824
:10247000A3260108972A0108A3260108DF2A0108DC
:10248000A3260108A3260108A3260108A326010804
:10249000A3260108A3260108A3260108A3260108F4
:1024A000A3260108A3260108A3260108A3260108E4
:1024B000A3260108A3260108392A0108E7290108F3
:1024C000B5290108A326010813290108F9280108E4
:1024D0008D280108A3260108732801080728010890
:1024E000DF270108CD27010871270108A32601086D
:1024F00041270108A3260108A32601081727010880
:10250000E9260108D5260108AD260108852601081F
:102510005B2601082F26010817260108A3260108BB
:10252000A3260108A3260108A3260108A326010863
:10253000A3260108A3260108A3260108A326010853
:10254000A3260108A3260108A3260108A326010843
:10255000A3260108F7250108A3260108A3260108E0
:102560009F250108A3260108A3260108A326010828
:10257000A3260108A3260108A3260108A326010813
:1025800085250108C84B1B78DB0700F18A800125EF
:10259000FBF774F9FBF7F6FF2B46FFF721BA5A1C3D
:1025A00032601A780F2A7CD8991C3160C2EBC202C3
:1025B000BE4958788854D81C30600A4499785170C4
:1025C000191D3160D9789170591D31601979D17018
:1025D000991D316059791171D91D31609979517105
:1025E00003F108013160DB799371012519F088FF4F
:1025F0002B46FFF7F5B93046F8F77AF8DFF8BC82DA
:10260000A8F80E003046F8F773F80125A8F80C007A
:102610002B46FFF7E5B93046F8F76AF8A44A00EB15
:1026200080004300012513802B46FFF7D9B91946D6
:102630005A1C32609F4A11F8020B107031605978B1
:102640005170D91C316099789170191D3160DB7817
:10265000D37001252B46FFF7C3B93046F8F748F889
:10266000DFF88482A8F810003046F8F741F8A8F89F
:1026700012003046F8F73CF80125A8F814002B4664
:10268000FFF7AEB91A46591C316012F8020B3260DE
:10269000DA1C597832609A781EF086FF00287FF4A1
:1026A000B8A94FF0FF352B46FFF79AB91A46591CC7
:1026B0003160814912F8020B087032607F495A7804
:1026C0008A70DA1C32607A4A9B78937001252B4617
:1026D000FFF786B97A4B7B4918684E22012529F00D
:1026E0003FFF2B46FFF77CB919465A1C3260764AE9
:1026F00011F8020B1070316059785170D91C31609B
:102700009B7893703046F7F7F3FF704B0125D88024
:102710002B46FFF765B93046F7F7EAFFDFF8AC81E3
:10272000A8F800003046F7F7E3FFA8F802003046AB
:10273000F7F7DEFF0125A8F804002B46FFF750B994
:10274000DFF8A89199F80030002B3FF462A9DFF878
:10275000A08100253046F7F7CBFF1AF013FC99F85B
:102760000030A8EC010A01359D42F3DBFFF751B9B7
:102770000D2A96D15A1C32601D78072D91D8DFF8AA
:10278000749130464FF00C08F7F7B2FF08FB05F8DC
:1027900009EB0805A8803046F7F7AAFFE880304625
:1027A000F7F7A6FF336828811A46591C316012F8E2
:1027B000021BA97232605B78EB723046F7F780FF3C
:1027C000012549F808002B46FFF70AB93046F7F70C
:1027D0008FFF3F4B012518802B46FFF701B95A1C8C
:1027E00032601878060600F1BD862F4B1B78DD0796
:1027F0003FF50FA9032828BF00200125FBF722F889
:102800002B46FFF7EDB85A1C3260304693F800A013
:10281000F7F756FF81463046F7F752FF0546304638
:10282000F7F74EFF80463046F7F762FF3046F7F77E
:102830005FFF3046F7F768FFBAF1000F00F07B86C4
:10284000BAF1100F7FF4E5A8224BC3F800905D6049
:10285000B8F1000F02D0204BC3F800801F49204B75
:102860000222081F01251A701FF0EAFC2B46FFF711
:10287000B7B80D4B1B78D8073FF5CBA80125FBF760
:10288000D7F8FBF77FFE2B46FFF7AAB8064B1B785D
:10289000DA073FF5BEA8134A1378012543F0040375
:1028A00013702B46FFF79CB8644F0020485500205A
:1028B0006C48002078510020D4A60020FC4C002059
:1028C00000920020C00D0408E04D0020C45B0020F1
:1028D00074510020C0240020084E0020C424002091
:1028E0005E5000205CAD0020A4A30020D54E002047
:1028F000185B00205C5C0020B74B1B78D9073FF5C4
:1029000088A8B64B4FF4C87201251A802B46FFF7F2
:1029100067B8092A7FF7C5AEDFF8EC821A46591C62
:10292000D8F80050316012F8021B297032605A78D2
:10293000AA70DA1C32609A78642A03F10401A8BFF5
:1029400064226A713160DA78642A03F10501A8BF54
:102950006422AA7131601A79EA719A1D32605A793B
:10296000642A03F10701A8BF64222A7231609A79B0
:10297000EA7003F108023260DB792B713046F7F719
:10298000B7FE726833686881D11A00290CDD591CC2
:10299000D8F800003160521A002A1978417203DD1C
:1029A0009A1C32605B784370012528F0A3F82B460F
:1029B000FFF716B88A4A1068DA1C01462133951EC3
:1029C000356012F8035C0D70551E356012F8025C1C
:1029D0004D70326012F8015C8D700332934201F148
:1029E0000301ECD1F3E05A1C32601A787D49002AC9
:1029F00000F053850A7842F00202981C0A707A4D62
:102A000030605B782B753046F7F75AFE2860304609
:102A1000F7F756FE68603046F7F76AFE28813046C1
:102A2000F7F766FE714AE8811378012543F0020347
:102A300013702B46FEF7D4BFC2F34705122D3FF6A5
:102A400030AEC5B107F1500307F12A0903EB450A7F
:102A5000C846AAF1260A3046F7F74AFE28F8020FC0
:102A6000C245F8D1624B39F8022F23F8022FC8452E
:102A7000F9D1112D09D85F4A6B00023B13440021A4
:102A8000223223F8021F9A42FBD15B4A01231D46E2
:102A90001370FEF7A5BF1A46591C316012F8025B8D
:102AA0003260DA1C587832609978002D00F0218568
:102AB000012D7EF4AEAF08F0F3F82B46FEF790BF81
:102AC000454A127812F001017FF4EBAD5A1C3260D6
:102AD0001878012508F026F82B46FEF781BFDFF8AD
:102AE0002C8100233046C8F80030F7F7E9FD0125B6
:102AF000C8F800002B46FEF773BF1A46591C316018
:102B00003E4912F8020BC87032603D495A784A714A
:102B1000DA1C32603B4A9B78D37001252B46FEF7C6
:102B20005FBF3046F7F7E4FD3046F7F7E1FD30468A
:102B3000F7F7DEFD3046F7F7E7FD3368284D194615
:102B4000581C2A68306011F8020B82F82C003160A2
:102B5000597882F83610D91C31609B7882F837306A
:102B60003046F7F7D1FD3046F7F7CEFD3046F7F7A0
:102B7000CBFD3046D5F80080F7F7BAFDA8F83A004B
:102B80003046D5F80080F7F7B3FD33687268A8F8CF
:102B90003800D11A01290ADD591C2A6831601B78D6
:102BA00082F82E303046F7F7AFFD33687268D31ADB
:102BB000032B0BDD3046D5F80080F7F799FDA8F818
:102BC000320030462E68F7F793FDB08628681AF079
:102BD00083F8FEF71EBF00BF644F0020F4AD002055
:102BE000009200205CAD002060AD00205C50002011
:102BF000CE4A0020D04A0020F44A0020FC4C00209D
:102C0000BC9100206C480020D4AD00201041002071
:102C10005A1C3260BA4DDFF810831B7888F80530F3
:102C20003046D5F80090F7F763FDA9F8200030464C
:102C3000D5F80090F7F75CFD72683368A9F81E00BC
:102C4000D11A072900F35B84D11A032900F34384C6
:102C5000D21A002A05DD591C2A6831601B7882F8D7
:102C60002630FAF715FE21F069FEA64B28681B688E
:102C7000002B00F01784012519F0D6FC2B46FEF737
:102C8000AFBE1A46591C3160DFF89C8212F8021B55
:102C900088F8021032609C495A780A70DA1C326057
:102CA0009A4D9A782A711A1D3260DB78092BA8BFD9
:102CB00009233046AB70F7F71BFD33687268288034
:102CC000D11A012905DD3046F7F712FD3368726825
:102CD000E8819A4240F05184FAF7DAFD336872686D
:102CE0009A423EF496AE5A1C32601B78EB70012576
:102CF0002B46FEF775BE3046F7F7FAFC05461FF087
:102D0000ADFBFF283EF485AE3F2D00F2A78307F10F
:102D10005009002309F8243D4FEAD508494607F138
:102D20002B0087F82B3008F101081FF077FB97F88C
:102D30002B305FFA88F805F00705434505F10105DA
:102D400003D197F82C30AB4203D0294640461FF000
:102D500071FB33687268D21A012A7EF75AAE5A1C88
:102D600007F15000326000221D7800F8252D1FF079
:102D700049FB97F82B30AB420AD0654B1B683BB13F
:102D80009A79AA4204D31B681B690BB1284698475D
:102D900033685A1C3260484600221D7887F82C2080
:102DA0001FF024FB97F82C30AB423EF432AE584B68
:102DB0001B68002B3EF42DAE1B685B69002B3EF4B4
:102DC00028AE28469847FEF724BE581C3060514A6A
:102DD0001D781570091A00297EF71BAE991C316009
:102DE0005B78003318BF0123012553702B46FEF793
:102DF000F7BD3046F7F77CFCDFF83081C8F80000FB
:102E00003046F7F775FCC8F804003046F7F770FC59
:102E10000125C8F808002B46FEF7E2BD3E49102AFE
:102E200013464FF0000228BF10230A604A608A60F0
:102E3000CA600A74002B3EF4ECAD326801391344C9
:102E40000132326012F8010C01F8010F9A42F7D1F9
:102E5000FEF7DFBDDFF8D8800023C8F80030304629
:102E6000F7F72EFCD8F8003001250343C8F80030EE
:102E70002B46FEF7B5BD5A1C32601D78132D3FF668
:102E800010AC9A1C326058787B6225F0BBF80028A1
:102E90003FF407AC7B6A214A017802F82510D91C5F
:102EA000316002EB850299785170191D3160D87834
:102EB0009070581D306012491B79D3700868012545
:102EC00027F0A6FD2B46FEF78BBD154A03F108013E
:102ED0000133336013F8010C02F8010F8B42F7D174
:102EE000FEF797BD591C1A4631600E4912F8020BC5
:102EF000887032605B784B7001252B46FEF770BD01
:102F000000920020F4470020905A0020A4A3002043
:102F100034920020FC470020384200200048002066
:102F20006FA80020F8AD0020D4A60020243A00208D
:102F3000249400200721B2FBF1F1C1EBC100121A69
:102F40007FF4AFABC9B201F1FF385FFA88F800290E
:102F50003EF45FAD08F1010815465A1C326093F942
:102F600000A050460CF00AF80135814600283FF4D5
:102F700098AB80F802A03046F7F7BAFB3268A9F8A0
:102F800000001346511C316013F8021B89F803102E
:102F90003360537889F80430D31C3360937889F810
:102FA0000630131D3360D27889F80520A845D4D1A6
:102FB000FEF72FBD5A1C32601A780E2A3FF671AB0D
:102FC000991C31605D78032D3FF66BABC748062135
:102FD00001FB02F1421803F1030E5571C6F800E03F
:102FE0009D784554191D3160D9785170591D316053
:102FF00019799170991D31605979D170D91D31605D
:103000009B79137101252B46FEF7EABC5A1C3260EE
:10301000B74A1B78537501252B46FEF7E1BC591CB6
:1030200031601D781F2D3FF63CAB052A7FF439AB8C
:103030003046F7F745FBAF4B43F8250018F0C0FAD0
:10304000FEF7E7BCAB4D05F140083046F7F750FB03
:103050003368A5F88000591C1A46316012F8021B2B
:1030600085F8821032605B7885F883300435A84596
:10307000EBD1FEF7CEBC5A1C32609D4D1B782B72F3
:103080003046F7F735FBA8833046F7F731FB288346
:103090003046F7F72DFB32686883531C3360127893
:1030A000EA747268D31A032B00F38E823368D11A44
:1030B000052900F37982D21A002A7EF7AAAC5A1C9D
:1030C00032601B7885F8213001252B46FEF788BC3D
:1030D0005A1C326093F80080B8F1110F3FF6E1AA54
:1030E0009A1C3260844D5B7805F818303046F7F74B
:1030F000FFFA40F6CA039842A8BF184640F2EE23F2
:10310000984205EB4801B8BF18460125A0F2EE220F
:103110002B46192092FBF0F24A70FEF761BC1A466A
:10312000591C764D316012F8021B297132605B78B0
:103130006B713046F7F7DCFA336828805A1C32602E
:103140001B78AB713046F7F7D3FA336868805A1CA6
:1031500032601B78EB7101252B46FEF741BC684AB3
:103160001278012A3EF655AC18465A1C3260DFF838
:10317000B08110F8022B88F80220DA1C891A30601E
:1031800001295878326040F302823046F7F7B0FAEE
:103190000125A8F800002B46FEF722BC0125F7F711
:1031A000FDFF2B46FEF71CBC5A1C3260554A1B78AB
:1031B000DFF8708113700023C8F800303046F7F74D
:1031C0007FFA3368D8F8002049494F4D10435A1C04
:1031D000C8F8000032601B780B723046F7F788FAA7
:1031E00028603046F7F784FA68603046F7F780FACF
:1031F000A8603046F7F77CFA3046F7F779FAFEF721
:1032000008BC336872689A4240F0E2803F4BFF226C
:103210001A704FF0000A3E4D09F0F2FE514620228E
:103220003C4885F800A02BF01CFC87F82CA097F8F0
:103230002C30072B00F21081DFF8EC90354E52460F
:1032400097F82C3003EB430309EBC3035B7CE3B13A
:1032500097F82C3003EB430309EBC30320215B6990
:103260009BB197F82C3003EB430309EBC303586978
:1032700046F82200F6F7A2FA2B7856F82300F6F764
:10328000EBFB2A780132D2B22A7097F82C30013346
:10329000DBB287F82C3097F82C30072BD0D9236875
:1032A000591C21601A70B8F1000F3EF4B2AB1A4BF2
:1032B000C8F8003001252B46FEF792BB174B3A6A3F
:1032C0009B68D4F800905A449A4200F2B480F7F711
:1032D00003FF5A464946386AF7F77EFF23680344DE
:1032E000236086427EF795AB002120E01C41002040
:1032F00070A80020188E0020AC4D0020E05B00205C
:1033000007940020FC470020243A0020BC22002023
:10331000CFAD002090AD0020FDA003087403002075
:103320000A94002024940020E4A2002023680130A5
:103330005A1CB04222601970F8D1FEF76ABB002D0A
:10334000BCD159462046F7F72DFA23685A1C226053
:103350001D70AD4B26689D683B6A0BEB03029542DE
:1033600080F0AB803B6AED1AF7F7B6FE2A4631468D
:10337000386AF7F731FF236803442360FEF749BB3F
:103380003046F7F7B5F9326871687B6A9142834637
:1033900047D106461D46FEF726BE3046F7F7A8F988
:1033A000DFF89C82FEF7F2BE9A1C3260974A597889
:1033B0001170D91C316099785170191D3160DB781A
:1033C0009370FEF726BB924B93E84200FEF75CBD7C
:1033D0005A1C194632608F4811F8022B0270316076
:1033E0005B784370042A03D9FF2A7EF4BEAA10E753
:1033F00089490978994205D8022A7EF4B6AAFF2B9A
:103400007EF4B3AA236801255A1922601D70B8F111
:10341000000F3EF4FEAA814BC8F800302B46FEF7A1
:10342000DFBA511C316012781D46131C064618BFC6
:103430000123FEF7D8BD3A6AA3EB0208F7F74CFE6A
:1034400042464946386AF7F7C7FE236803442360BB
:10345000002D3EF4DEAA44E7524620E707F12C098E
:1034600048461EF0B7FFBB8DAB423FF472AC6C4BCD
:103470001B68002B3FF46DAC1B689B69002B3FF46D
:1034800068AC2846984764E4DA46C7F824B0FEF7EB
:1034900041BE7D62AA46FEF73DBE0A7802F0FD02FB
:1034A000FFF7ABBA5F486049604A614B0360012592
:1034B0000B6013602B46FEF793BAF7F70DFE5A46E2
:1034C0003146386AF7F788FE2368012503442360F4
:1034D0002B46FEF785BA3046F7F70AF9A8F80E0032
:1034E0003046F7F705F933687268A8F81000FFF75F
:1034F000AFBB012519F060FA2B46FEF771BA3046D2
:10350000F7F7F6F8A8F80A003046F7F7F1F8A8F848
:103510000C003046D5F80090F7F7EAF8A9F8220039
:103520003046D5F80090F7F7E3F833687268A9F8E9
:103530002400FFF789BB364B1020C3F800905D6074
:103540000BF0ACFF3B4A137843F001031370B8F162
:10355000000F3EF45EAA384B0125C3F800802B46CD
:10356000FEF73EBA00F07F00032828BF00200125A7
:1035700007F0B2FB2B46FEF733BA5A1C32601B78B9
:10358000003318BF012388F80730FFF7A5BB2B4A8B
:1035900099781288012512FB00F22B4692FBF1F27A
:1035A000A8F80020FEF71CBA5A1C32601B78EB7298
:1035B0003046F7F785F83368E8605A1C32601B78AC
:1035C0002B743368726876E53046F7F791F8A88473
:1035D0003046F7F78DF833687268E884D11A03290A
:1035E0007FF765AD1A46591C316012F8021BA977A6
:1035F00032605B7885F820303046F7F779F8336829
:103600007268688453E500BF74030020D9920020DB
:10361000A0500020BC220020D54E002021C600086A
:1036200034920020385600208C5600208C5A0020FE
:10363000C18500085CAD0020084E002072460020C5
:103640007C4E00202DE9F047C44B1C6862072DED2D
:10365000028B03D4BDEC028BBDE8F087C04D2B7804
:10366000002BF7D06E6846F2A713861B9E42F1D955
:10367000DFF850936860B9F80070DFF84C83002FD2
:1036800040F0A68198F80620AB689FEDB60ADFED02
:10369000B60ADFF8F492013AB3FBF2F307EE903A80
:1036A000F8EE677AB7EE008A27EE800A29F03CFA36
:1036B000DFEDAE7A38EE400A20EE270A29F0C4F892
:1036C000B8F80830DFEDAA6A07EE103AEB68C01AC6
:1036D000B8EEC77A07EE900AA7EE668AB8EEE70A58
:1036E000D9ED097AF8EEE77A20EE080A67EEA67AB5
:1036F000A7EE270A29F0A8F89E4BC9F82400024635
:103700001860A30740F1AA81DFF8C0E29A4CDEED11
:10371000007A9FED9A5A2168F8EE677A27EE855A6B
:10372000002900F0BB81964B07EE101AD3ED026A18
:10373000B8EEC77AF8EEE66A86EE878A914991ED8F
:10374000004AB8F80C10D5ED054ADFED895A95ED21
:10375000066A67EE847A06EE901A67EE887A8A49DE
:10376000B6EE004AF8EEE66AF0EE643AE7EE843A26
:1037700066EEA56A91ED097A7E49F7EE005A75EE7C
:10378000E65AB8EEC77AA3EE856A77EEA47A27EEFA
:10379000257AC5ED057AF0EE477AE6EE267ABDEE9B
:1037A000E77AC5ED067A81ED007A78490978122921
:1037B00000F05B8100211960596099602160CEF8AA
:1037C0000010002F7FF446AFE869EA61121A07EE95
:1037D000102ADFED6F6A6F4B07EE906AB8EEC77A7A
:1037E000F8EE677A27EE267A40F2DC52C7EE276AB7
:1037F0000A21FDEEE67A17EE900A9042A8BF104625
:103800009842B8BF1846F7F747F9B8F80A309FED65
:10381000586AD5ED056A07EE103AB8EEC77AF7EEAA
:10382000007AE7EE467A05EE900AF8EEE55A66EE83
:10383000866A67EEA57AE7EE267AB0EE670AC5EDEE
:10384000057A29F001F805210646F7F725F9524ACD
:103850005249B2F90040086084EAE473A3EBE473D0
:10386000B3F5487F74DAB2F9022082EAE273A3EB7F
:10387000E273B3F5487F6BDA494B1B78002B40F0BD
:103880001181484B3B4A1B68126847489B1AB3F5A5
:10389000FA7FA8BF4FF4FA739842B8BF18460A21BE
:1038A000F7F7FAF8414B1C68637A00FB03F0002835
:1038B000B8BF7F30C211B2F5967F3D4BA8BF4FF421
:1038C00096729A42B8BF1A463A48E37E076895ED69
:1038D000087ADFED396A911B01FB03F3227F344E36
:1038E000002B01FB0272B8BF1F335B11B2F5C81F7A
:1038F0003249A8BF4FF4C812B3F5967FA8BF4FF462
:1039000096738A42B8BF0A46617F026007EE901A3A
:1039100037EE087AF8EEE77A27EE267AB34267EEBA
:10392000877AB8BF3346002AB8BF02F5FF52FDEED2
:10393000E77AB8BF1F3203EB623317EE902A962A5C
:103940006FF09501A8BF96228A42ACBF9F1A5F1AFA
:103950001B4A85ED088A17607CE600BF58AD002041
:10396000C022002008942537B1DC423ED048874A67
:103970006F12833A38AD002024540020BD378635BD
:1039800014540020DC5B0020C0420020F44E0020D4
:103990000024744924FAFFFF3CAD00202CAD002028
:1039A000104E0020084E00200CFEFFFF0092002069
:1039B000D4FEFFFF004E00200000003B0000E7FFA8
:1039C000F84D0020F2AD0020BC91002020540020D2
:1039D000374998F806A00A68AB689FED360ADFED14
:1039E000360A002A0AF1FF3AB3FBFAF39246B8BF4F
:1039F00002F1070AA2EBEA0203EB020ABAF1000F96
:103A00005346B8BF0AF10703DB1007EE903AF8EE11
:103A1000E77AC1F800A027EE800A29F085F8F7EED2
:103A2000007A77EEC07A9FED257A2B6967EE877A68
:103A30009A4518BF07F1FF33FDEEE77A14BF9FB236
:103A400000274FF00003C5ED037A18BFC5F810A09A
:103A5000A9F800706B61AB61002252E69FED188AF5
:103A6000DFF870E0174C184B9FE695ED057AD5ED21
:103A7000067ADFF864C02068996891FBF0F1BDEE2A
:103A8000C77AFDEEE77A17EE100A17EE909AACF8B7
:103A90000200ACF80010ACF804908BE69FED088AA9
:103AA000094B4BE6094A0A4B12681C680CE700BF39
:103AB000A000002008942537B1DC423ED048874A58
:103AC0000000000024540020145400200C4E00205C
:103AD0000092002020540020F84E00202DE9F843E9
:103AE000304B1B685B0701D4BDE8F8832E4C2F4D8B
:103AF00094F82490B9F1010F48D1EB692846984712
:103B00002B69284698472B6A04F12C0004F1280100
:103B10009847274B276B9B79A668E06A07F1010855
:103B20009845636B08BF84F8009003F1010208BF59
:103B30004FF00008032A1FD01E49626394F8382012
:103B400041F82300FAB904EB870704EB8803F86314
:103B5000DA6BAB89C4F83080B61A30440022A0601A
:103B600084F82420002BBFD0134A0A2B1268B8BF58
:103B70000A231361BDE8F8830E4B012298600023ED
:103B800084F8382063631AF0F5F9DCE76B6928469E
:103B90009847AB69284698470122EB8984F824208E
:103BA000E0E700BF58AD0020C0220020C042002046
:103BB000BC910020546D0020D0910020F8B5534BEB
:103BC0001B681C0700D4F8BD514C524F524D7B6806
:103BD000064604F1FC009847B4F9FC00B4F9FE2055
:103BE000B4F90031397D286028466A60AB6012F074
:103BF00027F84A4A137859073ED4D4F80401484BB1
:103C00001B7883B1474B2968B3F906C0B3F908E0C4
:103C1000B3F90A706A68AB68A1EB0C01A2EB0E0263
:103C2000DB1B85E80E000028CDD03F4B301A9842B0
:103C30003FD9B4F91451B4F91011B4F90871B4F9B9
:103C40000A21B4F91261B4F90C31364839443244CE
:103C50002B4401EBD17102EBD27203EBD3735B10F7
:103C6000491052100025C18002814381C4F80451DB
:103C7000BDE8F840FAF72EBE2C4FB5F90000B5F9B3
:103C80000410A4F8080123F0040313700022B5F90E
:103C90000830A4F81001C4F804613A60BA80A4F8AE
:103CA0000A11A4F81211A4F80C31A4F8143130460A
:103CB000A5E70020F5F75EFA2B68B4F908219342D6
:103CC000B4F91021B8BFA4F808319342C8BFA4F8D2
:103CD0001031B4F90A216B689342B4F91221B8BFCC
:103CE000A4F80A319342C8BFA4F81231B4F90C21E8
:103CF000AB689A42B4F91421C8BFA4F80C319A42B7
:103D0000BFF661AFA4F81431F8BD00BF58AD002074
:103D1000C022002054480020DC9100205CAD00202F
:103D2000784800206C4800207FC3C90172480020F9
:103D30002DE9F04F724B734A1C7893B000F59C410B
:103D40002031814606911160002C00F027856E4AD3
:103D50001268904240F227826C4A6D491768DFF87A
:103D6000E8B10492013C1C706A4C039107F480573F
:103D7000002F40F02582039B5B7D002B40F09B844D
:103D8000049B1B681D0400F17B87634B9945A37856
:103D900000F27383002B40F07383604B0693049B07
:103DA0001F6817F4805940F0FA83039BBBF9066043
:103DB0005B8B9E42B4BF00260126594B1B6813F053
:103DC000805300F00782069A127812F0010200F088
:103DD000088203985349408C91ED037A07EE900ACC
:103DE000F8EEE77AB4EEE77AF1EE10FA81F20F809E
:103DF000002E40F0FD814C4D95F8B811002940F09F
:103E0000F7814A484A49056895F82D500020086016
:103E1000486088604749002D40F0EB810D70002A12
:103E200040F0EC81444B1A78002A50D10399BBF939
:103E300000E04F8B898BBBF90200BE45CCBF8025CB
:103E4000002545F040038E45A8BF2B469B0843F054
:103E50008005B842C8BF2B4643F040058842A8BF42
:103E60001D46BBF904E0BBF90600AD0845F0800330
:103E7000BE45C8BF1D4645F040038E45A8BF2B4632
:103E80009B0843F0800E284DB842C8BF734643F0EC
:103E9000400E95F8BA718842B8BF73469F4201F050
:103EA0004481A5F8BC2185F8BE21244985F8BA31A2
:103EB0000F78002F01F0B5805F2B01F01C816F2B74
:103EC00000F0FD87069B1B78D90740F1BF87049B54
:103ED0001B4A1B68059203F00403002B40F04A853F
:103EE0000DF14008174D0023C8F8043005F15009C2
:103EF000109340F6330A192740F2833629E000BFB9
:103F0000104D0020CC4A00200C4D0020F8A60020C7
:103F100070A80020548F0020404B4C00644F0020BC
:103F200060460020F04F0020C022002000920020B8
:103F3000A84200204426002029A90020F41D0020CA
:103F400058AD002000480020AC79002004354D45D4
:103F500020D0AA78EB789A4217FB0261F6D26A78F1
:103F6000043217FB03633BF912205245A8BF5246A7
:103F7000B2F5617FB8BF4FF461729142E6DA9A42BE
:103F8000E4DC29782429E1D840460435F6F750FFCF
:103F90004D45DED1B04B98E803001F78AF4B83E866
:103FA0000300002F00F03C840121AC48F6F750FFDD
:103FB000002840F09A81E378002B40F09681A84CCD
:103FC00023881DB225F00105AEB2B342268000F071
:103FD000B686A44D02270E204FF014094FF0FF08BB
:103FE0002F7085F8019085F802800BF027F939468B
:103FF0009A482688F6F72CFF002841F0498026F0E1
:1040000002039BB2B34223800AD0964B1421FF22B5
:1040100002250E201D7059709A700BF00FF926883A
:10402000DFF884A2904B9AF8001058680393B50704
:1040300008BF81F00201C1F34001F5F713FD24210F
:104040008648F6F705FF30B9069A1378590744BF3A
:1040500023F004031370059B1B6813F00A0F1DD097
:1040600005217E48F6F7F4FE002800F09D8625889D
:104070006F0740F1B98779480621F6F7E9FE002875
:1040800000F07F866E0640F18C8707217348F6F7B3
:10409000DFFE002840F03083059B1B68980600F186
:1040A0003B8326886D480C21F6F7D2FE002800F0ED
:1040B000388146F48073B342238009D0694B0225CE
:1040C0001421FF220E201D7059709A700BF0B6F863
:1040D000664B1B78082B00F030810E2B00F02D81F1
:1040E000049B1B685E0544D5614B1B79002B00F0D7
:1040F000E18014215948F6F7ABFE002840F0DF803C
:104100001CF0F0FE01200AF075FF90B3DFF89C81EF
:1041100000254FF0CC0902E0DDB2022D29D809FBC1
:1041200005F76B1C58F80760002EF5D1C378514A8B
:1041300090F9020052F823300196032200920121E7
:10414000324609F0BFFE034605EB450000EB0010C8
:10415000049353B1314608EB8000CC222AF081FC55
:10416000049B48F807300135EDB21BF063FF0028CF
:10417000D3D1069B1B78DD0740F1F2803E493F4AD0
:1041800001230B701370039B9AF80010186801F05C
:104190000101F5F767FC059B1B685A0700F1508188
:1041A00013B0BDE8F08F364B364A1F68049307F40E
:1041B00080570392DFF8F8B0334C002F3FF4DBADAB
:1041C00000212648F6F744FE00287FF4D4AD09F01C
:1041D000B1F8D0E578023FF5F6AD069A127802F014
:1041E00001022A4D002185F8B811002E3FF409AED6
:1041F000274901200870002A3FF414AEF9067FF524
:1042000011AE244A1278D2063FF50CAEB9F1000F78
:104210007FF408AE002B7FF405AE7B023FF502AEC3
:104220001D4B1B78002B01F025841C4B9B78002E26
:1042300041F05D843BB11A4A1A4B12681B689B1A05
:10424000002BC1F28F841020104D0AF0F7FF0123DC
:1042500085F8B931E6E500BF6853002060460020CC
:104260004A8F00204C420020B8B70020FC470020B5
:10427000E04F0020E8190408654F00201C4E002084
:10428000F8A6002070A80020548F0020C022002033
:10429000442600205CAD0020F41D0020F8AD002075
:1042A0000CAE0020A83A0020B4B70020EC75002026
:1042B000AC790020069B1B78D8077FF521AF3C2006
:1042C0001AF0AEF800283FF454AF06F08BFF3C2004
:1042D0001AF03CF800283FF44CAF06F083FF3C2076
:1042E0001AF034F80028F0D143E7059B1B689A07C1
:1042F0007FF565AEBF4C2688F3073FF580AE46F0EC
:1043000001039E4223803FF47AAEBB4B1421FF226F
:1043100002250E201D7059709A700AF08FFF2688B2
:104320006DE626F480739BB2B34223807FF4C6AE61
:10433000B24B1B78082B7FF4D0AE228822F04003CA
:104340009BB29A4223803FF4CBAEAB4B02251421A3
:10435000FF220E201D7059709A700AF06FFFBFE6A1
:10436000A74B93F80090B9F1000F5FD1DFF8E4821A
:10437000A44F18F8030C3E794146A8F1030526F036
:1043800017FB002800F0F283002E40F0448405F172
:104390000801687926F00CFB002841F0ED819A496C
:1043A000A87A26F005FB002800F0F383022E41F0E6
:1043B000E7819649E87B26F0FBFA002841F0E4818A
:1043C0009349287D26F0F4FA002800F0F383042EA8
:1043D00041F0DE818F49687E26F0EAFA002841F03C
:1043E000DB818D49A87F26F0E3FA002800F0F383F3
:1043F000062E41F0BD81894995F8230026F0D8FAB0
:10440000002840F05C87864995F8280026F0D0FA0D
:10441000002800F0F383082E40F03B87814995F88F
:104420002D0026F0C5FA002840F0F3837E4B0122D0
:104430001A7026F040FD059B1B685A077FF5B0AE49
:10444000032026F0DFFA002800F06A86238813F0A4
:1044500008047FF4A5AE08200BF038F87348744DBB
:104460007449754A754BBBF8066000682E80086079
:1044700014601C6013B0BDE8F08F0BB90123A3706A
:104480006F4B06931B201F7894F8216026F0BAFA30
:10449000012E07F00109824600F0298607F0020389
:1044A000059394F82030DFF8B081664D052B69D86C
:1044B000DFE813F05B004F000600DC00FF008D001A
:1044C000012E04BF052384F82030B9F1000F00F05D
:1044D0005281039B5C4FB3F91810B8F800300022EA
:1044E00061F30F0263F31F42002361F30F0361F3D3
:1044F0001F43CBF8042039686269CBF800308A4248
:10450000C0F06C84012E41F00283032294F8203025
:104510000592CBE726F0A2FA012807D14A4FB8F856
:1045200002303A68642101FB03232361BAF1000FD2
:1045300004D098F80630002B40F09080012E21D056
:10454000414F22693B689A42C0F03586012384F8C6
:104550002030012E3BD098F80730012B00F0148159
:1045600019F038FA94F82030A0E7B9F1000FD1D152
:104570004FF48060BAF1000F00F0FF830AF0A6FF4D
:1045800000232361059B002B3FF409AC05980AF03A
:1045900055FE049B1F6817F480593FF406AC1D219B
:1045A0002A48F6F755FC00287FF4FFAB284A039B06
:1045B000D2881B8BBBF90660991A8E4240F30586A0
:1045C00013449E42B4BF00260126FFF7F6BB1E4FE0
:1045D0003A68B8F80230642101FB03234FF480608D
:1045E0000022236184F82020E2700AF057FF94F83B
:1045F00020305BE74A8F00204C420020FC4700201F
:10460000654F0020A000002010420020154200202D
:104610001A4200201F42002024420020294200208C
:104620002E420020334200201C4E002038AD0020D6
:10463000FC4D0020084E0020004E0020F84D0020C8
:10464000644F0020788F00200CAE002060460020D0
:10465000C45B002006420020E05B002019F0BAF99C
:1046600003224FF47A7384F82020E361A74F2B884C
:1046700043F002032B8008F05DFE3A68E3691344BF
:104680000422A36184F82020012E40F0A1853B681C
:10469000A2699A42BFF476AF9D4B187820B926F0F4
:1046A000B1F900287FF46EAF2B8823F002032B8032
:1046B0008EE7964FE8E7039A013BD27D3BF9133032
:1046C000002A40F08683A3F57A73B3F57A7FA8BFFA
:1046D0004FF47A7323EAE37307EE903A9FED8D7AF5
:1046E000F8EEE77A67EE877A8B4AFCEEE77A17EE08
:1046F000903A1380FFF749BB884B894AB3F90430DD
:10470000884982FB0302DB17C3EBA202059B0A80E8
:104710001B6898067FF5C5AC834B1B78990704D5B9
:10472000824F3B7D042B00F25985268816F0300F0E
:104730003FF4B8AC10200AF0B1FE20200AF0AEFE23
:104740007B4B268800221A707A4A7B487B4F7C4D2F
:10475000002111607B4A396000232960416081613A
:10476000036083604361C361136051609360536170
:104770009161D36196E4654F3B6847F23052032361
:10478000E26184F8203072E719F024F9032240F640
:10479000B83384F82020E3615C4F68E76A4F3B78C8
:1047A000002B00F09C87694BDFF8B481DFF8B4B1CF
:1047B000DFF8B4A1039345465E46049099460EE0A7
:1047C00019F804109847032C28DC88B93B782AF89C
:1047D000020F01349C4205F1040580F2EF80072CA2
:1047E000E1B23046DBF80430EADD984700B2EDE78D
:1047F00038F824206B88801A4FF47A719B1A01FBD9
:1048000000F040F6CA0290FBF3F00844904240F2F8
:10481000EE23A8BF10469842B8BF184600B2D5E7AD
:10482000DFF848A1DFF84881494D0AF15A064FF0F8
:10483000010951461AF8010C26F0BAF8F8B19AF8B5
:1048400004009AF802309AF803E000EB400105EB0F
:104850008101013BD1F8CC2103EB43034344934254
:104860000DD095F8F82181F8C8E109FA00F022EAA4
:104870000000C1F8CC31C1F8D07185F8F8010AF117
:10488000060A5645D5D13349204A334B334D096882
:104890001B78D2F8009008910793A5F5E47A0026DA
:1048A0006B685BB31F784FB3AA68A9EB0202002ABA
:1048B0000ADB9AF8F8210121B14022EA010209F548
:1048C000FA718AF8F821A960079ABAB12A7859785A
:1048D0000432D2B2002940F0A08203993BF91220A1
:1048E000098B01F1C800824240F337849AF8F8112D
:1048F0009A7841FA06F3D80740F1C6840136042EAF
:1049000005F10C05CCD1FFF74FBB00BF0CAE00206A
:10491000F41D0020AAF1823F488F00203CAD00200A
:1049200067666666F04D00205CAD002060AD00203B
:104930005E50002054510020045100201826002011
:10494000784E00202C510020644D002070A80020DB
:10495000C0220020D4AD0020158F00208824002024
:10496000784D002028920020D62300201D410020F1
:1049700070F10308A94D95F8C23153B1069B1B781D
:10498000DE0706D5039BBBF906205B8B9A4200F33A
:1049900051841121A248F6F75BFA002800F0258225
:1049A00095F8C6312BB995F8C03113B93223A5F863
:1049B000C431012385F8C631FFF792BADDF81090B3
:1049C000984A04921146984A0968A2FB092A42F2C1
:1049D00001020A404FEA9A1A059200F00282934DB2
:1049E0009348944C944A95F800E0007884F800E0ED
:1049F0001070BEF1000F04D08F4A92F800E08EF0E4
:104A0000010E864D0F2085F83C01002B00F0168327
:104A10008A4B039E0B931B78B6F826C00A931C465C
:104A20003B78B78C039E864A368B0E962646A2FBB1
:104A30000442520802EB4202B21AD2B2CDF820C0B0
:104A400001F48051079295F83D81DFF810B2DFF84C
:104A50002CC209900AF5967276460F9105F5A0745E
:104A60000020CDF830900D959646002E00F03C8247
:104A7000744A32F910201FFA82F9B9454FEA400111
:104A800003D3089DA94540F273825CF8202092452B
:104A900080F033823BF90120059D002D40F04782D4
:104AA000013098422BF8012004F10604DDDB09985F
:104AB0000D9D654ADDF8309085F83D810F280CBFCB
:104AC0000121002185F83C01117000F0BE825F4C8D
:104AD0005F4E604F35883868A1686268E06045F0D5
:104AE0000405401A9042524F3580534D4FF001015A
:104AF00088BF00223970297088BF84F82120002BDC
:104B000000F0B582049A03991768534EB1F824C097
:104B1000B1F818E0514817F48057354640F0C98283
:104B200039460EE06A7802EB820202EB820202F260
:104B3000EE2292B201318B4220F8022B05F10205E0
:104B40000ED016F81120002A00F01582022AE9D0B2
:104B50000131028820F8022B8B4205F10205F0D1C9
:104B60000B9A137801331370FFF702B908F10501AE
:104B7000687925F01DFF00283FF411AC012E40F0AC
:104B8000FB8505F10D01A87A25F012FF002840F001
:104B9000F7853349E87B25F00BFF00283FF410AC84
:104BA000032E40F0F1852F49287D25F001FF0028D4
:104BB00040F0EE852C49687E25F0FAFE00283FF48F
:104BC00010AC052E40F0E8852849A87F25F0F0FEBE
:104BD000002840F0CD85264995F8230025F0E8FE11
:104BE00000283FF410AC072E40F06983214995F866
:104BF000280025F0DDFE002840F04B831E4995F883
:104C00002D0025F0D5FE00283FF410AC092E3FF40E
:104C10000DAC4FF009094B463EE300BFC022002017
:104C200060460020F8A60020D34D6210A84A00205C
:104C300050010020158F002051010020114D00204F
:104C4000ABAAAAAAD82300209E530020548F00208C
:104C5000788F00200CAE0020AC4D0020AC790020F5
:104C6000154200201A4200201F420020244200204A
:104C7000294200202E42002033420020144D002003
:104C8000CC4DD5F8A031A9EB0303002BFFF67DA88E
:104C9000C94A95F8A431517C069AC5F8A021013380
:104CA000C64A039E32F81120B17D03F00F0385F848
:104CB000A4312B4492B292FBF1F283F8A82195F82B
:104CC000A81195F8A92195F8AA3195F8B4010A44DC
:104CD00095F8AB11134495F8AC21194495F8AD3112
:104CE0000A4495F8AE11134495F8AF21194495F88C
:104CF000B0310A4495F8B111134495F8B221194422
:104D000095F8B3310A44134495F8B51195F8B721D5
:104D1000184495F8B63101440B441A4442F30B127F
:104D2000642AF17DA8BF642213B209B1C2F1640301
:104D300007EE903A9FEDA27AF8EEE77AD2E40221EC
:104D4000A048F6F785F800283FF459A92580B70751
:104D50003FF566A946F00203B34223803FF460A901
:104D6000994B02201421FF2218700E2059709A705E
:104D70000AF064FA2688FFF753B90AF08FFBFFF7B1
:104D8000FFBB25F040039BB2AB4223803FF47DA9DB
:104D90008D4B02251421FF220E201D7059709A7030
:104DA0000AF04CFAFFF771B9238823F00405ADB27D
:104DB000AB4225803FF45FA9834B02251421FF22DB
:104DC0000E201D7059709A700AF038FA2588FFF786
:104DD00052B9C3F53B6308331BB274E40323059354
:104DE000CBE47A4A92F800E003E695F8C031002B54
:104DF0003FF476A8069B1B7813F001037FF470A89C
:104E0000012285F8C03185F8C121FFF769B8694DE5
:104E1000012185F8B811FFF7EBB9012900F00184F1
:104E20009AF8F8210123B34001361343042E8AF87F
:104E3000F83105F10C057FF433ADFFF7B5B8069BEB
:104E4000634A1B781060DF0700F1028295F8BE11FB
:104E500000297FF43CA8B5F9BC31322B7FF737A885
:104E600095F8BA210120572A85F8BE0100F09884F0
:104E7000049B1B6813F0040302D05A2A00F0E78554
:104E80005D2A00F0E5845B2A00F025855E2A00F0AB
:104E90006C85562A00F0CC85972A00F08785A72AD2
:104EA00040F09D844B49049B0A781B6842F0040241
:104EB0000A70494A059203F00403FFF70EB8B2F5F1
:104EC000FA7FFFF604A895F8BE21002A7EF4FFAF12
:104ED000069B1B780121D80785F8BE1100F1C38419
:104EE00007F08EFBFEF7F3BF002F3FD05CF82020C9
:104EF00092454FEA4001FFF4CDAD384A374D525C40
:104F000005EB0109002A00F0B780022A46D199F882
:104F1000012002EB820202EB820202F2EE2292B246
:104F2000032832DD059D12B2002D3FF4B9AD079D77
:104F300024F81520B8F1000F03D10A9D022D7FF649
:104F4000AFAD2288B4F80290B4F804804A4490448B
:104F5000234A0FFA88F882FB0852224DA2EBE8722E
:104F600025F8018012B24FF0010899E53A46410058
:104F70004CF820E090E5CAB2022A04D9032A7FF453
:104F8000E7AD6246D6E57246D4E5012505FA00F99B
:104F9000099D25EA090512B209957DE53BF8012036
:104FA000BEE745F04003AB4223807FF4F1AEFFF74C
:104FB0006CB800BFC0220020D07A0020EC7A00201C
:104FC00014AE2341604600204C420020158F002083
:104FD000AC3A00205CAD002058AD0020AC4D002064
:104FE000565555554824002045F004039D42238022
:104FF0000AD0B54B02251421FF220E201D705970D6
:105000009A700AF01BF92588B04BB14AB3F9043005
:10501000B04982FB0302DB17C3EBA2030B80FFF74F
:105020002AB83946AC48F5F713FF00283FF407AF1C
:1050300085F8BF7107F0E4FAFEF744BFA749A84A14
:105040000B91DFF8C0B2012111701B21A24805931A
:10505000F5F7FEFE059B00287FF439ADA14CA24F69
:10506000E2683B68A3609B1AC82B00F25A83049B3A
:105070001F6807F4805773E5C2B2022A40F2CF825C
:10508000032A8BD10E9A0F9D002D08BF3A4647E7A1
:1050900026F001039BB2B34223803FF458AE0E20AA
:1050A0002F7085F8019085F802800AF0C7F82688ED
:1050B0004DE600210FE06A7802EB820202EB8202E9
:1050C00002F2EE2292B20131994220F8022B05F150
:1050D00002053FF445AD16F811201AB1022AEAD0B4
:1050E0000288F0E7CAB2032AFAD87246EBE7002337
:1050F0000593FFF7D6B9B2F5FA7FFEF6E8AE95F85C
:10510000BE31002B7EF4E3AE069B1B7801210B40E1
:1051100085F8BE1100F0E78208F00CF9FEF7D7BE63
:1051200008200AF0BBF9FFF73BB8704A70491068D5
:10513000B5F9BC21C76981FB07018911FF17781AEE
:1051400000F5FF407F3082423EF7AFAEC91B0A44F4
:1051500012B2A5F8BC21FEF7A8BEC8398A425CDAB3
:105160009AF8F8119A7841FA06F3D9073FF5C6ABD9
:105170005242012009920AF079F97B1E099A162BF6
:1051800000F24281DFE813F0E301F901CA012202D3
:105190000F0236029D01880171015A01430140014D
:1051A0002202300136029D0188011A010401EE003D
:1051B000B201D600C00018F00DFC032240F6B8334F
:1051C00084F82020E361FFF752BA0126FEF7F5BD0F
:1051D0003A68E3691344A361FFF7D4B90A2025F0C4
:1051E00011FC26888046002800F05882F20640F123
:1051F0004483404D95F80882B8F1000F7EF452AF19
:105200000D200AF01BF8012385F808322688B8F132
:10521000000F7FF499AAFEF745BF9AF8F8310122F2
:10522000B24023EA020309F5FA728AF8F831AA605B
:10523000FFF764BB00212848F5F70AFE00287FF439
:10524000A8AB322385F8C201A5F8C431FFF7A1BB92
:10525000294B1B78002B3EF43AAEE378002B7EF40A
:1052600036AE95F8BF310133DBB2032B85F8BF3181
:105270007EF62DAE214B5B7813B9002E7EF427AE5F
:1052800008F058F8FEF71EBE002A0CBF01200220CD
:1052900070E74FF008094B4603EB83031D4487F882
:1052A0000490A97868781DF0C5F8069B144A1B780D
:1052B00001211170D9077FF5BCA8FEF764BF4FF03C
:1052C00007094B46E8E700BF4C4200203CAD0020F8
:1052D000676666667451002060460020114D00200C
:1052E0009E530020548F00200CAE0020D09100204F
:1052F000D34D6210C0220020158F0020F8AD002091
:105300001C4E0020AC790020DAF8FC01DFF81C8785
:1053100090F8361098F8023011446429A8BF64212F
:1053200021EAE17180F83610002B40F04B8417F031
:10533000D3FC75E5DAF8FC01DFF8F08690F8371059
:1053400098F802301144FE29A8BFFE2121EAE1713C
:1053500080F83710002BEAD0162025F0B1FBDAF8E0
:10536000FC01E4E7DAF8FC01DFF8C086817811443B
:10537000C829A8BFC82121EAE171817098F80230DC
:10538000002BD4D0142025F09BFBDAF8FC01CEE7EB
:10539000DAF8FC01DFF8948641781144C829A8BFE7
:1053A000C82121EAE171417098F80230002BBED08B
:1053B000132025F085FBDAF8FC01B8E7DAF8FC01E8
:1053C000DFF8688601781144C829A8BFC82121EAFE
:1053D000E171017098F80230002BA8D0122025F05E
:1053E0006FFBDAF8FC01A2E7DFF84086089898F82E
:1053F0000230417911446429A8BF642121EAE17196
:105400004171002B40F09383DAF8FC018FE7DAF862
:10541000FC01DFF81886017A98F802301144C82997
:10542000A8BFC82121EAE1710172002B3FF47FAFD0
:105430000B2025F045FBDAF8FC0178E7DAF8FC01EF
:10544000DFF8E885C17998F802301144C829A8BF6F
:10545000C82121EAE171C171002B3FF468AF0A2035
:1054600025F02EFBDAF8FC0161E7DAF8FC01DFF841
:10547000BC85817998F802301144C829A8BFC82199
:1054800021EAE1718171002B3FF451AF092025F031
:1054900017FBDAF8FC014AE7DAF8FC01DFF88C8543
:1054A000417998F802301144C829A8BFC82121EADF
:1054B000E1714171002B40F04183112F7FF456AF11
:1054C00035E7DAF8FC01DFF86485017998F80230F5
:1054D0001144C829A8BFC82121EAE1710171002B3C
:1054E00040F07483102F7FF457AF20E70898DFF85F
:1054F0003C8541781144B1F5967FA8BF4FF4967171
:1055000021EAE171417098F80230002B3FF47CAF42
:10551000152025F0D5FADAF8FC0108E70899DFF83C
:105520000C850F791744642FA8BF642727EAE77713
:105530000F7125F0DFFA98F80230002B3FF464AFCA
:105540000320394625F0BCFADAF8FC01EFE60898AA
:10555000DFF8D88401781144FA29A8BFFA2121EA9A
:10556000E171017098F80230002B3FF44DAF01203B
:1055700025F0A6FADAF8FC01D9E60898DFF8AC8441
:10558000817811446429A8BF642121EAE171817006
:1055900098F80230002B3FF437AF022025F090FA44
:1055A000DAF8FC01C3E60898DFF88084C17998F83E
:1055B0000230114481F30801C171002B3FF424AF84
:1055C000052025F07DFADAF8FC01B0E6089BDFF84B
:1055D0005C84997998F8020011446429A8BF642179
:1055E00021EAE1719971002840F0B0820D2F7FF41B
:1055F000FDAE09E7DAF8FC01DFF83084C17898F8ED
:1056000002301144C829A8BFC82121EAE171C17044
:10561000002B40F084820F2F7FF4D4AE87E60E9AE1
:105620007EE43BF912209978B2F5617F4FF49663DE
:1056300093FBF1F34ADB40F633019142A8BF1146D8
:105640000C2FA1F5617191FBF3F100F08481182F0B
:105650007FF4E6ABC9B2C8290B46A8BFC823DAF865
:10566000FC01C27DDFB297423FF4DAAB9A1ADFF851
:10567000BC83C77548BF0732D71098F8023001378E
:10568000FFB23BB9002F3FF4CBAB384609F0EEFE3A
:10569000FFF7C6BB182025F013FAF3E7F30600F175
:1056A00050810B2025F0AEF9002840F01881B70694
:1056B00000F15381C34D95F80832002B3FF4A0ADA3
:1056C000B8F1000F7FF440A8FEF7ECBC0C2F00F0FF
:1056D000EA80182F7FF4A4AB00210B46BFE7BA4A3B
:1056E0000392FFF76DB9B949096811F4003140F030
:1056F00040810B46B648C65C0F2E03F10C031ED04A
:1057000001311529F7D1049BB2491B680591FA3A7A
:10571000A5F8BC21002203F0040385F8BE21FEF7A2
:10572000DCBBAD4A049B1F68138823F0040313807D
:10573000012307F4805784F82130FFF711BAA74EF0
:10574000D6F800E04B00BEF1000F07D05F1800EB69
:1057500087079EF801E07F787745D4D20B44A04FAD
:10576000A04900EB8300002330603B800B60CAE758
:105770004FF006094B468FE54FF001094B468BE58C
:105780004FF002094B4687E54FF003094B4683E58E
:105790004FF004094B467FE54FF005094B467BE58A
:1057A000914B92491A684FF47A73B3FBF2F3C3EB4F
:1057B000431203EB8203049A1268DB001206A1F87D
:1057C000B43000F1E680834B05931B685F0700F15E
:1057D000D780049B1B6803F00403FEF77EBB002107
:1057E000BB2A109100F08081B72A00F07981BE2A8F
:1057F00000F07481BD2A00F04D81792A00F0DB8130
:105800007A2A00F0D1819E2A00F0C8819D2A00F0FA
:10581000BE81AE2A00F00182AD2A00F0F781EF2AA6
:1058200000F0EE81FD2A00F0E581FB2A00F0DC812A
:10583000FE2A00F0D381F72A00F08E817B2A7EF4C5
:1058400046AB4FF4FA61022005F06CF9FEF73FBB5E
:10585000674B00220120674D67492A700B6009F0F1
:1058600005FEFEF734BB049B64491B680A60594A75
:10587000059203F00403FEF730BB102009F026FE6A
:10588000202009F00BFE5E494E4D081F1CF0D8FC8D
:105890005C4B02221A7095F80832002B00F03B8115
:1058A0002688FEF751BF00273946524B09915B7895
:1058B000BB423FF4B5AADFF87481384605F00CFA14
:1058C00098F8023009991BB1C9B20C2025F0F8F8FC
:1058D0000137FFB2D6E64C4B01220220BBE74B4A10
:1058E0004B4B528993ED007A07EE902AF8EEE77A57
:1058F000B0EEC77AB4EEE77AF1EE10FA7FF5D7AEE4
:1059000093ED017AB0EEC77AF4EEC77AF1EE10FAB1
:105910007FF7CDAEB3063FF5CDAE202009F0D6FD22
:10592000284D97E80C0005F5017105F50070C5F8E4
:105930000022C5F804321CF083FC324B01221A709D
:10594000A9E7102009F0AAFD2E4B268883F80080D5
:105950004FF00108A5E6CFB2A7E7202009F09EFD91
:10596000284B184D00221A7095E72A4B022203207B
:1059700071E729490978032900F0C4801946B9E67E
:10598000049B264A1B680A21118003F00403FEF7DA
:10599000A4BA234B1B789B077FF515AF214B1B7DCA
:1059A000042B7FF610AF1CF0D5FB0CE7049B1E4ABE
:1059B0001B684FF4C8711180064A059203F0040376
:1059C000FEF78BBAC022002070A8002010410020F2
:1059D0003C03040858AD0020788F0020F0250020FB
:1059E0008E26002090260020E8A6002044AE00204D
:1059F000EE920020F191002000920020AC3A0020AD
:105A0000A45000205E5000203C930020F85000205D
:105A1000F04F00208A930020508F0020F2AD00202C
:105A20005CAD002060AD0020F4AD00200A940020A1
:105A300010F05CFBF4F752FC10F040FBF8F7A2FD0D
:105A4000012009F013FD95F8BA21FFF725BA95F862
:105A5000C021002A40F0938095F8C23183F0010301
:105A600085F8C231002B40F085800C2009F0E6FB60
:105A7000FEF72DBA002E3EF4E6AB6B4D95F8B9312A
:105A8000002B3EF4CFA909F0BDFB002385F8B93106
:105A9000FEF7C8B94FF6FE73644A654896890590CB
:105AA000D089334401449381D18110F01FFBF4F776
:105AB00015FC10F003FBF8F765FD012009F0D6FC9A
:105AC000049BB5F8BC211B68FA3A0021A5F8BC215B
:105AD00003F0040385F8BE11FEF7FFB90223DBE7EC
:105AE0000B464FF6FE71D7E70B460221D4E7002B99
:105AF000C3D05049504A09684FF47A7000FB031331
:105B00001360BAE709F07EFBB5F9BC21FBE503237E
:105B10000593FEF73BBD4FF00108FFF771BB0F2067
:105B2000099224F0CDFFDAF8FC01099A73E50E2002
:105B300024F0C6FFDAF8FC01FFF7F9BB1120099247
:105B400024F0BEFFDAF8FC01099AB6E40D200992B0
:105B500024F0B6FF099A49E50021042004F0E2FF91
:105B6000FEF7B5B9304D07F0E5FB002385F8B931F4
:105B7000FEF758B90B2009F061FBFEF7A8B92C4AD3
:105B800085F8C01185F8C1010592FEF7A6B900217C
:105B9000FF2026F097FC95F8BA213AE6012026F07E
:105BA00091FC95F8BA2131E6244A137A43F00103B7
:105BB0001372FEF78CB9214A137A23F00103137292
:105BC000FEF785B9172024F07BFF1DE41020099211
:105BD00024F076FFDAF8FC01099A83E4002103201F
:105BE00004F0A0FFFEF773B90021022004F09AFF31
:105BF000FEF76DB90021012004F094FFFEF767B9AC
:105C00000021084604F08EFFFEF761B9FF21002055
:105C100026F058FC95F8BA2101E60121002026F073
:105C200051FC95F8BA21F7E5C0220020FC4C002079
:105C300058AD00200CAE0020A83A0020845300206C
:105C40002DE9F04F2DED0A8B404B1B7893B0012BC3
:105C5000039001F0C4803E4C94F80021002A41F0EA
:105C6000CF80072B01F0D6804FF0000ADFF8ECB0B0
:105C7000DBF8043058469847002800F06F81BBF8E5
:105C8000B46000228BF85520002E40F06887BBF9E5
:105C90003C50DBF82410BBF93E00DBF82820BBF9B0
:105CA0004030691ACBF830102A490191821ADBF88A
:105CB0002C00CBF834200D461B1A9BF85610CBF85D
:105CC00038300BF130000FF0BBFF2B68990040F12A
:105CD000E980DBED0D5ADBED0C7A1F4A94ED416A49
:105CE000D4ED426A94ED437AD4F810311268B8EEDC
:105CF000E58ADBED0E5AF8EEE77AF8EEE58A013335
:105D000077EE867A38EE268A78EE878A9342C4ED5B
:105D1000417A84ED428AC4ED438AC4F8103101F01F
:105D2000FD820A4B1E78142E02F0B1840023D4F8B1
:105D300018510293062D00F2A880DFE815F0071332
:105D4000F6121B128B1211003114CA13F44E0020EC
:105D5000CC240020F8A600202443002044AE0020DC
:105D6000D74B1A78D4F81C71DFF8BCE39FEDD57AD5
:105D7000F8000EEB000383ED007A002A7AD0D249B6
:105D8000B0EE476AF0EE476A0023F1EC017A013386
:105D900067EEA77A05EE903AB4EEE77AF1EE10FAE4
:105DA000F8EEE55AB8BFB0EE677A9A4276EEA76A87
:105DB000A7EEA56AE9D1F5EEC06A0EEB0003F1EE9D
:105DC00010FA83ED007A55DDC6EE265ABF4BC04A65
:105DD0001288F7EE007A75EEE75AD3ED007A65EE99
:105DE000A77AFDEEE77A17EE903A812B43F32783EB
:105DF0009342A8BF134607EE903AF8EEE77AB54B08
:105E0000C11903EB810393ED057AD3ED003A93EDCD
:105E1000066A93ED014AD3ED046AD3ED034A93ED8C
:105E2000025AA3EEA77AA4EE276A66EEC76AA7EE27
:105E3000646ABDEEC77AE5EE276A17EE101A81296B
:105E400083ED056AC3ED066A43F3F6828A42A8BF72
:105E50000A4607EE902AF8EEE77AFCEEE77ACDEDF7
:105E6000047ABDF810300EEB0002938017B9132EA0
:105E700003F0B687152E42F0CF817044DFF8AC8274
:105E8000838828F81730D4F81851934B013583FBD9
:105E900005235A19EB17C3EBA203C3EBC303ED1A97
:105EA000C4F818518D4B1B78002B01F0EF808C4DFE
:105EB000CDF808A0DFF87882DFF87092DDF804A052
:105EC00005F2DC670026874BDBED087A1B78172B81
:105ED00001F04E8495ED007AB8EEC78A082B28EEC3
:105EE000278A07D1B0EE480A019326F0ADFC019B4A
:105EF00029F81600DAF8002092000BD5002E04F0E5
:105F00001981B0EE480ADBF8783707F1700098473E
:105F1000B0EE408AB0EE480ADBF89836A7F1700080
:105F20009847DBF80837384698476E4B1B78032BA9
:105F3000B0EE408A01F0FB83D5F85C06DBF8B830A0
:105F4000B0EE480A98470136032E07F12407A8EC63
:105F5000010A05F10405B6D1DDF808A0614B1F78F0
:105F6000072F00F0BC8694F828310493002B40F0F2
:105F7000C4865D4B5B79002B40F0EB850123594AC9
:105F800084F828311278072A01F0848600230693CA
:105F9000564B94ED4C9A93ED007A554BDFF8948173
:105FA000D3F800A0534B0293F7EE007A37EEC9BA4C
:105FB00008F11C032BEE07BA0025B4EEE7BAF1EEA8
:105FC00010FA0593D4ED4BBA4B4BDFF86CB1DFED13
:105FD0004B8A9FED4BAADFED3BAADFED4A9ADFF833
:105FE0005C91494F019388BFB0EE67BA2E46474B8C
:105FF00098ED008A2B44D3ED007AF5EE407AF1EE6D
:1060000010FA17D0424B2B44D3ED006A38EE667A73
:10601000B0EEC76AF4EEC67AF1EE10FA08D5B5EE26
:10602000C07AF1EE10FACCBF37EEA68A36EEE78AD8
:1060300083ED008A374B1A88930700F08180022E87
:106040007ED0354B9AF82E1033F9163007EE103A01
:10605000059B07EE901A2B44F8EEE76AB8EEC77A74
:10606000D3ED007A4B42A6EEA77A700007EE903A85
:10607000F8EEE77AB4EEE77AF1EE10FA0AD407EE1A
:10608000901AF8EE677AF4EEC77AF1EE10FA88BF4C
:10609000F0EE477A214B22490344085EB3F90C30F5
:1060A000C01A07EE100AB8EEC77AD007E7EE687A92
:1060B00040F12B861B4B93ED008A27EE888A3FE048
:1060C0002A43002000000000CC2400202C430020A4
:1060D0002843002060450020932449921C4300205F
:1060E00074AE0020F44E0020D4A60020E45A002014
:1060F00000920020E8A600209C420020CDCCCC3DA0
:10610000AE47813F0000C842A8420020D85A002074
:106110000C2600204A8F002018260020FC4C00206E
:106120003CAD0020C05A002048450020F84E002019
:10613000ECA600200026002034560020B4420020A7
:10614000029B94F868212B44D3ED01CA38EE6CCA47
:10615000002A3DD0D34BD4F86C2103991B688A1ACE
:106160009A4235DD9AF84830022B01F0CA85022E9A
:1061700003F06787CC4B1B68990740F16E87CB4BC8
:10618000CB49DFF8A0E331F916C09EED008ADFF8B5
:1061900098E3C7ED00AA03EB460028EE288AB0F981
:1061A0000C00A0EB0C0007EE900AF8EEE77ADEF8A0
:1061B000000027EE888A904238EE6CCAC1F28380D4
:1061C000F7EE007AB4EEE79AF1EE10FA01F15280A0
:1061D000B84B2B4493ED000A019B2BEE800A022E54
:1061E00020EE0C0AA3EC010A019303F05287B24B94
:1061F0009BED007AD3ED007AB04BD7ED006A93EDBA
:10620000006AAF4B67EE277A2B4427EE8B7AD3EDEB
:10621000007A67EE277AF0EE665AECEE275AB1EE76
:10622000467AF4EEC75AF1EE10FA08D4F4EEC65AE4
:10623000F1EE10FA8CBFB0EE467AB0EE657A94EDCE
:106240004C6AF7EE007AB4EEE76AF1EE10FAACBFF2
:106250000123002343B1F0EEE66AF0EEC77AF4EED4
:10626000E67AF1EE10FA01D587ED007A022E03F0FE
:10627000E186944A944B52F826001B68B0EE6C0AF3
:106280009847924A924B52F826001B6898479AF812
:10629000373023B18F4B1B88002B00F0C085B0EE48
:1062A0006A8A8D4B9BED007A38EE400A2B4493EDC1
:1062B000008A83ED000A9AF8483030EE480AC0EEB2
:1062C000077A2BB3854B1B78DB0721D5B7EE007A15
:1062D000B4EEC79AF1EE10FA04DB94F86831002BA3
:1062E00000F06F87D4F86C31039AD31A6D4A1268A4
:1062F0009A420DDD7A4B93ED007AB0EECCCAB4EE43
:10630000C7CAF1EE10FA40F1FA87002384F8683129
:10631000744B94F878212B4493ED007A2BEE877A16
:1063200067EE277AC9ED007A32B9019BC7ED00AA62
:1063300043ED01AAC9ED00AA0136032E08F10408B5
:1063400009F1040907F1040705F104057FF44FAED4
:10635000654B1B78072B01F02182012B01F09F84F4
:106360000023029394F88031002B40F0A1855F4B0D
:106370005F4A1B68126813F4805C92F82C2040F08E
:10638000AE865C495C4891ED006A408B5B4984EDC8
:10639000646A91ED007A5A4984ED657A07EE900AB5
:1063A000F8EEE76AD1ED037A564984ED626A37EE7A
:1063B000467A77EEE67AD1ED006A84ED617A0121C2
:1063C00084F89811C7EEA65A4F48504990ED005AEC
:1063D0004F489FED506A90ED004A4F48DFED4F6AFD
:1063E000D0ED004A91ED007A35EE045AF7EE007ACE
:1063F000F4EEE75A35EE245AF1EE10FA88BFF0EECB
:10640000675A25EE065AF4EEE65AB1EE476AF1EE07
:1064100010FAB4EEC65AB8BFF0EE665AF1EE10FAB2
:10642000C4ED675A01F10780B4EEC75AF1EE10FAD5
:1064300088BFB0EE475A3449DFED366AD1ED017AB4
:10644000334991ED014A344977EE847AD1ED014A1E
:1064500077EEA47A67EEA67AB4EEE76AF1EE10FA68
:1064600008DCB4EEE77AF1EE10FA8CBFB0EE676AA2
:10647000B0EE476A2449DFED276AD1ED027A24495C
:10648000D1ED024A264977EEA47A91ED007A67EEC3
:10649000A67AB1EE473AF4EEC37AF1EE10FA4ED492
:1064A00044E000BFEC5A002058AD0020FC4C002016
:1064B0003CAD0020945A0020A8000020085B00207A
:1064C000A05A00203C56002038560020905600204C
:1064D0008C5600204A8F00203C260020644F00206C
:1064E000F85A0020AC5A0020F44E0020F8A60020F4
:1064F000009200207846002070A80020B85B0020A1
:10650000F04F0020CC5B00209C4200200C5B002060
:10651000A84200206F12833AB4420020000000001D
:10652000105B0020C05A0020E85A0020F4EEC77A21
:10653000F1EE10FA8CBFB0EE473AB0EE673AED4993
:10654000497809B9B1EE433A002A41F04B82F7EE9F
:10655000003ADFF8C8B39BF80020002A02F0458219
:10656000E549DFEDE67AD1ED024AD1ED016A91ED20
:10657000037A66EE244AE5EE264AE3EE074A63EE26
:10658000A44AF4EEE74AF1EE10FAB4BFB0EE674A5F
:10659000B0EE644A98BFF0EE647A012ACDED0A4A63
:1065A00002F0448291ED067AD1ED052AD1ED076A19
:1065B00026EE077AA5EE227AA3EE267A23EE877AD4
:1065C000B4EEE77AF1EE10FAB4EEC47A8CBFF0EED6
:1065D000676AF0EE476AF1EE10FA88BFF0EE676A7C
:1065E000B4BFF0EE447AF0EE477A022A8DED0B7AD2
:1065F00000F0DE8091ED0A7AD1ED092A91ED0B4A87
:1066000026EE077AA5EE227AA3EE047A23EE877AA5
:10661000B4EEE67AF1EE10FAB4EEE77A8CBFB0EEA3
:10662000664AB0EE474AF1EE10FA98BFF0EE446ABF
:10663000A8BFF0EE477A032A8DED0C7A00F0B880FF
:1066400091ED0E7AD1ED0D2A91ED0F4A26EE077AE3
:10665000A5EE227AA3EE047A23EE877AB4EEE67AE8
:10666000F1EE10FAB4EEE77A8CBFB0EE664AB0EE07
:10667000474AF1EE10FA98BFF0EE446AA8BFF0EE78
:10668000477A042A8DED0D7A00F0928091ED124A3E
:10669000D1ED112A91ED137A26EE044AA5EE224A95
:1066A000A3EE074A23EE844AB4EEE64AF1EE10FA6E
:1066B000B4EEE74A8CBFB0EE667AB0EE447AF1EE03
:1066C00010FA98BFF0EE476AA8BFF0EE447A052AA8
:1066D0008DED0E4A6CD091ED164AD1ED152A91ED53
:1066E000177A26EE044AA5EE224AA3EE074A23EEC5
:1066F000844AB4EEE64AF1EE10FAB4EEE74A8CBFF3
:10670000B0EE667AB0EE447AF1EE10FA98BFF0EE91
:10671000476AA8BFF0EE447A062A8DED0F4A47D0AB
:1067200091ED1A4AD1ED192A91ED1B7A26EE044A11
:10673000A5EE224AA3EE074A23EE844AB4EEE64AC7
:10674000F1EE10FAB4EEE74A8CBFB0EE667AB0EE26
:10675000447AF1EE10FA98BFF0EE476AA8BFF0EE67
:10676000447A072A8DED104A22D091ED1E7AD1EDA0
:106770001D2A91ED1F4A26EE077AA5EE227AA4EE95
:10678000037A27EE237AB4EEE67AF1EE10FAB4EE4D
:10679000E77A8CBFB0EE666AB0EE476AF1EE10FAA7
:1067A0008DED117A98BFF0EE466AA8BFF0EE477AF9
:1067B00077EEE67AF7EE006AF4EEE67AF1EE10FA9A
:1067C000C4ED4C7A43F3A88286EEA77A022ADDED67
:1067D0000B7A67EE244A67EE877ACDED0A4ACDED53
:1067E0000B7A2DD0DDED0C7A67EE877A032ACDED9A
:1067F0000C7A25D0DDED0D7A67EE877A042ACDED8F
:106800000D7A1DD0DDED0E7A67EE877A052ACDED83
:106810000E7A15D0DDED0F7A67EE877A062ACDED78
:106820000F7A0DD0DDED107A67EE877A072ACDED6D
:10683000107A05D0DDED117A27EE877A8DED117A89
:106840002F49096811F0805800F0A387F6EE005A2E
:10685000C4ED675A002A02F0BF8094F99801D4ED84
:10686000654A284D284994ED646A284E284FDFF880
:10687000B0E0B5F81AA0C978B6F9069097ED005ABD
:106880009EF800E0D4ED616AD4ED627A07EE100A5A
:10689000FDEEE44A1F4814EE905A0078FDEEC64A19
:1068A00003F0100603F4800300F00107B8EEC77A86
:1068B00014EE900A0193002941F0D4800E49002E75
:1068C00040F0898791ED006A9DED0A5A124B25EE42
:1068D000866AA5EE076AB0EE675AA6EE265ABDEEA6
:1068E000C56A16EE10EA16EE106AAE45A8BF2E462F
:1068F00018E000BFFC470020385B002000000000CB
:106900006046002070A80020548F0020AC79002041
:10691000145B0020644F0020FC420020D54E002074
:10692000C8A300207045C8BF064606EE106AB8EE40
:10693000C66A012A83ED006A00F0DC8091ED046AEA
:106940009DED0B5A25EE866AA5EE076AB0EE675AF2
:10695000A6EE265ABDEEC56A16EE10EA16EE106ACD
:10696000AE45A8BF2E467045C8BF064606EE106A63
:10697000B8EEC66A022A83ED016A00F0BB8091ED91
:10698000086A9DED0C5A25EE866AA5EE076AB0EE00
:10699000675AA6EE265ABDEEC56A16EE10EA16EE46
:1069A000106AAE45A8BF2E467045C8BF064606EE23
:1069B000106AB8EEC66A032A83ED026A00F09A8074
:1069C00091ED0C6A9DED0D5A25EE866AA5EE076ADB
:1069D000B0EE675AA6EE265ABDEEC56A16EE10EA6C
:1069E00016EE106AAE45A8BF2E467045C8BF0646D3
:1069F00006EE106AB8EEC66A042A83ED036A79D0FF
:106A000091ED106A9DED0E5A25EE866AA5EE076A95
:106A1000B0EE675AA6EE265ABDEEC56A16EE10EA2B
:106A200016EE106AAE45A8BF2E467045C8BF064692
:106A300006EE106AB8EEC66A052A83ED046A59D0DC
:106A400091ED146A9DED0F5A25EE866AA5EE076A50
:106A5000B0EE675AA6EE265ABDEEC56A16EE10EAEB
:106A600016EE106AAE45A8BF2E467045C8BF064652
:106A700006EE106AB8EEC66A062A83ED056A39D0BA
:106A800091ED186A9DED105A25EE866AA5EE076A0B
:106A9000B0EE675AA6EE265ABDEEC56A16EE10EAAB
:106AA00016EE106AAE45A8BF2E467045C8BF064612
:106AB00006EE106AB8EEC66A072A83ED066A19D098
:106AC00091ED1C6A9DED115A65EE865AE7EE055A66
:106AD000E6EEA57AFDEEE77A17EE901A8D42A8BF92
:106AE0000D468842C8BF054607EE905AF8EEE77A91
:106AF000C3ED077A2FB922B19200D649D64825F0C6
:106B00002FFDD64B1B68002B40F0AE84D44B1B7876
:106B100093B19BF8000060B1CF4ED24F0025E8B290
:106B20003B68B6EC010A98479BF8000001358542A6
:106B3000F5DBCD4B1B689847CC4B1B78072B00F03F
:106B40004286012384F8003113B0BDEC0A8BBDE806
:106B5000F08FC74B1B78013BDBB2FFF710BAC54B78
:106B600002934FF47A751B68B5FBF3F3C3EB43153F
:106B7000C149DFF8388391F80190BC49B8F90600A3
:106B80000F7803EB8503DD00ADB2AE4201F09386D2
:106B9000DBF88810BBF93CE0DBF86C304A1C07EEF0
:106BA00090EA7344012ACBF88820CBF86C30F8EED9
:106BB000E77A01F08D86DBED1E5ADBED206A07EEE9
:106BC000102A37EEE56AB8EEC75A012E86EE057A2E
:106BD00037EE257A77EEC77A8BED1F7AE7EE866A75
:106BE0008BED1E7AF0EE667ACBED216ACBED206A52
:106BF00002F05E80DBF89C10BBF93EE0DBF8703001
:106C00004A1C07EE90EA7344012ACBF89C20CBF88B
:106C10007030F8EEE77A01F07686DBED235ADBED93
:106C2000256A07EE102A37EEE56AB8EEC75A012E3C
:106C300086EE057A37EE257A77EEC77A8BED247AE1
:106C4000E7EE866A8BED237AF0EE667ACBED266A64
:106C5000CBED256A02F05580DBF8B010BBF940E0BF
:106C6000DBF874304A1C07EE90EA7344012ACBF833
:106C7000B020CBF87430F8EEE77A01F05F86DBEDF8
:106C8000285ADBED2A6A07EE102A37EEE56AB8EEDD
:106C9000C75A012E86EE057A37EE257A77EEC77A47
:106CA0008BED297AE6EE276A8BED287AF0EE667A8C
:106CB000CBED2B6ACBED2A6A02F04C80A8F80600D7
:106CC000BBF8B430694A013B1778ABF8B43002998D
:106CD0000023072F4B608B60CB607FF444A9F7F74C
:106CE00031FFDFF8C88194F828310493A0EB0A0043
:106CF000A8F80000002B3FF43CA9013B84F82831A0
:106D000013B0BDEC0A8BBDE8F08F94ED577AB1F962
:106D10000000D4ED586AB1F902E0584AF4EEC76AAF
:106D200080EAE0738EEAEE71A3EBE073F1EE10FA05
:106D3000A1EBEE71B4BFB0EE476AB0EE666A8B426B
:106D4000B8BF0B4607EE103A1378B8EEC77A27EEB5
:106D5000287A002B40F00682494BD3ED005AF4EE1E
:106D6000CA5AF1EE10FA40F19087B7EE005A75EE6C
:106D7000654ADFED446A9FED445A444B36EEC77ACC
:106D800024EE855AD3ED006AE7EE055A65EEA65A61
:106D9000F5EEC05AF1EE10FA40F2F784C9EEA56A9A
:106DA000B7EE007AF0EE475AE6EE665AF0EE656A04
:106DB000F4EEC76AF1EE10FA88BFF0EE476AF5EE1E
:106DC000C06AF1EE10FAB8BFF0EE6A6A304B93ED8C
:106DD000007A67EE877AA7EEA68AFFF7B1B92D4B46
:106DE0002D4C19682D4ADFF8C48094F80031C96928
:106DF0001288A8F80010A8F80220002B3EF434AF47
:106E00000FF0ACFD002384F80031184B1B78072BE2
:106E10007EF42AAFF7F796FE8246FEF727BF204B97
:106E2000204A2B4493ED007AD2ED007A1E4B67EE98
:106E3000277AF7EE006AF4EEE67AF1EE10FA93EDB7
:106E4000007A88BFF0EE667A67EE877A27EE888A46
:106E5000FFF727BA185B0020FC4200202C560020C8
:106E6000D0A60020BCA30020C4A30020F44E002024
:106E7000905A0020E8A60020D4A60020CC5A00207A
:106E8000D45A002000003443610BB63BC85A00209E
:106E9000C45A0020D0910020CC240020E43F0020E0
:106EA00028260020BC5A0020B85A0020F84E0020A6
:106EB000D94BDFF8B8B31B789BF80020DD077FF5CE
:106EC0001AAE002A3FF41DAED4ED583A94ED574A5D
:106ED000D24BD4ED627A93ED005A94ED617AD4ED01
:106EE000555A94ED546ACE49CE4BF4EEC43AF3EEC3
:106EF000046AF1EE10FA77EEA64A00F15B8791ED95
:106F0000026A26EE656AB0EE674AA6EE074AB4EE5C
:106F1000E44A34EE666AF1EE10FA48BFB0EE456A14
:106F2000012A83ED006A3FF4ECAD91ED066A26EE8E
:106F3000656AB0EE674AA6EE074AB4EEE44A34EE5C
:106F4000666AF1EE10FA48BFB0EE456A022A83ED98
:106F5000016A3FF4D6AD91ED0A6A26EE656AB0EE9D
:106F6000674AA6EE074AB4EEE44A34EE666AF1EEEA
:106F700010FA48BFB0EE456A032A83ED026A3FF477
:106F8000C0AD91ED0E6A26EE656AB0EE674AA6EED8
:106F9000074AB4EEE44A34EE666AF1EE10FA48BFEE
:106FA000B0EE456A042A83ED036A3FF4AAAD91ED81
:106FB000126A26EE656AB0EE674AA6EE074AB4EE9C
:106FC000E44A34EE666AF1EE10FA48BFB0EE456A64
:106FD000052A83ED046A3FF494AD91ED166A26EE1E
:106FE000656AB0EE674AA6EE074AB4EEE44A74EE6C
:106FF000666AF1EE10FA48BFF0EE456A062AC3ED64
:10700000056A3FF47EADD1ED1A6A66EEE56AB0EE30
:10701000674AA6EE874AB3EE046AB4EEE44A74EE19
:10702000466AF1EE10FA48BFF0EE456A072AC3ED52
:10703000066A3FF466ADD1ED1E6A66EEE55AE5EEEE
:10704000877AF4EEE74A77EEC67AF1EE10FAC8BF17
:10705000F0EE457AC3ED077A53E5734BC7ED00AA0E
:107060001B689342BFF6ACA8704B1A88002384F8C3
:107070006831002A41F015846D4A6E4B117818680A
:1070800081F00101F2F7EEFCFFF7A2B86A4EDFF8DB
:10709000E08106F24C7506F5F767F6EC017A9BED98
:1070A000080ADBF87837F8EEE77A284627EE800AF8
:1070B0009847A5F1E000DBF898369847A5F17000F5
:1070C000DBF808379847D6F85806DBF8B830984709
:1070D0002435AF42A8EC010ADFD1FEF73FBF4E498D
:1070E0000978C80703D45549098BA4F88C11544971
:1070F0005448098890ED037A07EE901AF8EEE77A83
:10710000B4EEE77AF1EE10FA40F20C864E480088B1
:1071100007EE900AF8EEE77AB4EEE77AF1EE10FAAD
:10712000C0F2D08549484A49D0ED006A91ED006A25
:107130004848C4ED646ABCEEC75A76EE665A15EE4E
:10714000101AC4ED626AC4ED615A84ED656AA4F850
:107150008C110121D0ED006A84F8981177EE677ADE
:10716000FFF730B93C4B93ED005AB5EEC05AF1EE43
:1071700010FA40F30A83394BD3ED006AF5EEC06A8A
:10718000F1EE10FA40F3018336EEC77A66EE695AE3
:1071900087EE266AC5EE856AB7EE007AB4EEC76A56
:1071A000F1EE10FA88BFB0EE476AB5EEC06AF1EEB4
:1071B00010FA76EE876AB8BFB0EE6A6A66EE266AA3
:1071C000F6E5274A92ED007AF0EEE76AF4EEC76A38
:1071D000F1EE10FA7FF786A8224A92ED007AF0EEDF
:1071E000CC6AF4EEC76AF1EE10FA7FF77BA81E4A6C
:1071F00098ED007AD2ED006AB0EEC77AB4EEE67A86
:10720000F1EE10FA7FF56EA801220399C4F86C1113
:1072100084F86821FFF76AB8644F0020145B0020EF
:10722000385B0020FC420020E85A0020C4B7002050
:10723000C6B70020C8B7002074AE002070A8002098
:10724000D05B0020F04F0020D25B0020BC5B002010
:10725000B85B0020D85B0020C85A0020D05A00201C
:10726000FC5A0020F85A0020005B0020D54E002078
:10727000ECA600200299724BD1ED017A93ED007AD1
:10728000F0EEE77AF4EEC77AF1EE10FA7EF5A0AFF1
:10729000D1ED027AF0EEE77AB4EEE77AF1EE10FA89
:1072A0007EF796AFD1ED037AF0EEE77AB4EEE77AA7
:1072B000F1EE10FA7EF78CAF624B1B689A077FF5F0
:1072C000D3AE6149614BB3F90C20B1F900E06048DD
:1072D000AEEB020E00688EEAEE72A2EBEE72824214
:1072E000BEF676AFB3F90E30B1F90220D21A82EAB7
:1072F000E273A3EBE27398427EF76AAFB4E6554BB4
:1073000098ED007AD3ED006AB0EEC77AB4EEE67A73
:10731000F1EE10FA7EF7FCAFFEF7F7BF07EE103A7A
:107320004D4BDFF840811B78C4F81061B8EEC77A86
:10733000F7EE006A132B86EE879AB8F90400B4F8CA
:1073400014519BED080A01F03882444B444A93EDF6
:10735000001A93ED053A93ED122A93ED176AD3EDD7
:10736000091A93ED0E4AD3ED015AD3ED063A93ED87
:107370000A7A93ED0F5AD3ED132AD3ED186AD3EDA1
:10738000044AD3ED030A67EE897A69EE288A29EE6A
:10739000088AA1EE273A02EB85060021A2EE286AB0
:1073A000C4F80411C4F80811A1EE884AE5EEA73A22
:1073B000A7EE085A93ED167AD3ED0D5A93ED021A03
:1073C000D3ED0C1A86ED003AE2EEA86A64EEC34AE9
:1073D00027EE467A93ED0B2AD3ED152A86ED204A47
:1073E000E0EEC33A65EEC45A93ED143AC3ED053AA4
:1073F000E1EE274AF0EE477AA1EEC45AE2EE085ACF
:10740000E2EEC66AE3EE287AC3ED064A83ED0E5A31
:10741000C3ED0F5A86ED406AC3ED176AC3ED187AC3
:10742000C4F80C11013505F01F05A4F81451A8F893
:107430000400FEF776BCB0EE465AFEF7FCBF00BF74
:10744000F45A002058AD00203CAD0020FC4C002038
:10745000F05A0020005B0020F44E0020CC450020B4
:1074600048430020F84E0020B44B1B78192B07D856
:107470000121B34A01FA03F31A40002A41F078844B
:10748000B04BB14EB14F01931B689D061CD5FB7AE2
:10749000FF2B04D0AE4A12789A4201F2F380B7F97A
:1074A0000880FB7DA6F80080FF2B04D0A84A127844
:1074B0009A4201F2E280B7F914507580082023F057
:1074C000A1FA002840F03586B7F90600B6F900C0E9
:1074D000B6F902E0B7F91210B7F91E20B6F9045058
:1074E000B7F90430B6F906806045A8BF604671451B
:1074F000A8BF7146AA42A8BF2A469C45A8BF03461A
